:020000040800F2
:10000000F0FF001099B706084D3D060879E9010890
:1000100039B8060839B8060839B8060800000000E3
:10002000000000000000000000000000513D060834
:10003000553D060800000000593D0608D19B000808
:1000400039B8060839B8060839B8060839B80608B4
:1000500039B8060839B80608D5BD0008DDBD000866
:10006000E5BD0008EDBD0008F5BD000849B8000871
:100070005DB8000871B8000885B8000899B8000894
:10008000ADB80008C1B8000839B8060839B8060884
:1000900039B8060839B8060839B80608FDBD0008A1
:1000A00055D00008B5CF000865D00008A5CF0008DE
:1000B000DDCF0008EDCF0008FDCF000891AD0008AE
:1000C0002DC7000899AD000831C7000839B80608E7
:1000D00039B80608E1EF000809F1000831F200081C
:1000E00005BE000839B80608957E060875D00008D8
:1000F0002DD0000885D000081DD00008D5B8000814
:1001000039B8060839B806080DD0000839B806080D
:1001100059F3000881F4000839B8060839B8060810
:10012000E9B80008FDB8000811B9000825B90008B1
:1001300039B9000839B8060839B8060839B80608C8
:1001400039B8060839B8060839B806085D3D06080A
:100150004DB9000861B9000875B90008A9F5000893
:10016000A1AD000835C7000839B8060839B8060837
:1001700039B8060839B8060839B8060839B8060883
:0801800039B8060839B8060879
:1080000010B40C4B4FF0E02C1A68DCF8180019681B
:108010008A42F9D159688842F6D89C684FF47A713F
:1080200001FB04F31B1AB3FBF4F35DF8044B01FBF3
:1080300002307047C81A0020074BD0F8E4105B6884
:10804000D0F8F0205B1A9A42B8BFC0F8F030012394
:1080500080F81C3100207047001000E0C04B00EB9E
:10806000800103EBC101F0B5CA685268B2F814E0B0
:108070001EF0010F4FEA800C73D15FFA8EF4A50752
:1080800042D5BFF35F8F91F82840012CE5B200F094
:10809000DC80118BBFF35F8F0CEB000103EBC101A0
:1080A00091F82840022C00F0F2800CEB000103EB69
:1080B000C10191F82840032C07D191F82A1021B171
:1080C00093F88510002940F0F280918889B241F43C
:1080D0008061918093F984400CEB000103EBC101B6
:1080E00091F828100131A1420DD1002183F88510AB
:1080F00093F88610002940F0C380604403EBC00071
:10810000002380F82530F0BD67071FFA8EF593F93C
:1081100084E05FD414F0400400F0D280148A0D6B28
:10812000E4B205F80E405FFA8EFE91F828600EF179
:10813000010149B2CD1CAE4283F884100C4600F018
:1081400024810CEB000503EBC50595F82850A942E6
:10815000C2D10EF1020E4FFA8EFE83F884E074460F
:10816000BAE7B2F800E02EF4006E4FEA0E4E4FEA86
:108170001E4EA2F800E01488A4B244F48064148077
:1081800091F82A40002583F88450002C4CD093F8B5
:108190008540002C44D0012183F885100CEB0001B0
:1081A00003EBC10191F82810022904D1118889B28A
:1081B00041F4006111800CEB000103EBC10191F867
:1081C000261041F001011182844403EBCC0393F8A3
:1081D0002830F0BD91F82A50012483F8864093F8A6
:1081E0008540002D00F08780002C40F088800CEB4B
:1081F000000103EBC10191F82910002900F0A680CD
:1082000011880EF1010489B24FFA84FE41F4007125
:1082100083F884E011801188CE05FCD474465BE7B6
:1082200091F82710FF29B6D00CEB000103EBC10138
:1082300091F8264004F0FE04148291F82720FF2ACA
:10824000C2D0FF2283F88420BEE791F82A100029CB
:108250003FF41FAF93F8851000293FF41AAF11883F
:1082600021F480610904090C1180BFF35F8F118B29
:10827000118883F8865089B241F40071118024E797
:10828000918821F440710904090C918035E791F837
:108290002A1000293FF409AF93F8851000293FF414
:1082A00004AF118821F480610904090C11809188C0
:1082B00021F480610904090C918093F984400BE753
:1082C0002D06ABD5BEF1FF3F66D0CC6A14F80E5038
:1082D000EDB2158291F828100EF1010464B2A142AA
:1082E00083F884407FF4F8AE918821F4806109041A
:1082F000090C9180F0E6002C3FF479AF80E791F80B
:1083000028600F6B5FFA8EF4651C022E6DB229D9BE
:10831000168826F480663604360C1680168AF6B265
:1083200007F80E6002344FFA84FE0C6B118883F854
:1083300084E089B241F400711180118AC9B261559B
:10834000918889B241F48061918064E7118889B293
:1083500041F480711180012183F885105BE700BF33
:10836000C81A00201688B6B246F400761680168A1F
:10837000F6B207F80E6003344FFA84FE0C6B118AD4
:1083800083F884E0C9B2615545E7958825F4806596
:108390002D042D0C9580D4E683F8844091F8274075
:1083A000E4B2148291F82A4024B991F828100029E7
:1083B0007FF40AAF918821F480610904090C91804F
:1083C00002E700BF10B404698269E4684168146080
:1083D00000234024C2E90234446993630C31C2E9AA
:1083E0000433C2E90633C2E90833C2E90A33C2E9F9
:1083F0000C33516084B1C269C2E90233C2E904336B
:10840000C2E90633C2E90833C2E90A33C2E90C33D0
:10841000E0689363C2E900015DF8044B704700BF58
:10842000D0E9001300221A60037D1F2B07D9203BDF
:10843000202202FA03F343F01803CB607047202296
:1084400002FA03F343F018038B6070471B4B01687B
:1084500003F57D7C02E02C3363452CD01A688A42F8
:10846000F9D170B593F804E0427996450BD02C33DE
:10847000634505D01A688A42F4D02C336345F9D19C
:108480004FF0FF3070BD9E468468DEF80C50A54268
:108490004FF0000208D00132032A0EF10C0EE6D094
:1084A000DEF80C50A542F6D1DEF81050C668B54291
:1084B000F1D150B270BD4FF0FF307047DCD60608E6
:1084C000002A4FEA014C30B503460ABFE6468E4605
:1084D0008C4600F1C005002419689A6841EA0C0135
:1084E00042EA0E029A60C3E900140C33AB42F3D1A6
:1084F000D0F8C030C0F8C44043EA0E03C0F8C03022
:10850000C0F8C84030BD00BF83691969B3F80CC01A
:108510000A6830B49C6822F0010224680A60A289CB
:1085200092B222EA0C02A281027D00681F2A06D9BB
:108530004568203A082494402C4245D0FEE705685F
:10854000082494402C42F9D1202404FA02F28260DB
:10855000264A1278002A35D01A7E012A39D0D3F85B
:10856000F4200132C3F8F420EFF31181502282F39A
:10857000128858685C6C026822EA04029C6C2243F0
:10858000C9B2026081F31188D3E90C401A69996875
:108590001D6C096814605061D3E90E40546090600E
:1085A0000024B3F8A800D5604C62C86210680124AA
:1085B000204310601C7683F8F1408A899B8913431D
:1085C0009BB28B8130BC7047202404FA02F2C26057
:1085D000BEE7002283F8F120D3F8F8000A680130E2
:1085E00022F00102C3F8F8000A60EBE70400001073
:1085F00010B40C4C6368002B11DD002004F1080C52
:108600000146DCF8A03003F1C00259600C339342FC
:10861000FBD16368013083420CF5807CF1DC5DF8AE
:10862000044B704704000010F0B5484C04EB4012B6
:1086300092F8243403B9F0BD454B4FF08C0C0CFB81
:10864000003C93F8E86493F8E9549CF88A7082F847
:108650000A74AE424FF000024FEA401E8CF88A20A6
:108660000ED005EB450203EBC20292F8ECC40CF10C
:10867000FF37012F4FEA450259D9BCF1030F51D002
:1086800004EB0E00A0F80814EFF31182902383F39B
:10869000128890F80A34B0F8081443EA4103002124
:1086A000D2B29BB280F80A1482F311882178D0F8F4
:1086B00020441A0982EA13225A40C9B1D0F80C1496
:1086C000D4F8A040D2431B019BB202F00F0201205C
:1086D0008840134304F1C0015A0013F4004F93B2D1
:1086E00002D16268024362600C34A142F4D1F0BD51
:1086F000D0F80C14D4F8A0401B0110319BB202F04A
:108700000F0201208840134304F1C0015A0013F402
:10871000004F93B202D16268024362600C34A142FE
:10872000F4D1F0BD6F1C07F00307B742A8D02A446C
:1087300003EBC203184490F8F9140029A0D004EB0D
:108740000E03012283F80A249AE700BF04000010F8
:10875000C81A0020704700BF024B03EB401393F888
:1087600025047047040000104368B0F8502010B48E
:108770001A83EFF31182502383F312884168446C0B
:108780000B6823EA0403C46C2343D2B20B6082F368
:108790001188D0E907418268036912681C60596139
:1087A000D0E909415C60C46A9960B0F86010DC608F
:1087B0000023D1625DF8044B0376704710B4037D4B
:1087C00002681F2B09D95468203B202101FA03F3CA
:1087D0001C4215D15DF8044B70471468202101FA42
:1087E00003F31C42F6D00D494068002481F84C4543
:1087F00001685DF8044B21F001010160936070474E
:1088000006494068002481F84C4501685DF8044B36
:1088100021F001010160D360704700BFC81A002039
:10882000704700BF0B4890F83C1589B101EB41013E
:10883000002310B4490000F244501C4650F8232095
:10884000063302B114608B42F8D15DF8044B7047D7
:10885000704700BF040000100B4890F83C1589B128
:1088600001EB4101002310B4490000F244501C46C2
:1088700050F82320063302B114608B42F8D15DF822
:10888000044B7047704700BF040000100120704780
:10889000034B00EB400003EBC00393F85505704712
:1088A000040000101F4890F83C35002B39D00022FE
:1088B0002DE9F04300F244531B4E1C4D4FF0500E77
:1088C0004FF02C0C144607E053F8181B0C6090F87E
:1088D0003C150132914222DD197C0029F4D05F68F9
:1088E000B90AA1F5801105EB010952294FF0FE08E4
:1088F00098BF99F8F483EFF311898EF31288796A9F
:108900000CFB08680131C8F87815B98A89B241F0C2
:1089100001015FFA89F8B98288F31188D4E7BDE8CC
:10892000F083704704000010C81A0020DCD6060847
:1089300000EE100AB8EE400A704700BFBCEEC00A55
:1089400010EE103A98B2704708B51D2015F07EF968
:1089500008B183794BB11E2015F078F908B18379FD
:1089600003B108BD5523C38008BD5523C380F2E77A
:108970000C4B0D49DB68DB43C3F30223C3F1040353
:108980000122DBB202FA03F301EB000C1B0103F03E
:10899000F0038CF80033430900F01F00824041F8D7
:1089A0002320704700ED00E000E100E010B4037DFB
:1089B00002681F2B09D95468203B202101FA03F3D8
:1089C0001C4215D15DF8044B70471468202101FA50
:1089D00003F31C42F6D00D494068002481F8B847E3
:1089E00001685DF8044B21F001010160936070475C
:1089F00006494068002481F8B84701685DF8044BD7
:108A000021F001010160D360704700BFC81A002047
:108A1000122301480B80704788010020042301487D
:108A20000B8070479C0100201C48D0F8103AD0F809
:108A3000182A10B59B184FF01A040C8001D1184861
:108A400010BD174AD0F8140A02F1100411464FF075
:108A5000000E4FEA137CB3F1204F34BF0CF1300C01
:108A60000CF1370C81F802C081F803E002318C422E
:108A70004FEA0313EDD102F108040021030FB0F116
:108A8000204F34BF303337339374D1740232944261
:108A90004FEA0010F2D1024810BD00BF0070FF1F66
:108AA000A0010020D0E90920131A5842584170470C
:108AB00090F84F3830B53BB990F84D1890F84E38D3
:108AC0000124DAB2914200D830BDB0F8565804FA09
:108AD00003F22A43A0F856280133F2E7037902464D
:108AE00013F0010006D0D2E90731D2685B1A013ACF
:108AF00003EA0200704710B5037913F0010304463E
:108B00000ED0FFF7EBFF034650B1226A6369E168BC
:108B10009B5C0132B2FBF1F001FB1022DBB222625E
:108B2000184610BD03799B070AD5436A8269D15460
:108B3000436A02690133B3FBF2F102FB1133436272
:108B400070477047017170470379014613F00200C6
:108B500007D00B69D1E90921013B521A1A40D2B260
:108B6000981A7047C36B33B15B68426D9BB29A42EF
:108B700005D3D01A7047D0E907239A42F9D2C168C9
:108B80000A44D01A704700BFD0E909120369914224
:108B900038BFC9188A1A016C013B21B1496812FA21
:108BA00081F2934201D9981A70470020704700BFA4
:108BB000036C13B190F864007047D0E90903181AE8
:108BC000B0FA80F0400970470346C26BD96840692B
:108BD00010B452B15A6D8C1A013A005D5DF8044B25
:108BE00018BF1146C0B2596570471C6A005D04F198
:108BF000010C8C4538BF6246C0B25DF8044B1A6266
:108C0000704700BF836E70B504460D460BB19847A0
:108C1000B8B1636AA269D554636A2169226C0133D1
:108C20008B4228BF0023636252B3EFF311835022BB
:108C300082F31288226C1168C90703D5DBB283F373
:108C4000118870BD516889B291B9D4E90950854243
:108C50001CD0A6699CBF0D462169064494BF081A22
:108C6000281A80B20021D660A56284F86410506092
:108C7000116841F00101DBB2116083F3118870BD0E
:108C8000226ED36843F08003D36070BD012284F864
:108C90006420D3E7836E03B118477047F8B590F8A6
:108CA0007D30012B1CD0002A164619DD0269436A6B
:108CB00005460F46D41AB442A869A8BF34463946BF
:108CC0002246184464F076FA6B6A2A692344361BFC
:108CD000B3FBF2F1002E02FB11336B622744E9DC97
:108CE000F8BD00BF90F87D30012B0ED0036C002B37
:108CF0002CD0EFF31183502282F31288026C11689A
:108D0000C90703D5DBB283F311887047516889B274
:108D100070B491B9D0E90954A5421DD086699CBFB1
:108D20000D460169264494BF0C1B2C1BA4B20021E4
:108D3000D660856280F864105460116841F00101CA
:108D4000DBB2116083F3118870BC7047026ED36888
:108D500043F08003D3607047012280F86420DBB2C7
:108D600083F31188F0E708B519F002FC052808D84C
:108D7000054BD3F8BC370344187BBDE8084014F01A
:108D800065BF002008BD00BFC81A002070B50B4C9D
:108D900005460726013E00D170BD94F9000019F088
:108DA000E7FB031E08DBEA1861789171A178E954AA
:108DB000052BDCBFE37813730434EBE723DB0608F1
:108DC00082B01D4B1D49002201920193019B043387
:108DD0000193019B1A688B6803F00C03042B02D0EB
:108DE000082B05D0164A174BC3F8C02702B07047AE
:108DF00048684B68400203F03F0314D44A681049A6
:108E0000B1FBF3F3C2F3881203FB02F20B4B5B6876
:108E1000C3F3014301335B00B2FBF3F2094BC3F828
:108E2000C02702B070474968B2FBF3F2C1F3881360
:108E300003FB02F2EAE700BF50280040003802407E
:108E40000024F400C81A0020012343770020704753
:108E500008B503468269006BD96A02449A6101B180
:108E60008847002008BD00BF436A1B681B6A5B6817
:108E70005B78024613F0010008BF5077704700BFCF
:108E8000C2628161704700BF704700BF0430704705
:108E90000D4B93F8C827D3F8C4170244D2B283F815
:108EA000C82793F8C82701441206C3F8C41705D58C
:108EB00093F8C82782F0800283F8C827034B012269
:108EC00083F83220704700BFC81A002088010020B4
:108ED0002DE9F047154FD7F8CC57ED0A20D00026E2
:108EE000B14607F604087419D7F8D0371048D3F8FC
:108EF00028A0C7F8FC9704EBD474641010234246F2
:108F0000E102D0470F280BDD0A4B03F1100153F8A3
:108F1000042B013207D18B42F9D12546B542E2DC60
:108F2000E802BDE8F087661CF8E700BFC81A002019
:108F300098220020CC2200201A4B1968D3F814285C
:108F40008A1A322A16D8D3F828288A4200D37047C2
:108F5000D3F81C2812B31068928810B444693231D7
:108F6000224218BF42835DF8044B08BF0283C3F856
:108F70002818704793F81828D3F81C1802F001023B
:108F800019B10868898822B901830022C3F828280A
:108F9000704700224183C3F8282870473231C3F854
:108FA00028187047C81A0020084A92F81838D2F8D2
:108FB0001C2803F001031AB19188126813B91183B8
:108FC0000020704751830020704700BFC81A00205E
:108FD0004FF40070034B1060D3F838380B6000205A
:108FE000704700BFC81A002000207047012070475A
:108FF000012070470020704710B41C6994420CD3C4
:1090000094460A4661448C42996938BFA4EB0C022D
:1090100061445DF8044B64F0CDB85DF8044B7047D3
:1090200030B585B068465AF0B9FA0F480F4AD0F803
:10903000FC10009B0E4D41F08071C0F8FC10002424
:1090400000F1C840C2F8B05FA0F565005460116837
:10905000084CA0F67D60A0FB030341F001019B0CCE
:10906000A360116005B030BD00ED00E0001000E02D
:1090700055CEACC5C81A00202DE9F0411D4CDFF8D3
:109080007C801D4F82B004F54075012602E0083453
:10909000A54223D0A379002BF9D1206800F13F43EA
:1090A00003F57E0308EB932393F860345A09032AEF
:1090B00003F01F0306FA03F317D0042A11D0022A83
:1090C00002D17A6C13437B640023A1881A46CDE950
:1090D0000036083460F0C4FBA542DBD102B0BDE825
:1090E000F0813A6B13433B63EEE73A6C13433B6406
:1090F000EAE700BF3023002000380240DCD6060833
:1091000009494B6C10B5094C43F480434B64402231
:10911000002104F6683064F0A5F84FF0FF33C4F87E
:10912000A83BC4F8AB3B10BD00380240C81A002071
:109130002DE9F0411348144D4FF41A72002164F0E8
:1091400091F84FF00008A5F58D6705F6880440F208
:10915000222655F82810002354F8332091420BD0D2
:1091600001330E2BF8D1002008F107085FF09EF8BC
:10917000B045EED1BDE8F08107EBC30393F8F40CE2
:10918000F2E700BF1820002044DB0608F8B50468A9
:10919000D4E904235568117D1768002B40D01F299E
:1091A0005E6898612CD820228A4042F01802BA608A
:1091B0001A7D19681F2A2DD9203A2023934043F0A5
:1091C0001803CB6000232B6033603368A16943F040
:1091D0001003336028465AF0C1FAE16930465AF06C
:1091E000BDFA2B68626843F001032B60336843F0DB
:1091F0000103336093889BB243F003039380F8BD6F
:10920000203920228A4042F01802FA601A7D19683B
:109210001F2AD1D82023934043F018038B60D1E755
:109220001F29906119D820238B4043F01803BB609D
:1092300000232B602B68A16943F010032B602846A4
:109240005AF08CFA2B68626843F001032B60938814
:109250009BB243F002039380F8BD203920238B405A
:1092600043F01803FB60E3E738B5274D95F8E82491
:1092700095F8E9349A4241D1244A92F80406F0B1B3
:10928000234B92F80846D5F8B02B00EB400003EBD7
:10929000C000B4B140F20D3C00E01A6899689C89A6
:1092A0004C600C6844F001040C60A2F848C091893D
:1092B000183389B241F4807183429181EDD138BD78
:1092C0001A68118821F0800109041833090C1180F3
:1092D00033F8141CD162118889B241F080011180E9
:1092E0005462B2F80CC033F8041C41EA0C0189B294
:1092F0008342918123F8044CE2D138BD60F034FF01
:109300000028B9D138BD00BFC81A002004000010E1
:109310007826002010B5044663F014FB81B2204685
:10932000BDE81040FFF780B938B50B4D00EB4000A9
:1093300005F2445303EBC00393ED027AD3ED037AB5
:10934000E7EE007AC4002544B0EE670A63F0FAFA4B
:10935000D5F84435186038BD04000010F8B50C4B42
:109360001D685A69154005405D617DB1094F0126B0
:10937000B5FA85F4C4F11F0407EB840306FA04F47C
:10938000D3F8680B03689847A543F1D1F8BD00BF37
:10939000003C0140C81A00202DE9F843038AB0F8C8
:1093A0000C801FFA88F818EA030829D005460E46F3
:1093B0004FF00047B8FA88F327FA03F2D24391B28C
:1093C0001B3B298208EA0208042B16D8DFE803F0C9
:1093D000352C231A0300B36A002B37D003F1FF3971
:1093E00000231FFA89F9B362746A34B123682046F6
:1093F000494698476468002CF8D1B8F1000FD9D1DC
:10940000BDE8F8837068696B036889B29847B8F162
:10941000000FCFD1F4E7B068A96B036889B2984711
:10942000B8F1000FC6D1EBE7F068E96B036889B2C9
:109430009847B8F1000FBDD1E2E73069296C0368A5
:1094400089B29847B8F1000FB4D1D9E7EB6A1FFA97
:1094500083F9C9E70A4608B5054920B905485AF015
:1094600009FC034808BD04485AF004FC004808BD44
:10947000382700206C6907089469070810B5044C68
:1094800004480A4621465AF0F5FB204610BD00BFAD
:1094900038270020BC69070810B5044C04480A4668
:1094A00021465AF0E7FB204610BD00BF38270020B8
:1094B000D069070810B5044C04480A4621465AF002
:1094C000D9FB204610BD00BF38270020DC69070803
:1094D000F8B5A0F668042379DB0725D5657994F8FB
:1094E0004C3805F001073D46FBB1D4F848341A6802
:1094F000D36A5B08536294F8503823B1B4F85A38F1
:109500000133A4F85A38606C85F001015EF0D4FD97
:10951000012384F84F38002384F84D3884F84E38FE
:10952000A4F8563884F84C38F8BD94F84F68012EEA
:1095300004BF94F84D3884F84E382046FFF7B8FA47
:109540004EB9012384F84F3887EA0301606CBDE807
:10955000F8405EF0B1BD002384F84F383946F5E796
:1095600038B5A0F668040022606C344D03685A6276
:10957000A1F12903302B31D895F86F3D95F8701D76
:109580000133DBB2012B85F86F3D09D9B4F85638A9
:1095900085F86F2D5B08A4F856384B1C85F8703D94
:1095A00095F8702D0023082AA4F8583815D185F8AD
:1095B000703DB5F8723D01339BB2032BA5F8723DA7
:1095C00008D92379DB0705D5E36A94F8560843B335
:1095D000216B98470023A4F8563838BD5B396C29B5
:1095E0000CD8B4F8563885F86F2D5B0843F080032B
:1095F000A4F8563895F8703D0133CFE794F8513808
:10960000002BCDD1012185F86F3DA5F8723D802357
:1096100084F85118A4F8563885F8701D5EF04CFD9A
:10962000BEE7E3696269D054E369E2680133B3FBE2
:10963000F2F102FB1133E361CCE700BFC81A00204E
:109640002DE9F843DDF820800F4615460021202241
:1096500004461E4663F006FEB8F1000F0CD0D8F8A1
:109660000030E3811B0C2382D8F80430B8F80A20BC
:10967000E3821B0C62822383384661F03FFBEB06DA
:1096800019D4431EB8B107EB000C01E0013B12D323
:109690001CF801EDBEF12E0FF8D1C01A421E032AAC
:1096A000A8BF0322082B03F10109A8BF0823904695
:1096B000B9441A4606E008280246B946A8BF08225F
:1096C0004FF000084FF02033394623606360204696
:1096D00063F070FD04F10800154B238142464946B2
:1096E000837063F067FD611EE21D11F801CFACF1DC
:1096F0006103192B9CBFACF1200C81F800C0914292
:10970000F3D104F10A0011F8013FA3F16102192A13
:109710009CBF203B0B708142F5D118232373330C7F
:10972000A382E572099B6683E361BDE8F88300BF0D
:109730002020200008B55AF043FE0C4B93F8791D09
:1097400029220129A3F8C628A3F8CE2801D0012098
:1097500008BD0748C3F87C0D00F120014C3060F0D3
:10976000D9F8044B002083F8230008BDC81A002054
:10977000BC01002000ED00E02DE9F04FDFF84CB413
:10978000DBF8000085B0CBF81408002B60D0134440
:109790000C46174601F5FE7A99461FE0002F64D06B
:1097A000DBF84438BB4200F0C680DBF84038BB42EF
:1097B00000F0F880DBF84838DBF84C18BB424BD897
:1097C000B94200F27081791A20465EF015FB01372C
:1097D0004F4504F500740AF5007A39D0DBF85038AB
:1097E000BB42DBD8DBF86058FB1A296BDA0802327F
:1097F0008A4203F0070602D3AB6B9A420BD9294683
:10980000104602925EF0C8FA029A0546002800F05F
:109810006A81CBF860082B79002B40F01E81D5F8C7
:109820002880B8F1000F00F057812B6BD21AEB683B
:1098300006EBC20203EB422220462B464FF4007196
:109840000137C0474F4504F500740AF5007AC5D1C9
:10985000002005B0BDE8F08FB942B4D94FF40072D2
:109860000021204663F0FEFCB1E74FF40072394658
:10987000204663F0F7FC802384F8BE310C2384F883
:10988000C231DBF84018C54ADBF83838C4F8C611D5
:109890009142C4F8CA3100F30B81C14AC14D82FB29
:1098A000010285FB01050A44C817C0EB6212C0EB38
:1098B0002530BD4D84F8C10185FB0265C2EB8216DF
:1098C0008010891B013120F03F0015440843D11757
:1098D000C1EBE5110A4484F8BF21B04A84F8C00105
:1098E000013B934200F3F080AD4AAE4882FB031285
:1098F00080FB03101A44D917C1EB6212C1EB20316F
:10990000A94884F8C51180FB0250C2EB821589106A
:109910005B1B013321F03F0110441943D317C3EB04
:10992000E0131A4484F8C41184F8C3214AF655237D
:10993000A4F8FE314BE74FF0FF3384F8EC3184F8A4
:10994000ED3184F8EE3184F8EF31522323706370E7
:109950006123A37084F8E7314123E37084F8E63192
:109960007223002584F8E43184F8E531DBF85838B7
:10997000C4F8E8314FF4F0722946201D63F072FC00
:10998000552384F8FE316FF05503C4F8F051C4F844
:10999000F451C4F8F85184F8FC5184F8FD5184F86E
:1099A000FF3114E74FF400720021204663F05AFCA7
:1099B0007E4B03CB45F6EB0323809023C4F80710BE
:1099C000A37002220821F823C4F8030061732274F3
:1099D0006375DBF838382273A27384F82C20DBF827
:1099E00040289B1A2362DBF84828DBF84C389B1A86
:1099F00063620023E372E3736377A377E37784F80A
:109A00002D3084F82E3084F82F3084F83130684BB4
:109A1000A361684BC4F842303E232377012384F8C6
:109A20003030654A802384F8403084F846104AF686
:109A30005521A4F8FE1103CA604BC4F84700C4F8CE
:109A40004B1003CB1388A4F84F309378C4F852001E
:109A5000C4F8561084F85130B9E64FF40072002172
:109A6000204663F0FFFB002E44D12B6C04F120084C
:109A7000002B7BD02B6B52491122CDE9006620468A
:109A8000FFF7DEFD2B6C1A6C002A7ED01B6B4D4954
:109A9000CDE9006640461122FFF7D2FD04F14008EF
:109AA0004FF4E0736DE0F91A20465EF0A5F98EE6FA
:109AB000FF2284F8C1214FF6FF72A4F8BF21374A74
:109AC000013B93427FF710AFFF2384F8C5314FF677
:109AD000FF73A4F8C33129E741464FF400722046D2
:109AE00063F0C0FB73E6384A231F43F8042F9A45FE
:109AF000FBD16CE6D5E910253301002A43D0023BA7
:109B0000002D3FF464AE013BAD6CF9D1A0464FF49B
:109B10000073002D3FF45BAECDE9027A08EB03063B
:109B2000A24608E00024CDE900C4FFF789FDAD6C32
:109B3000BDB1B04515D02C7929682B6B404605F195
:109B40001C0C112208F12008002CEBD16A792C6939
:109B500042F02102CDE900C4FFF772FDAD6C002D8B
:109B6000E7D15446029FDDF80CA030E6CDE900664F
:109B70003346DBF83C1808222046FFF761FD4FF41E
:109B8000F0736D6CC5E7013BBAE7CDE900660D499E
:109B9000334640461122FFF753FD7FE7FF03FB00EA
:109BA000832008829755454181808080F4690708A9
:109BB0003F00FF0029940E0D006A07080C6A070891
:109BC000EC690708F0690708DEADBEEFC81A00208F
:109BD00010B4EFF31182102383F31288084B196835
:109BE0004FF0E02001311960816959600024C3F809
:109BF000804D0369D3B283F311885DF8044B70473D
:109C0000C81A002010B4EFF31181102383F31288D7
:109C10004FF0E022C9B29469136913F4803F0C4BF2
:109C20001EBF0120C3F8800D94691868D3F8802DF9
:109C300081F31188996802444FF47A7000FB01F3B4
:109C40001B1B5DF8044BB3FBF1F300FB02307047C4
:109C5000C81A0020234B5B68C3F3080310B4DBB9B8
:109C6000EFF31183C3B9204B4FF0E02C1A68DCF8F6
:109C7000180019688A42F9D159688842F6D89C6858
:109C80004FF47A7101FB04F3181AB0FBF4F05DF89D
:109C9000044B01FB02007047EFF31181102383F3A3
:109CA00012884FF0E022C9B29469136913F4803F1F
:109CB0000D4B1EBF0120C3F8800D94691868D3F8BE
:109CC000802D81F3118899684FF47A73024403FB65
:109CD00001F0001B5DF8044BB0FBF1F003FB020048
:109CE000704700BF00ED00E0C81A00202DE9F04FDA
:109CF000037D02681F2B83B0044609D95068A3F185
:109D000020052021A940014207D103B0BDE8F08F12
:109D10001068202199400142F7D04949D4F81880B1
:109D2000484F4868484D8C2101FB0871C5F80C0666
:109D300095F808C6D1F890000668BCF1000F18D15C
:109D4000D1F80801B1F894C0016821F00101016067
:109D5000B18989B221EA0C01B1812978B9B91F2BE7
:109D600061D9A3F1200120238B40D36003B0BDE86B
:109D7000F08F0069016821F001010160B18921F4CF
:109D800080710904090CB18129780029E7D04FF0CE
:109D90008C0909FB08F907EB0903DFF8B0B0D3F829
:109DA00008211046CDE9002359F042FC019B012215
:109DB00083F8DC20D5F8143609F1180ADA44002BB0
:109DC00038D033889BB243F08003338009F17409A3
:109DD0004FF0FF330BEB0901F362304659F09CFE64
:109DE0008C2303FB0877514600230098C7F8AC305A
:109DF00059F0B4FCD7F8083116225A601A6842F0BC
:109E000001021A60D7F89020B7F89430126891894F
:109E10000B439BB293810A49237D49682268C5F8A8
:109E200010161F2B9DD8202101FA03F3936003B075
:109E3000BDE8F08FFFF70EFFC5F81406C1E700BFBD
:109E4000001000E0C81A002004000010501B002081
:109E50002DE9F843FFF7FEFE204F214E7C680546B2
:109E60004FF00008002C2DDD00231A4607EB0321DC
:109E7000013391F8F9109C4242EA0102F6D142EA1C
:109E800008095FFA89F990467368C3F30803B3B908
:109E9000EFF311839BB9FEF7B3F8401BB0F5FA6FEF
:109EA00002DCB8F1000FDDD1B9F1000F04D00D4B89
:109EB00093F8842D532A09D04846BDE8F883FFF76C
:109EC000A1FEEAE7C1464FF00008DDE7B3F88C2DAC
:109ED0000132A3F88C2D4846BDE8F8830400001039
:109EE00000ED00E0C81A0020AD4B1B780BB9012033
:109EF00070472DE9F04FDFF8BCB2AA49DBF800202B
:109F0000A94BA1FB02125209A3FB0213DB08A449CF
:109F100087B003EB8303A2EB4303D1F81826049226
:109F200001F21C64DAB2059204EB8307002201F609
:109F3000FC03019301F5816A9046049B984580F2E9
:109F40000D81DAF81820DAF80490D2F8E830D2F867
:109F5000EC600293FFF77EFE029B03904FEA890CB0
:109F60009BF8849D9BF8980D0CF1085C06F18061CC
:109F70000CEB431C3939B9F1530F0CEB81110CEB8D
:109F8000801301D1ABF88E0D994240F27D811A68A1
:109F9000002A00F071811A6C002A00F08381D3F846
:109FA0008020002A00F08081D3F8C02003F5807360
:109FB000002AE9D1A3EB0C0C99424FEAAC1240F213
:109FC0006381B11A45294FF0000628BF452130466C
:109FD000B64603EB81111D4616460DE01A6C002AA9
:109FE00040F0EA80D3F88020002A40F01581D3F8B1
:109FF000C02003F580732AB9994206D91A68002A4D
:10A00000ECD04033994200F2DB8032467646112E86
:10A0100040F23E81DEF1150100F13A81634B1D46AD
:10A02000D3F89C309A4238BF2B46039D38BFC3F803
:10A030009C20DBF89C3DEA1A002A18DB03F5F42388
:10A0400003F590739D4284BF2B460533CBF89C3DAE
:10A05000564B564AD3F89C30052B86BF053BDBB2E6
:10A0600000238BF8983D4FF0FF33C2F89C3031B19C
:10A0700000FA01F1C6F114060120B04008434C4E2D
:10A08000C0F3C43306EB8303D3F8601D00F01F0355
:10A0900006EB8303D3F8602D42EA0132C0F344118A
:10A0A00006EB8101C0F3842306EB8303D1F8601D26
:10A0B000D3F8603D42EA011141EA032181EA11230C
:10A0C00083EA131303F00F02354BD3F804390F2A38
:10A0D00003F1010340F0BD80B1F5803F80F0B9800D
:10A0E000B9F1530F4FEA111140D02D4AB1F5606F0D
:10A0F000C2F8043945D0019B998194F858300598ED
:10A1000083420CD0BA6823689B1A23603A6B636859
:10A110009B1A63600023BB603B6384F8580023688C
:10A1200001332360BB680133BB604FF6FF73994274
:10A1300005D16368013363603B6B01333B63019B73
:10A1400008F101081433B8F1080F04F15C0407F1B9
:10A150005C0701930AF1200A7FF4EFAE104A012355
:10A16000012082F8003A07B0BDE8F08FBBF8882DD7
:10A170000132ABF8882D0A4AB1F5606FC2F8043994
:10A18000B9D19BF8E93403EB43030BEBC30343441E
:10A1900093F8F9340D2BAED1019A80239377ACE775
:10A1A000040000101F85EB51CDCCCCCC88010020E1
:10A1B000DCD60608C81A0020803399427FF625AF06
:10A1C000A3EB050C3C4A4FEAAC1C0CF1010C82FBE2
:10A1D0000C52A2EBEC72012AB8BF012290404FF062
:10A1E000010C9644013A0CFA02F210439C46DCF84A
:10A1F00000209AB1DCF84020002A57D0DCF88020FB
:10A20000002A56D0DCF8C0200CF5807C42B16145B4
:10A21000EDD81D466346EFE6C033F3E60CF1400C83
:10A220006145F6D9ACEB03029211234B013283FB5B
:10A230000253A3EBE273012BB8BF012398409E4465
:10A240000122013B02FA03F3184363461D466346AD
:10A25000D2E6B9F1530F04D1BBF8882D0132ABF827
:10A26000882D164AC2F80439D2F800390133C2F8F1
:10A2700000394FF6FF7140E74033A3EB0C0C9942D5
:10A280004FEAAC123FF69DAE10B101388BF8980D35
:10A29000B9F1530F7FF453AFBBF88A3D0133ABF8EC
:10A2A0008A3D4CE7803385E6C03383E60CF1800CB1
:10A2B000B6E70CF1C00CB3E7565555550400001035
:10A2C000F8B51D4B93F8E82493F8E9349A422ED15F
:10A2D0001A4F7D68002D11DD3846002410F8086BF8
:10A2E00016B1037E012B1CD002691368013443F0C0
:10A2F0000103AC4200F580701360F1D1FFF7AAFCB6
:10A30000D7F8044A002C0BDD0D4A02EBC404116897
:10A3100093888889083203439BB294428B81F6D19B
:10A32000F8BD002380F8F030FEF71EFADCE75FF09E
:10A330001BFF0028CCD1F8BDC81A00200400001073
:10A340000C0A0010454B5B68C3F308032DE9F0438A
:10A350000546002B5ED1EFF31183002B5AD1404B01
:10A360004FF0E0241A68A06919688A42FAD1596846
:10A370008842F7D89E684FF47A7101FB06F4241ADC
:10A38000B4FBF6F401FB0244344E10274FF0E02CEE
:10A390004FF47A7E4FF001087268C2F30802CAB91E
:10A3A000EFF31182B2B91A68DCF8180019688A4212
:10A3B000F9D159688842F6D8D3F808900EFB09F114
:10A3C000091AB1FBF9F10EFB0212121BAA42E3D3E8
:10A3D000BDE8F083EFF3118287F31288DCF81800F0
:10A3E000DCF81010C90344BFC3F8808DDCF81800F6
:10A3F000D3F80090D3F8801DD2B282F3118849447B
:10A40000D3F808900EFB09F2121AB2FBF9F20EFB18
:10A410000122DAE7EFF31181102383F312884FF062
:10A42000E022C9B29669136913F4803F0C4B1EBF3A
:10A430000120C3F8800D96691868D3F8802D81F348
:10A440001188024498684FF47A7101FB00F4A41B50
:10A45000B4FBF0F401FB024496E700BF00ED00E01E
:10A46000C81A00202DE9F0473A4B3B4D471E1026F5
:10A470004FF0E0204FF47A7C4FF001086A68C2F395
:10A480000802002A52D1EFF31182002A4ED11A6835
:10A49000846919688A42FAD159688C42F7D8996858
:10A4A0000CFB01FEAEEB040EBEFBF1FE0CFB02EE5C
:10A4B0006A68C2F30802E2B9EFF31182CAB91A68F6
:10A4C000846919688A42FAD159688C42F7D8D3F85E
:10A4D00008900CFB09F1091BB1FBF9F10CFB02120E
:10A4E000A2EB0E02B2F57A7FE2D3013FC6D2BDE8FD
:10A4F000F087EFF3118286F3128884690169C9033A
:10A5000044BFC3F8808D8469D3F800A0D3F8801DC0
:10A51000D2B282F31188D3F8089051440CFB09F2AF
:10A52000121BB2FBF9F20CFB0122D9E7EFF3118108
:10A5300086F3128884690269D20344BFC3F8808D10
:10A540008469D3F800E0D3F8802DC9B281F3118873
:10A550007244A4E7C81A002000ED00E02DE9F84F8E
:10A5600001307E4C7E4D01F1FF385FFA80FB1026F2
:10A5700001275EF0C1FA4FF4FA794FF0E0214FF471
:10A580007A7C6B68C3F30803002B40F0C080EFF3C4
:10A590001183002B40F0BB802368886922689342B6
:10A5A000FAD162689042F7D8A2680CFB02FEAEEBCB
:10A5B000000EBEFBF2FE0CFB03EE6B68C3F3080358
:10A5C000002B40F08680EFF31183002B40F0818058
:10A5D0002368886922689342FAD162689042F7D86A
:10A5E000D4F808A00CFB0AF2121AB2FBFAF20CFB28
:10A5F0000323A3EB0E03B3F57A7FDED3B9F1010990
:10A60000BFD158464FF47A795EF040FC4FF0E0211C
:10A61000CC466B68C3F30803002B40F08B80EFF34C
:10A620001183002B40F0868023688869226893425A
:10A63000FAD162689042F7D8A2680CFB02FEAEEB3A
:10A64000000EBEFBF2FE0CFB03EE6B68C3F30803C7
:10A650000BBBEFF31183F3B9236888692268934237
:10A66000FAD162689042F7D8D4F808A00CFB0AF23D
:10A67000121AB2FBFAF20CFB0323A3EB0E03B3F5A1
:10A680007A7FE2D3B9F10109C3D1B8F10108BFF46F
:10A6900070AFBDE8F88FEFF3118386F31288D1F81D
:10A6A00018A00A69D20344BFC4F8807DD1F818A06D
:10A6B0002068D4F8802DDBB283F311880244A068AF
:10A6C0000CFB00F3A3EB0A03B3FBF0F30CFB023328
:10A6D000D3E7EFF3118386F31288D1F818A00A6943
:10A6E000D20344BFC4F8807DD1F818A02068D4F804
:10A6F000802DDBB283F311880244A0680CFB00F3C9
:10A70000A3EB0A03B3FBF0F30CFB023371E7EFF3A7
:10A71000118286F3128888690B69DB0344BFC4F891
:10A72000807D88692368D4F880EDD2B282F31188E5
:10A73000734439E7EFF3118286F3128888690B6955
:10A74000DB0344BFC4F8807D88692368D4F880EDBA
:10A75000D2B282F3118873446EE700BFC81A00209A
:10A7600000ED00E02DE98848954C964E431C5FFAB9
:10A7700083FB0A254FF0100801275EF0BDF94FF466
:10A78000FA7C4FF0E0204FF47A717368C3F308034A
:10A79000002B40F0CE80EFF31183002B40F0C980F6
:10A7A000D4F800E0836922689645F9D16268934243
:10A7B000F6D8D4F8089001FB09F2D21AB2FBF9F2EC
:10A7C00001FB0E227368C3F30803002B40F0D58011
:10A7D000EFF31183002B40F0D080D4F800E0D0F8E4
:10A7E000189023689E45F8D163689945F5D8D4F848
:10A7F00008A001FB0AF3A3EB0903B3FBFAF301FB87
:10A800000E339B1AB3F57A7FDCD3BCF1010CBCD1BB
:10A8100058465EF03BFB4FF47A7C4FF0E0206146F7
:10A820007368C3F30803002B3ED1EFF31183002BB1
:10A830003AD1D4F800E0836922689645F9D162687C
:10A840009342F6D8D4F8089001FB09F2D21AB2FB71
:10A85000F9F201FB0E227368C3F30803002B46D103
:10A86000EFF31183002B42D1D4F800E0D0F8189018
:10A8700023689E45F8D163689945F5D8D4F808A0B7
:10A8800001FB0AF3A3EB0903B3FBFAF301FB0E335D
:10A890009B1AB3F57A7FDED3BCF1010CC0D1013D28
:10A8A0007FF46BAF5EF020F9EFF3118288F312882A
:10A8B000D0F818E00369DB0344BFC4F8807DD0F80A
:10A8C00018E02368D4F8809DD2B282F311884B44FB
:10A8D000D4F8089001FB09F2A2EB0E02B2FBF9F2E8
:10A8E00001FB03227368C3F30803002BB8D0EFF316
:10A8F000118388F31288D0F818A0D0F810E01EF465
:10A90000803F1CBFC4F8807DD0F818A0D4F8009018
:10A91000D4F880EDDBB283F31188CE44D4F80890EC
:10A9200001FB09F3A3EB0A03B3FBF9F301FB0E33BD
:10A93000AEE7EFF3118288F31288D0F818E00369CC
:10A94000DB0344BFC4F8807DD0F818E02368D4F856
:10A95000809DD2B282F311884B44D4F8089001FB59
:10A9600009F2A2EB0E02B2FBF9F201FB03227368BB
:10A97000C3F30803002B3FF42BAFEFF3118388F3ED
:10A980001288D0F818A0D0F810E01EF4803F1CBF49
:10A99000C4F8807DD0F818A0D4F80090D4F880EDE9
:10A9A000DBB283F31188CE44D4F8089001FB09F39D
:10A9B000A3EB0A03B3FBF9F301FB0E3321E700BF5E
:10A9C000C81A002000ED00E030B50C4683B0054603
:10A9D000D8B1036803F13F4303F57E039B0A0C4A99
:10A9E000134493F860045DF061FCC4F34112C4F3B6
:10A9F0000013CDE90032C4F38103A988286804F06C
:10AA000003025EF02DFF03B030BD4FF0FF33E6E7E9
:10AA1000DCD6060800B1D7E7704700BF70B50F4C11
:10AA2000D4F81866002E16DD04F58164002504E0D4
:10AA30000135B54204F120040DD0237F002BF7D05F
:10AA4000E0680028F4D0217D0135FFF7BDFFB54255
:10AA500004F12004F1D1012070BD00BF04000010FA
:10AA6000F8B5037D856902681F2B04464BD95068F1
:10AA7000203B20219940084237D0D16010219940D5
:10AA8000D1605168D940CE077FD4EFF311835022B3
:10AA900082F312882A6C1168C90757D4516889B2A9
:10AAA00091B9D5E9096086424DD0AF699CBF0E4689
:10AAB0002969074494BF081A301A80B20021D76070
:10AAC000AE6285F864105060116841F00101DBB29C
:10AAD000116083F3118895F86430002B3DD1237DFC
:10AAE00022681F2B194614D9203B50680821994031
:10AAF000084200D0D1605068042101FA03F31842E3
:10AB000000D0D360F8BD16682020984006420DD1D1
:10AB10001946106808238B40184200D093601068D3
:10AB200004238B401842EDD09360F8BD102199406A
:10AB3000906091601168D940C807A6D5012101FA3B
:10AB400003F39360A1E7012285F86420DBB283F36D
:10AB5000118895F86430002BC1D095F87D30002B1A
:10AB6000BDD195F8710013F071F82A6E938923F026
:10AB700008031B0401211B0C938185F87D1000281C
:10AB8000ADD02021FFF720FFA9E7012101FA03F34F
:10AB9000D3607AE710B42A492A4A91F804367BB385
:10ABA000D2F8B04BA04239D0012B29D0D2F8C84BF3
:10ABB000844239D0022B23D0D2F8E04BA04235D0CA
:10ABC000032B1DD0D2F8F84BA04231D0042B17D064
:10ABD000D2F8104CA0422DD0052B11D0D2F8284C21
:10ABE000A04229D0062B0BD0D2F8404CA04225D051
:10ABF000072B05D0D2F8584C844208BF07230ED04B
:10AC000003F1010C81F804C603EB430102EBC1021E
:10AC10005DF8044BC2F8B00B184670470023DBB256
:10AC200018465DF8044B70470123F8E70223F6E766
:10AC30000323F4E70423F2E70523F0E70623EEE716
:10AC400004000010C81A002038B5414C8C2303FBC7
:10AC5000004393F8973003B938BD94F8E8C494F8EA
:10AC6000E9349C450ED003EB430204EBC20292F898
:10AC7000ECE40EF1FF35012D4FEA430246D9BEF157
:10AC8000030F3ED08C2202FB0042A2F88810EFF3A3
:10AC90001181902383F31288B2F8885092F88A3099
:10ACA00043EA45030025C9B29BB282F88A5081F37A
:10ACB000118828491A090D7882EA13225A4005B1F1
:10ACC000D2431B019BB202F00F021A4391F80836DF
:10ACD000D1F8285A4BBB8C2303FB00440121D4F844
:10ACE0001001A847D4F80C11B4F894508A8AD4F80B
:10ACF00008312A438A8258601A6842F001021A60B9
:10AD000038BD5D1C05F003056545BBD01A4404EB56
:10AD1000C202024492F8F9140029B3D08C2303FB39
:10AD20000043012283F88A20ACE78C2303FB004414
:10AD3000D4F89030D4F80C115B79086903F0FC0367
:10AD400018440421A847D4F80C318000988138BDFC
:10AD5000C81A00200400001043680B4A23F0407317
:10AD600023F4807343F48073436083681A4042F095
:10AD700002028260C36A0139C9B223F4700343EA54
:10AD80000153C362704700BFFDF7FFC0704700BFAB
:10AD90000020FDF763B900BF0120FDF75FB900BFD8
:10ADA0000220FDF75BB900BF10B1036882881A83E7
:10ADB000704700BF30B1036882881B691A4214BF14
:10ADC00001200020704700BF10B1036882885A83B9
:10ADD000704738B5054600780C4612F037FF611C05
:10ADE000C9B2044610B141238371C171204669780C
:10ADF000FFF710FEAB78204613B1BDE83840D3E72B
:10AE0000BDE83840E0E700BF2DE9F047804E074637
:10AE10004FF0010A3C6897F888806368B8881A8800
:10AE200084F824A022F040021204120C1A80228915
:10AE3000824221D01A88774922F0380212048B42CC
:10AE40004FEA124200F0BF8001F580618B4200F0B2
:10AE5000BA800146B1F5807FA8BF4FF48071022906
:10AE6000B8BF022191FAA1F1B1FA81F1013942EAA8
:10AE7000C10292B21A802081397BA27A8A420CD018
:10AE80001A8822F003021204120C1A801A8892B255
:10AE9000002900F095801A80A1721A8894F80C900D
:10AEA00092B242F040021A80226A9168002900F0B2
:10AEB000A5804FF0000C1432E64652F8100C8E4478
:10AEC00000EA060120B1B1F1805F25D0616919B3B4
:10AED00052F8141C143201EA060011B1B0F1805F7F
:10AEE0001AD052F80C1C0CF1010C0029E5D1B9F173
:10AEF000000F11D0B8F1000F0ED0BCF1010F6FD8C8
:10AF0000BEF1070F6CD80CEB8C0C4FEA8C01226A57
:10AF10000A44127B002A63D0226A92684FF000082C
:10AF2000002A52D0B8F1000F02D098F80C2022B1BC
:10AF3000BA6812B1116892884A83226A1568226A37
:10AF40005168226A9268501E9AB12DB32A4612F8AF
:10AF500001EB15461A899207FCD5A3F80CE01A8973
:10AF6000D207FCD59A8992B209B101F8012B0138B8
:10AF7000EBD2236A1B7BE3B9236A1B697BB1236A8B
:10AF8000D7F894001B69984701280DD0022806D1F4
:10AF900000232362BDE8F0874FF0FF0EDAE7D4F814
:10AFA0002080236A14332362236A9B686BB1636831
:10AFB000B8E7BB68002BDFD01A689B881383DBE7F8
:10AFC00042F0030267E7410844E7236A1B68E3B1E4
:10AFD000236AD3E9007222620022C3E9002219E742
:10AFE000386800215FF056FEBB6813B11A689B8871
:10AFF00053833846BDE8F047FEF7C8B8B9F1000FF3
:10B000008AD0B8F1000F82D186E72362C2E700BF81
:10B010000000FFFF0038004030B40568EFF3118CEA
:10B02000102383F3128803681B6AEBB18B68044614
:10B030000A461BB1D3691432002BFBD12B6A6BB1CA
:10B04000986838B9934209D0186828B15B68986845
:10B050000028F7D01433F3E7C3E900415FFA8CFC12
:10B060008CF3118830BC704729625FFA8CFC8CF33A
:10B07000118830BCC8E600BFF0B5224C224A234BF1
:10B0800095B0054604F1A800CDE90002049304F14F
:10B09000AC000023CDE90503CDE90E331C4A09922B
:10B0A0000B9304F1A0021093139311936B6A2F7FFB
:10B0B0000A921868012302228DF80C3007938DF84C
:10B0C00020308DF834308DF848303B1D02920E460A
:10B0D0000C935FF0DBFD97B1330E84F8A130A234FE
:10B0E000320C330A22706370A670686A6946FFF7F3
:10B0F00093FF6B6A18685FF0C9FD15B0F0BDA1340D
:10B10000EEE700BF8801002068280020698E000853
:10B11000498E000810B5044694B05022064968468E
:10B1200062F048F8606A6946FFF776FF636A18685C
:10B130005FF0ACFD14B010BDBCE406082DE9F04191
:10B140000446406A00681E460F4690465FF09EFD2A
:10B15000237FA069002B3ED0284D030E85F8B13027
:10B16000052205F1B2039870C5F8E820020C000A28
:10B1700058701A703B68C5F8F4300020D8F80030D9
:10B18000C5F8FC30012E2363C5F80C0128D0022E2F
:10B190001FD1D8F80420C5F80401796885F80001AA
:10B1A000C5F8081113441649C5F81021012023637E
:10B1B00085F81401C5F81811124B627F606AA3F17B
:10B1C0001401002A08BF1946FFF726FFE36A7BB186
:10B1D000206BBDE8F0810C4B0422A3F1B105C2E75E
:10B1E000074B85F80061C5E94130C5F81001E3E778
:10B1F000636A18685FF04AFDEAE700BF8801002033
:10B20000518E0008540200203902002000B583B09E
:10B2100081610192049A0093C26201236A4601A9E6
:10B22000FFF78CFF03B05DF804FB00BF38B52C4A74
:10B23000D0F8E0305268D0F8D810044673B1501AF4
:10B2400083420BDC94F8D030C4F8D820012B10D006
:10B25000D4F8D4300133C4F8D43038BDD4F8E43055
:10B26000C4F8D8200B44C4F8DC3094F8D030012B5B
:10B27000EED16168201D04F1E805EFF3118C102375
:10B2800083F3128863681B6A0BB3D4F8F0302A4644
:10B290001BB1D3691432002BFBD10B6A6BB19968D7
:10B2A00039B9934209D0196829B15B6899680029B6
:10B2B000F7D01433F3E7C3E900055FFA8CFC8CF395
:10B2C0001188D4F8D4300133C4F8D43038BD0D62BD
:10B2D0005FFA8CFC8CF31188FFF796FDB8E700BF8E
:10B2E000001000E02DE9F041826992F8DC30012B7A
:10B2F0008AB005464CD0023B012B54D892F84C3111
:10B30000D2F89C202E4C63F07F0313708769D7F826
:10B31000A030D7F8108003F1010E0FCCEC46ACE85A
:10B320000F00D7F89C30CDE9003E0FCCACE80F0001
:10B3300094E8030007F110068CE80300EFF3118096
:10B34000102383F312883B691B6A002B2FD0029BCA
:10B350006A461BB1D3691432002BFBD1D8F82030D8
:10B3600073B1996839B99A420AD0196829B15B68F2
:10B3700099680029F7D01433F3E71E60C3F804D0AE
:10B38000C0B280F31188AA6911690B6A002BFCD145
:10B39000D2F8A0305A8852BAEA819A8852BA2A82E0
:10B3A000DB885BBA6B8201200AB0BDE8F081C8F887
:10B3B00020D0C0B280F311883046FFF725FDE2E7C8
:10B3C0000CE506082DE9F04190F8DC30D0F8A050EB
:10B3D000012B8AB0044673D041D9023B012B6BD8B4
:10B3E00090F84D31D0F89C205E4E63F07F031370CF
:10B3F000D0F8A030D0F8108003F1010E00F1100752
:10B400000FCEEC46ACE80F00D4F89C30CDE9003EFE
:10B410000FCEACE80F0096E803008CE80300EFF3D2
:10B420001180102383F3128823691B6A002B00F01C
:10B430008F80029B6A461BB1D3691432002BFBD16B
:10B44000D8F820302BB3996839B9934221D01968C4
:10B45000E1B15B6899680029F7D01433F3E7D0F8BD
:10B460009C304FF0FF321A605A609A60DA60D0F870
:10B47000E0300522B3F57A7FC0F8F0203BD80323F3
:10B4800080F8DC3001200AB0BDE8F0811F60C3F80D
:10B4900004D0C0B280F311882269136A002BFCD15A
:10B4A0006B885BBAA4F8D030AB885BBAA4F8D23012
:10B4B000EB885BBAA4F8D43001200AB0BDE8F08173
:10B4C00090F84C2190F84D319B1A5B100133DBB2A0
:10B4D00005EB430235F813305BBAA0F8D03053883F
:10B4E0005BBAA0F8D23093885BBAA0F8D4300120C0
:10B4F0000AB0BDE8F08103691A7B2AB35B691BB30C
:10B5000090F8983003B390F84C31D0F89C20C4F8F0
:10B51000A40063F07F03137090F84C1190F84D3144
:10B52000D0F8A0201048C4F804015B1A07330121A9
:10B53000C4F8FC30D4F89C3084F800110A44C4E903
:10B540003D3284F8DC10B7E7022384F8DC30B3E73F
:10B55000C8F820D0C0B280F311883846FFF754FCF9
:10B560009AE700BF0CE506083980000870B504684A
:10B57000236A1B69054683B1236AD0F894001B69CE
:10B5800098470128014626D0022801D005E0236211
:10B59000236ADA691433002AF9D1236ADA6942B9D5
:10B5A0005869F8B199692162BDE87040C3E9052284
:10B5B0002AE4216A94F824200E7B1433F6B2236225
:10B5C000CAB98EB92846FDF7E1FD28680121BDE81A
:10B5D00070405FF05FBB236A2868143B23625FF012
:10B5E00059FBDAE7206270BDAB68002BEAD01A681D
:10B5F0009B885383E6E7286800215FF04BFB00231C
:10B6000084F82430002EDDD0EEE700BF80690028EA
:10B6100034D003681A6A127B1ABBD3E904125B6840
:10B6200049686AB110B4546800220A6022609A889E
:10B630005DF8044B22F003021204120C9A8095E785
:10B640001A891206FCD41A89D20708D400220A608B
:10B650009A8822F002021204120C9A8086E79A89D4
:10B66000F1E78268002AD8D0116892880A83D3E96A
:10B6700004125B684968002AD4D1E1E7704700BF33
:10B68000806900B97047016830B4D1E904424B6861
:10B69000646872B15568002222602A609A8822F09C
:10B6A00003021204120C9A800B6A1B7B9BB930BCFC
:10B6B0005CE71A891506FCD41A89D20713D4002234
:10B6C00022609A8822F002021204120C9A800B6AFD
:10B6D0001B7B002BEBD08368002BE8D01A689B887B
:10B6E000138330BC42E79A89E6E700BFD3B2012B4F
:10B6F0001DD8104B02EB420210B54FEA820E0EF13C
:10B70000080403F5137C02E01C3363450DD01A785E
:10B710008242F9D15A788A42F6D11A59002AF3D0D6
:10B720000EF1040E03EB0E0010BD002010BD002032
:10B73000704700BF34E5060810B40C4C002304F633
:10B74000A45C01E0152B0CD003EB430201331CF881
:10B7500002108142F6D1144494F9A60D5DF8044B11
:10B7600070474FF0FF305DF8044B7047C81A002057
:10B77000D3B2022B22D870B502EB4202104C4FEA32
:10B78000820E23460EF10C05002204E00132172A36
:10B7900003F12C0310D01E68B042F7D193F804C017
:10B7A0008C45F3D15E59002EF0D02C210EF1080308
:10B7B00001FB0233E01870BD002070BD002070470F
:10B7C000DCD60608002839D030B51D4D90F804C0ED
:10B7D000002305F6A45401E0152B2DD003EB430202
:10B7E0000133A15C6145F7D11544046895F9A63D84
:10B7F00090F805E0DAB2022A1ED803EB43031148A1
:10B800004FEA830C0CF10C050346002204E00132E0
:10B81000172A03F12C030FD019688C42F7D119793C
:10B820007145F4D159590029F1D02C210CF10803AC
:10B8300001FB0233184430BD002030BD704700BF0B
:10B84000C81A0020DCD606080348D0F8403113B1EE
:10B8500000F5987018477047880100200348D0F819
:10B86000643113B100F5AA701847704788010020B1
:10B870000348D0F8883113B100F5BC701847704701
:10B88000880100200348D0F8AC3113B100F5CE7028
:10B8900018477047880100200348D0F8D03113B111
:10B8A00000F5E07018477047880100200348D0F881
:10B8B000F43113B100F5F270184770478801002089
:10B8C0000348D0F8183213B100F5027018477047DA
:10B8D000880100200348D0F83C3213B100F50B700A
:10B8E00018477047880100200348D0F8603213B130
:10B8F00000F5147018477047880100200348D0F8FD
:10B90000843213B100F51D7018477047880100207C
:10B910000348D0F8A83213B100F5267018477047D5
:10B92000880100200348D0F8CC3213B100F52F7005
:10B9300018477047880100200348D0F8F03213B14F
:10B9400000F5387018477047880100200348D0F888
:10B95000143313B100F54170184770478801002077
:10B960000348D0F8383313B100F54A7018477047D0
:10B97000880100200348D0F85C3313B100F5537000
:10B980001847704788010020094B0A4A013800EB2C
:10B99000C00003EB80030848D3F83031116B8342B9
:10B9A00014BF4FF480034FF400130B43136370472D
:10B9B000880100200038024000600240F0B40138E5
:10B9C0003B4C3C4E3C4D00EBC00C04EB8C0CDCF8CB
:10B9D0003071AF4214BF4FF480054FF40015376B40
:10B9E0003D433563354DCCF84831DCF83431CCF883
:10B9F0004011AB424FEAC0013FD005F58065AB4234
:10BA00003BD0A5F57A75AB4246D005F58065AB42D3
:10BA100042D0A5F57A75AB4240D005F58065AB42C2
:10BA20003CD0A5F57A75AB4234D005F58065AB42C4
:10BA300030D0A5F57A75AB4232D005F58065AB42C2
:10BA40002ED0A5F57A75AB422CD005F58065AB42BA
:10BA500028D0A5F57A75AB4226D005F58065AB42B6
:10BA600022D0A5F57A75AB4220D0154D06F5325699
:10BA70003836B34218BF002500E0124D0B1804EB16
:10BA80008304C2F3871194F84501C4F85051F0BC07
:10BA90005CF0AABA0C4DF1E70C4DEFE70C4DEDE769
:10BAA0000C4DEBE70C4DE9E70C4DE7E7044DE5E7FE
:10BAB000880100200038024000600240106002400F
:10BAC00000800028208000100080001800880010EE
:10BAD000008020102080002000880020008020208E
:10BAE0002DE9F04F934A92F8F53D012B85B021D016
:10BAF000022B15D0002300938F4F4FF0000807F161
:10BB0000780A3B78022B17D008F10108B8F1030F2F
:10BB100007F128070AF1050AF3D105B0BDE8F08F57
:10BB200092F8EA3D33B192F8E63D083B18BF012395
:10BB30000093E1E70093DFE79AF903307F4D029726
:10BB4000591C15BFDBB200239B464FF0010B1E466C
:10BB5000DAB2012A00F2DB8006EB460189007300AD
:10BB6000774C019308315FFA88F703E01C34AC424C
:10BB700000F0CD802378002BF8D16378BB42F5D15B
:10BB800060580028F2D011F0B1FF009B814623B12C
:10BB9000A0F10901072940F2BF807A1CD2B214211A
:10BBA000484611F08BFF002800F0B180DDE9013735
:10BBB000334404EB830409F1FF33E068614C5942DC
:10BBC00003EBC30201F0070103F0070358BF4B4228
:10BBD00004EB820104F5987404EB8202C1F83C0185
:10BBE0003A61484681F83831FFF7CEFE9AF90430C1
:10BBF0005A1C00F09A80DEB23246CDE902974F4DD2
:10BC0000F3B29346012B62D806EB4601890073001C
:10BC10004B4C019308315FFA88F902E01C34AC42C6
:10BC200055D02378012BF9D163784B45F6D1605874
:10BC30000028F3D011F05AFF009B07461BB1A0F17A
:10BC40000901072947D909F10102D2B21321384667
:10BC500011F034FF00283AD0019ADDF80890324400
:10BC6000BB4604EB82040BF1FF325142E068354CD5
:10BC7000039F02EBC20501F0070102F0070258BF63
:10BC80004A4204EB850104F5987404EB8505C1F87C
:10BC90003C017D61584681F83821FFF775FEB9F106
:10BCA000000F3DD0BBF1000F1BD02846FCF7B8FBBE
:10BCB0003869FCF7B5FB3846FCF784FB00231A46CD
:10BCC00021495846FFF77AFE01233B731CE70136F2
:10BCD000F3B29B4596D2DDE90297B9F1000F1FD070
:10BCE0001A4C09F1FF33242202FB0340002438617F
:10BCF0007C61FCF795FB3846FCF764FB234614494E
:10BD000022464846FFF75AFE01233B73FCE6013604
:10BD1000F2B25A457FF61DAF029F4FF0000965E76A
:10BD200000220023C7E90423EEE601231A46002679
:10BD300063E700BFC81A0020D828002080E7060863
:10BD400034E50608880100200DB60008B80200207E
:10BD500081B600080C4A0D4903469342D1F8C0074A
:10BD600010D0A2F5806293420CD002F5804293423B
:10BD700008D002F58062934204D002F580629342BB
:10BD800018BF4008704700BF00040140C81A0020D7
:10BD9000800AA0F58010522808D8054B034493F878
:10BDA000F4330D2B02D8034AD05670470020704759
:10BDB000DCD60608EC6A070848B182880449B2FA62
:10BDC00082F208684FF00043D34003430B60704792
:10BDD000003C01400120FDF7C1BA00BF0220FDF781
:10BDE000BDBA00BF0420FDF7B9BA00BF0820FDF7B7
:10BDF000B5BA00BF1020FDF7B1BA00BF4FF478709C
:10BE0000FDF7ACBA4FF47C40FDF7A8BAF0B5054693
:10BE100083B0A0B307681D4B144607F13F4202F5FB
:10BE20007E0203EB92230E4693F860045CF03EFA28
:10BE3000A988B1FA81F3C3F11F03C3F3CC0207EB66
:10BE4000820203F00703156A4FF00F0C9B009C4021
:10BE50000CFA03F325EA03031362136A1C4314620A
:10BE6000C6F30013C6F34112CDE900323846C6F3DB
:10BE7000810306F003025DF0F3FC03B0F0BD034B59
:10BE800093F85F045CF012FA2B68FFDEDCD606083C
:10BE900000B1BBE7704700BF2DE9F047684E06EBE5
:10BEA0000013D3F8984E002C76D093F8A07E054668
:10BEB0004FEA001838465CF0F9F907F01F027F09D5
:10BEC0000123032F03FA02F372D0042F6BD0022F49
:10BED00064D006EB0803013593F89C0E11F0B6FE12
:10BEE000EDB2824610B11223C571837106EB0803CF
:10BEF00093F89D0E11F0AAFE814610B11323C5716F
:10BF0000837106EB080393F89E0E11F09FFE07461F
:10BF100010B11423C571837106EB0803504693F8E2
:10BF20009F5E4A212A46FFF7B3FF2A4648462A2148
:10BF3000FFF7AEFF2A460A213846FFF7A9FF414B1B
:10BF40009C423AD0404B9C4242D0404B9C424AD00B
:10BF50003F4B9C4252D03F4B9C425AD03E4B9C425E
:10BF600062D0A38823F003031B041B0CA380238847
:10BF700003F4415343F4457343F003032380A38B3D
:10BF800023F400631B041B0C0722A3832282238853
:10BF90009BB243F040032380BDE8F0872F4A516AEB
:10BFA0000B43536295E72D4A11690B43136190E7E8
:10BFB0002A4A116A0B4313628BE703F584335A6AEA
:10BFC00042F480525A625A6A22F480525A62C8E796
:10BFD00003F500331A6A42F480421A621A6A22F4A4
:10BFE00080421A62BDE703F5FE331A6A42F400424A
:10BFF0001A621A6A22F400421A62B2E703F5823327
:10C000005A6A42F400525A625A6A22F400525A6240
:10C01000A7E703F568435A6A42F480125A625A6AE3
:10C0200022F480125A629CE703F564435A6A42F490
:10C0300000125A625A6A22F400125A6291E700BF53
:10C04000C81A00200030014000380040003C004089
:10C0500000340140005001400054014000380240CB
:10C06000431C00F056812DE9F04FDFF87CA400EB73
:10C0700080030AEBC30287B0D2F80C90810005461A
:10C080000191DB00B9F1000F06D0D2E90548002C80
:10C0900000F00B81A27912B107B0BDE8F08FB8F1C2
:10C0A000000F00F0608198F80620002AF4D11833C0
:10C0B0000AF10C06F018D9F80470F250691CC0E9B6
:10C0C00001221523C260C9B2A3711623E17188F859
:10C0D000071088F8063099F818005CF0E7F8BB887C
:10C0E0002268A08823F440731B041B0CBB80D8F883
:10C0F00000301083B8F804201A8311212046FEF77F
:10C1000063FC11214046FEF75FFC09264FF0330B1C
:10C110002CB9F5E0BBF1010B08D0FEF713F922684A
:10C12000A188136919424FF00A00F3D0518305200A
:10C13000FEF708F92368A2881A830520FEF702F9A2
:10C14000013EE3D1002C00F03081332603E0013EB4
:10C1500008D0FEF7F7F82268A188136919424FF05A
:10C160000A00F4D051830520FEF7ECF8B8F1000F77
:10C1700000F04881D8F80030B8F804205A83052030
:10C18000FEF7E0F82368A2881A830520FEF7DAF8A4
:10C19000D8F80030B8F804201A830520FEF7D2F84A
:10C1A0002368A2881B691A4240F0B480019B2B448B
:10C1B0000AEBC303997F1A7F002940F0B78020461D
:10C1C0001221FFF723FE1221019B2B440AEBC3032C
:10C1D0005A7F4046FFF71AFEBD4B9F4200F0308168
:10C1E000BC4B9F4200F03781BB4B9F4200F0448123
:10C1F000019B2B440AEBC3034FF47A721C8CBB885F
:10C2000023F440731B041B0CBB803B889BB243F0A0
:10C2100001033B80BD8802A802FB04F425F03F0522
:10C2200057F0BCF90499AD4B2D04A3FB01232D0C51
:10C2300045EA9345BD803A8822F001021204120CAF
:10C240003A80A74A980C9442034675DC6200B1FB21
:10C25000F2F292B20133042A38BF04223B84BA833B
:10C260003B889BB243F001033B803B8823F481630E
:10C2700023F002031B041B0C4FF4804243F4806341
:10C280003B803A813B8823F080031B041B0C3B80DE
:10C2900099F81A0000215BF0A7FE99F81900002117
:10C2A00007B0BDE8F04F5BF09FBEB8F1000F00F0A3
:10C2B000F88098F80620002A7FF4EEAE18330AF1D1
:10C2C0000C01CA18D9F80470CC50C2E901441623F5
:10C2D000D46088F806306B1C88F8073099F818008D
:10C2E0005BF0E4FFBB88B8F8042023F440731B0420
:10C2F0001B0CBB80D8F800301A8302E7FEF722F847
:10C30000BBF1010B4FF00A00F8D10520FEF71AF837
:10C3100013E77047019BD8F800202B440AEBC303B6
:10C3200012699A7F002A00F0A1801A7F32212046EC
:10C33000FFF76CFD322147E704EB4404B1FBF4F155
:10C340008AB2C1F30B0109B942F0010265494FF409
:10C35000967300FB03F3A1FB03139B09013342F423
:10C3600000423B847BE70AF10C011833CA18D9F864
:10C37000047041F80380C2E901881523C2F80C80DB
:10C38000A371431CE37199F818005BF08FFFBB8821
:10C39000A28823F440731B041B0CBB80236811216B
:10C3A0001A832046FEF710FBAFE6332401E0FDF7C9
:10C3B000C9FF013C4FF00A00F9D10520FDF7C2FF8B
:10C3C000B8F1000F63D0D8F80030B8F804205A83D1
:10C3D0000520FDF7B7FF0520FDF7B4FFD8F80030C2
:10C3E000B8F804201A830520FDF7ACFF019B2B440D
:10C3F0000AEBC3039A7F002A18BF32215A7F08BF75
:10C400001221E6E60520FDF79DFF2368A2881A8326
:10C410000520FDF797FF0520FDF794FF2368A2880C
:10C420001B691A4262D1019B2B440AEBC303997F1B
:10C430001A7F002969D020463221FFF7E7FCCBE6BE
:10C4400003F5F2331A6A42F400121A621A6A22F4ED
:10C4500000121A62CCE603F5F0331A6A42F4800245
:10C460001A621A6A22F480021A62C1E61A7F204612
:10C470001221FFF7CBFCA6E603F5EE331A6A42F46D
:10C4800000021A621A6A22F400021A62B0E605205B
:10C49000FDF758FF0520FDF755FF0520FDF752FF7A
:10C4A0009AE618330AF10C01CA18D9F8047041F859
:10C4B0000380C2E90188C2F80C8099F818005BF08B
:10C4C000F5FEBB8823F440731B041B0CBB801CE6E9
:10C4D0000054004000580040005C004083DE1B43D5
:10C4E000A0860100D34D6210C81A0020019B2B4486
:10C4F0000AEBC30320469A7F002A18BF32211A7F15
:10C5000008BF1221FFF782FC66E620461221FFF7E2
:10C510007DFC61E62DE9F8430746FDF773FBDFF884
:10C520004C8007EB8709044608EBC90542F20F76F9
:10C5300004E0FDF767FB001BB0420BDC95F82530EB
:10C54000002BF6D108EBC90898F8240080F0010010
:10C55000BDE8F883B8F8C83E013338469BB2A8F866
:10C56000C83EFFF77DFD0020BDE8F883C81A002013
:10C5700010B582B004468DF807300DF107035BF06B
:10C5800029FE08B902B010BD2046FFF7C3FF02B074
:10C5900010BD00BFB0F1FF3F6DD02DE9F04F022874
:10C5A00083B0044614DC354E984600EB800306EB5E
:10C5B000C305DB00D5F810A00093BAF1000F07D037
:10C5C000894695F82510934601F0FF02019219B1B2
:10C5D000002003B0BDE8F08FFDF714FB009B019A2B
:10C5E000203307464FEA490106F10C00C9B200EBBF
:10C5F000030C85F826104FF0010E0C9985F827B032
:10C6000085F8292085F82AE0C150CCF8041085F877
:10C61000288085F825E085F82420BAF804309905AB
:10C620001DD4BAF80030DA0512D442F20F7504E0D6
:10C63000FDF7E8FAC31BAB4213DCBAF800309B05E8
:10C64000F6D4BAF800309BB243F48073AAF80030F5
:10C65000BAF804309BB243F44073AAF804300120C6
:10C66000B7E7B6F8C83E01339BB22046A6F8C83EED
:10C67000FFF7F6FCACE70020704700BFC81A0020A7
:10C68000E0B5294E00EB800306EBC30384B0DA6803
:10C690005568AA8A92B20392039A12F4706F1CBF73
:10C6A000012283F82420039B13F4E06F4FEA8007F4
:10C6B0000DD1AB8A074423F4706306EBC7061B0455
:10C6C0001B0C0022AB8286F8252004B0E0BD2B8B2A
:10C6D000AB8823F480631B041B0CAB80039B9A057F
:10C6E000E7D42B889B05E4D42B88D9050FD52B885C
:10C6F000DA05FCD42B889BB243F400732B802B8883
:10C700009B05FCD40190FFF7ABFC0198D1E72B8887
:10C710009BB243F400732B80AB8823F440731B045B
:10C720001B0CAB80C5E700BFC81A00200020A7E79C
:10C730000120A5E70220A3E770B590F871301C092D
:10C74000013C052C0FD81A4E06EB4402054632F880
:10C75000540C03F00F0340FA03F2D20703D595F807
:10C760007D20012A01D0012070BD9A40013A10407D
:10C77000264460F00BFE16F8483C0E4A034402EBD8
:10C78000C30452F83320A38810691840ECD0EB6E34
:10C79000002285F87D2093F8212002212046FFF712
:10C7A00035FB2A6E93899BB243F008039381DAE745
:10C7B000D4E7060830230020094BD3F8CC2ED3F859
:10C7C000D01E40F22A40002350604B620B889BB27F
:10C7D00043F001030B80136843F0010313607047BB
:10C7E000C81A002010B41D4B1D48196C1D4A41F099
:10C7F0008051012485B0196404625321FF24CA20AA
:10C800005462506251625B6FDB0017D416480423F8
:10C81000002102910290029A1A440292029A043371
:10C820001C2B1160F5D103910390039B0393039B91
:10C830000E4A1A6005B05DF8044B70470A4B00229F
:10C8400001920193019B0193019A084B12689A424D
:10C85000DCD105B05DF8044B704700BF00380240E2
:10C8600000000E420028004050280040316665421A
:10C8700030B5154C154D85B00139002389B2A04261
:10C88000ADF80C30ADF806308DF80E300291D5F8C9
:10C89000C0370FD00E4988420CD001F58041884244
:10C8A00008D001F58061884204D001F5806188429A
:10C8B00018BF5B08B3FBF2F301A9013BADF80430EC
:10C8C00057F0D2F805B030BD00040140C81A00206E
:10C8D000000001402DE9F041046ED0F80880A389E2
:10C8E00023F400531B0407461B0C90B0A38143792B
:10C8F0003D79C3F38000190305F001061B0215F012
:10C9000002054FEA00304FEA860203F4806318BF45
:10C9100042F0080203431A43238A9BB201F40051F8
:10C9200023F440530B432382A38923F4B05323F011
:10C930000C031B041B0C1A43A281A38A23F440732B
:10C940001B041B0CA38201A856F028FE6B4B9C42D3
:10C9500005D003F580639C4201D0039B00E0049B5B
:10C96000A2896749A089120403EB83034CBF4FEAF5
:10C9700048084FEA880803EB8303B3FBF8F3A1FBF5
:10C9800003C252094FF0640C00040CFB12334FEA4F
:10C99000021200F19A801B013233A1FB0313C3F38F
:10C9A000431313439BB2238197F9380097F805800E
:10C9B000FCF7D9F930B10368828818F0010F14BF71
:10C9C0001A835A8318F0080FA38A78D09BB243F0D9
:10C9D0000803A382A3899BB243F40053A381002ED2
:10C9E0002FD0FE6B002E7DD00023CDE90833CDE99A
:10C9F0000C33CDE90E33049306937B6C0193FB6DEE
:10CA00000293FB6805937B6903934FF480714FF4A5
:10CA10008033CDE90A1330464FF48063079356F014
:10CA200007FE01A9304656F099FE336843F0010332
:10CA30003360A38A9BB243F04003A38273689BB226
:10CA40007B65002D33D03E6C002E46D0BB6C01932D
:10CA5000BB6D02933B690593402304934FF48033ED
:10CA6000002530460B934FF480630793CDE90855BA
:10CA7000CDE90C55CDE90E55039506950A9556F06E
:10CA8000D7FD01A9304656F069FE736943F0800373
:10CA90007361336843F0160333607560A38A9BB2F9
:10CAA00043F08003A382E36843F04003E360A3897B
:10CAB0009BB243F40053A38110B0BDE8F08123F092
:10CAC00008031B041B0CA38284E7DB003233A1FBA9
:10CAD0000313C3F34213134364E7E36843F0800393
:10CAE000E360E0E74FF6DF732380E36843F0200361
:10CAF000E360E36843F01003E360A2E70010014045
:10CB00001F85EB518160E5E60171E3E6BFF34F8FCE
:10CB10000549064BCA6802F4E0621343CB60BFF3D9
:10CB20004F8F00BFFDE700BF00ED00E00400FA05F5
:10CB300008B50021032056F093FE72B6FFF7E6FF1A
:10CB4000154C08B5D4F8D43E94F8DA0EABB91420DD
:10CB5000FDF788FC00BFD4F8D43E5BB11A689B880F
:10CB6000116994F8DA2E0B4012B91BB1FFF7E0FF00
:10CB7000002BFBD0FCF7E0F9ECE719689A880B6909
:10CB8000134020B1002BE2D10B691340FAE7002BD0
:10CB9000DDD00B691340FAE7C81A002008B572B659
:10CBA000FFF7B4FF00B583B00D4900220092009159
:10CBB000009B0C330093009B1B68012B02D003B039
:10CBC0005DF804FB01920191019B06490C3301932E
:10CBD000019B1A600B6883F308884B689847FEE74F
:10CBE000502800400000FF1F38B5FFF7FBFDFFF79E
:10CBF000D9FF012056F044FE6E4A936823F00303E8
:10CC00009360936813F00C0FFBD113686949A0B9C6
:10CC100043F00103136041F2883302E0013B00F06E
:10CC2000C7800A689507F9D5634C00220823C4F829
:10CC3000DC2EC4F8E03E02251EE043F4803313608E
:10CC400041F2883302E0013B00F0B2800A689403AD
:10CC5000F9D5594C594B5A4DB0FBF5F5B0FBF3F0F3
:10CC6000B5EB400F18BF28464FF48003C4F8DC3EF4
:10CC7000C4F8E00EB5FBF0F50220C4F8E45E56F00F
:10CC8000FFFD03280DD84F4B03EBC0039988DA88CA
:10CC9000C4F8EC1E5B88C4F8F02EB3FBF5F3C4F8BF
:10CCA000E83E444B48491A6C42F080521A640A68C4
:10CCB00042F440420A609A689A609A6842F40042DC
:10CCC0009A609A6842F4A0529A60D4F8DC1ED4F8B4
:10CCD000E02E0A43D4F8E81E42EA8112D4F8F01E8E
:10CCE00042EA0162D4F8EC1E4908013942EA0142E5
:10CCF0005A601A6842F080721A601A689201FCD574
:10CD0000324A40F205711160996821F0030199607F
:10CD1000996841F00201A2F580629960936803F07E
:10CD20000C03082BFAD12A49D823B3FBF5F39B0156
:10CD300043F000530120C2F884308866FCF740F8C5
:10CD4000244D1C4B244AEA60596F244AC4F8F41E4F
:10CD5000AA605A6B224922F080025A635A6F42F04D
:10CD600080725A671A6B42F4CE021A635A6B5A6386
:10CD70009A6B9A631A6C0A431A64596C194A0A43EB
:10CD80005A64FCF74DF9184AD4F8C037A2FB0323C4
:10CD90009B09013BB3F1807F09D24FF0E022F020E4
:10CDA00053610021072385F823009161136138BD89
:10CDB000014CC5E700380240C81A002080841E00DC
:10CDC00040420F0094E7060800700040003C02401B
:10CDD0000000474200ED00E00005FA0500000020D9
:10CDE000FFC9FE36335F0700D34D621030B50468CB
:10CDF0002A482B4D85B00139002389B28442ADF811
:10CE00000C30ADF806308DF80E300291D5F8C037F1
:10CE10000FD024498C420CD001F580418C4208D0BF
:10CE200001F580618C4204D001F580618C4218BF0D
:10CE30005B08B3FBF2F301A9013B2046ADF80430D7
:10CE400056F012FE2288184892B242F001020023E6
:10CE500000F54F61228051F83320944208D001330D
:10CE60000E2BF8D1002005B0BDE83040FBF780BDA7
:10CE700000EBC30090F8F54C2046FBF779FD1B2C26
:10CE800005D02E2C08BF2C20EDD005B030BD1920C8
:10CE900005B0BDE83040FBF76BBD00BF00040140AA
:10CEA000C81A002000000140DCD6060870B50468EE
:10CEB000A30AA3F58013522B50D8364D2B4493F878
:10CEC000F4C3BCF10D0F49D84379022023FA00F5D1
:10CED0000CEB8C03A8400CEB43031FFA80FE2B44A1
:10CEE000002949D0A5892C48ADB200EB830645EA5C
:10CEF0000E05C6F85415C6F86425A581EFF3118612
:10CF0000502383F312882C2202FB0C03D3F8501514
:10CF100061B3C3F87415214B04310CEB8C02204D26
:10CF20000CEB4202920005EB020E1032134453F850
:10CF3000042F0AB10A60111D7345F8D10022F3B223
:10CF40000A6083F311882C2303FB0C00D0F874359E
:10CF50002BB1A3899BB243F00103A38170BDA389C8
:10CF600023F001031B041B0CA38170BD0B4B02FBC0
:10CF70000C3202F12401D0E7A08980B220EA0E0031
:10CF8000A081054800EB8305C5F85415C5F8642554
:10CF9000B4E700BFDCD60608C81A0020182000201D
:10CFA0003820002001490248FCF7F6B9182000207B
:10CFB0000000014010B5064C064804F5AA61FCF7D4
:10CFC000EBF904F2DC610448BDE81040FCF7E4B979
:10CFD000C81A0020000001400044014002494FF0FF
:10CFE0008040FCF7D9B900BF442000200149024825
:10CFF000FCF7D2B97020002000040040014902482B
:10D00000FCF7CAB99C2000200008004001490248F2
:10D01000FCF7C2B9C8200020000C004001490248BA
:10D02000FCF7BAB94C2100200004014010B5064CB1
:10D03000064804F28461FCF7AFF904F5EC6104489A
:10D04000BDE81040FCF7A8B9C81A00200004014050
:10D05000001C004001490248FCF79EB978210020DD
:10D060000040014001490248FCF796B9D021002058
:10D070000048014001490248FCF78EB9FC2100201C
:10D080000018004001490248FCF786B954220020EC
:10D090000020004010B50C2935D8DFE801F09134AC
:10D0A000343463343434073434343500038C5488D6
:10D0B000B2F80CE023F480731B041B0C0384038C74
:10D0C000B0F804C0818B21F073014EEA040E09040C
:10D0D000148823F40073090C1B042143764C1B0CA9
:10D0E00043EA0E23A0421FFA8CFC9BB200F094800E
:10D0F00004F58064A04200F08F809268A0F804C01C
:10D100008183C263038410BD038C5488B2F80CE0A1
:10D1100023F480531B041B0C0384038CB0F804C05D
:10D12000818B21F4E6414EEA040E0904148823F4AD
:10D130000053090C41EA04211B045F4C1B0C43EA19
:10D140000E33A0421FFA8CFC9BB289B27ED004F54C
:10D150008064A0427AD09268A0F804C081830264FF
:10D16000038410BD038C5488B2F80CE023F0100344
:10D170001B041B0C0384038CB0F804C0018B21F446
:10D18000E6414EEA040E0904148823F02003090C3A
:10D1900041EA04211B04484C1B0C43EA0E13A04235
:10D1A0001FFA8CFC9BB289B26CD004F58064A0425B
:10D1B00068D09268A0F804C001838263038410BD24
:10D1C000038C5488B2F80CE023F001031B041B0C01
:10D1D0000384038CB0F804C0018B21F073014EEA84
:10D1E000040E0904148823F00203090C1B042143D4
:10D1F000314C1B0C43EA0E03A0421FFA8CFC9BB27D
:10D200002CD004F58064A04228D09268A0F804C015
:10D2100001834263038410BDD489B2F810E023F483
:10D22000006343EA0423548A2CF4405C4EEA040E63
:10D230004CEA0E1C94884FF6FF3E03EA0E0E4EEAAF
:10D24000042E1FFA8CFC1FFA8EF356E7148A2CF476
:10D25000804C4CEA841C1FFA8CFC7CE7D489B2F821
:10D2600010E023F008032343548A2CF4407C4EEA58
:10D27000040E948823F004034CEA0E0C1FFA8CFC75
:10D280002343C2E7D489B2F810E023F0800343EAD5
:10D290000413548A2CF4406C4EEA040E4CEA8E0CB3
:10D2A00094884FF6BF7E03EA0E0E4EEA041E1FFA64
:10D2B0008CFC1FFA8EF37CE7000001402DE9F04F53
:10D2C000B14BDFF8DC8293F8F6EDB04CB04D95B081
:10D2D0000EF1FF37FBB200930023CDE9013EC246B9
:10D2E000DFF8C0B2DBF80070BB0AA3F58013522B45
:10D2F00000F20A81234493F8F4330D2B00F20481E9
:10D3000015F90390029B012B00F00981029B022B6F
:10D3100002D1B9F1080F6DD100263146484611F00F
:10D32000E5F911F06FFA037813B1542B40F0F08255
:10D330000436B6B2102EF0D1019B002113B3424641
:10D340000BE0234493F8F4330D2B0DD8EB564B45EB
:10D350000DD002F58072524512D0906803689B0A86
:10D36000A3F58013522BECD900234B45F1D143791F
:10D370009BF8050098423DD002F580725245ECD1F1
:10D38000002937D15846FBF761F8C3B2022B9BF84E
:10D3900005E000F20A8300F1010C7C4A0CEB4C0C16
:10D3A0004FEA8C0C02F57D7003E02C32824200F0D3
:10D3B000FC8213689F42F8D113797345F5D152F876
:10D3C0000C30002BF1D07348002142689A4200F0E3
:10D3D000A2800131102900F12400F6D14FF0FF3373
:10D3E0006D4A03EBC30302EB830393F84C31002B2C
:10D3F00000F0A182694B0BF11C0B9B457FF472AFCF
:10D40000019B0133042B01930AF5807A7FF468AF06
:10D41000DFF894B1DBF8183605934FF0000A0BF2F1
:10D4200044530BF581690193CDF800A0059B009A48
:10D43000934266DD544BD9F80C7093F8F82E99F8A6
:10D4400010300393002F5CD03B68DBF8040004939A
:10D4500003F13F4505F57E05BB88029300284FEA9E
:10D46000952564DD002302E0013383425CD01C0279
:10D4700058F80410A942F7D14444039B89F81030AE
:10D48000029B009DC9F80C70B3FA83FCCCF11F0617
:10D490004FF003020135C9F80460C9F81840BA71A9
:10D4A000FD717300E16C606C012203279F4002FA5A
:10D4B00003F319439BF80030E164384302FA06F69F
:10D4C0006064276DD4F8A000B1B2002B00F0268272
:10D4D0003E432665049E029B3383FAF7F1FF204604
:10D4E000FBF742F940F20112A9F81C20019A0095BD
:10D4F00001235374082D02F1180309F12009019347
:10D5000094D115B0BDE8F08F009B012B7FF672AF70
:10D510004FF0000900E74B1CDBB2013B60E7B9F1BB
:10D52000010F3FF4F9AE65E7042B00F007820BEB27
:10D5300000230102069119690791002900F02B824E
:10D540006C1C0892E4B24FF054029D6083F80421F1
:10D5500083F80541079B01305E79CBF8040018463B
:10D560001D680996FAF772FFC3B2022B00F21D8202
:10D5700000F1010C0CEB4C0C044B089A4FEA8C0C9C
:10D580000021B64618E000BFC81A0020DCD6060805
:10D59000EC6A0708B802002088010020B0E80608FD
:10D5A0000C000010B4E70608040000100131172930
:10D5B00003F12C0300F0F9811E68B542F6D11E7903
:10D5C0007645F3D153F80C60002EEFD02C2300EBFE
:10D5D000400001FB03F3BC49DFF830A303EB8003F9
:10D5E0000B4450461969069B0C915B44C3E90661E4
:10D5F000002105E00131102900F1240000F0A28192
:10D600004368B342F6D14B1CDBB2B049013B03EB9C
:10D61000C30301EB830393F84C110B91002940F0F5
:10D620009181069883F84D41C11101EB2021A84C4E
:10D6300001EB011104EB8104069908948C20A54CA0
:10D64000091200FB01F104EB410C0699089CCDF88E
:10D6500028C05944C1F8F400C1F8A8400498C86033
:10D66000542483F84C419C48C1F8F0C03323C1F8DE
:10D67000AC309A4B0699D3F8C037854208EB0104C9
:10D680000FD097498D420CD001F580418D4208D0D2
:10D6900001F580618D4204D001F580618D4218BF93
:10D6A0005B08062A00F07481072A8E488E4A8F494B
:10D6B00018BF11468E4A18BF02460698B3FBF2F215
:10D6C000B3FBF1F3013A0BEB000192B2013BA1F87D
:10D6D000B030A1F8682000F154010023A4F85C30B8
:10D6E000284648F80130A265414456F0BDF90023B0
:10D6F000ADF840302B8809999BB243F080032B8012
:10D700002B8823F001031B041B0C2B80794B0F93F8
:10D710004FF0020E4FF48073CDE912E328460A233E
:10D720000FAA1193FFF7B6FC079B1879002840F069
:10D7300019812B889BB243F001032B800023DAF878
:10D740000420964203F1010300F00881102B0AF136
:10D75000240AF4D14FF0FF335C4A6749674803EB72
:10D76000C30302EB8303664AD3F830318B4214BF04
:10D770004FF480034FF40013116B0B431363099AAA
:10D780000C2A9BBF5F4B03EB42030022B3F8DC2063
:10D79000069B5B449A82002306E08D4200F00081E4
:10D7A0000133042B00F0FE8050F833100029F4D12F
:10D7B000DBF8041A0131CBF8041A0BEBC301DB00D0
:10D7C000C1F8085A03440B9899880A439A804E4935
:10D7D00023469022FEF7F2F83368069A049843F045
:10D7E00010033360089BE3660C9B636602F16401DF
:10D7F00004234FF40032C4E9232340233322C4E935
:10D800001C3200F1180200254FF4806AA2664FF422
:10D8100080504FF48042C4E9200241443046C4E9BC
:10D820002555A567C4F88850C4F89C50C4F87CA05E
:10D8300055F094FF3068E0617069206270680C9B5D
:10D840006062B068A062F068C4F8AC300423C4F829
:10D85000D8300A9BE062C4F8B4300498069AC4F841
:10D86000C4A04FF44033C4F8D4308C23C4F8BC3087
:10D8700000F1100302F1AC01C4F8B0304FF4804263
:10D880004FF40063C4F8C830C4E937554144C4F8C4
:10D89000CC20C4F8B850C4F8C050C4F8D050C4F874
:10D8A000E450304655F05AFF33682363736963636D
:10D8B0007368A363B368E363F3682364336843F076
:10D8C00010033360D9E500BFDCD6060888010020CC
:10D8D000C4290020F42C002000040140C81A0020B4
:10D8E00000000140D0DD06004495080010552200DC
:10D8F00040771B0060000100006002400C0A00102D
:10D9000000380240D4E7060809850008B802002064
:10D91000019B0121002B7FF412AD6BE5CCF12F0CA4
:10D9200002FA0CF23A432265049A029E56831A4682
:10D93000FAF7C6FDD3E5CAF808B061E51C4A03232F
:10D9400082F8F93E1B491C4A1C4BCBF8501ACBF805
:10D95000482ACBF8583A15B0BDE8F08FDBB20B93EC
:10D96000013BF9E610F072F90D9038B1079B0221E6
:10D97000DA79FEF74BFA0D9B5422DA80B5F8443081
:10D980006FEA43436FEA53439BB2A5F84430D0E6B5
:10D990000B490C4A91E6064A022382F8F93ED1E788
:10D9A000DB000FE700239B88FFDE00235B68FFDEC0
:10D9B000C81A0020BD8C0108B98C0108C58C01086B
:10D9C000882A1100A0BB0D000C2911D8DFE801F056
:10D9D0002310101019101010111010100700838B55
:10D9E00023F400631B041B0C43EA02239BB28383D2
:10D9F0007047838B23F008031B041B0C1A4382839C
:10DA00007047038B23F400631B041B0C43EA0223BF
:10DA10009BB203837047038B23F008031B041B0C8A
:10DA20001A430283704700BF2DE9F04F994D2B78C0
:10DA300089B01BB9012009B0BDE8F08FDFF864920E
:10DA4000D9F80040FCF706F995F89C3A0393002BAF
:10DA500000F01482904BA3FB0432904B5209A3FBBD
:10DA60000213DB0803EB8303A2EB4303D5F8142670
:10DA7000821A049205F21C6BDAB207920BEB830355
:10DA800009F1E80405F6FC02029200279846019489
:10DA900032E0304655F0CCFD8C2303FB0793002584
:10DAA00083F8DC509AF805A0204651462A46FFF735
:10DAB0008BFF019C2246FFF7EDFA51460822FFF743
:10DAC00083FF402344F83C3CA4F14801304655F024
:10DAD00045FE04F18C030193029B143302933368D7
:10DAE00043F010033360039B01379F420BF15C0B43
:10DAF00008F15C0800F0D880049A002A05DB019B3D
:10DB000053F8083C934200F3A5818C23019A03FB50
:10DB1000079352F858AC93F8DC30166ADAF80040F4
:10DB2000002BB6D07568A389ADB2114632F8542CDB
:10DB3000C5F116059BB223EA0203072DA381A8D9DC
:10DB4000544AD2F804390133C2F804398A6A0021F0
:10DB5000CDE90572106896468C46012315E0BCF1AC
:10DB6000140F1EDC12F1080748BF02F117073A1123
:10DB70000CEB271C571E01FA02F201210B4401FA9B
:10DB800007F79D4247EA02010BD302465EF8040FF5
:10DB90009D42A0EB0202E2D8CCF115024FF0150C29
:10DBA000E8E7BCF1150FDDE9057266D13C4DC1F324
:10DBB0008423C1F3441005EB830305EB8000D3F805
:10DBC000F830D0F8F8001B0243EA001301F01F0000
:10DBD00005EB8000C1F3C43105EB8101D0F8F800FA
:10DBE000D1F8F810034343EA013383EA132181EAB1
:10DBF000111101F00F010F293FD1C3F30F134FF69D
:10DC0000FF718B4239D0B3F5606F00F02781029A23
:10DC100093819BF858200798824214D0D8F80810B6
:10DC2000DBF80020521ACBF80020D8F83010DBF8CF
:10DC30000420521ACBF804200022C8F80820C8F8A3
:10DC400030208BF85800DBF800200132CBF80020A0
:10DC5000D8F808200132C8F808204FF6FF72934226
:10DC60007FF417AFDBF804300133CBF80430D8F879
:10DC700030300133C8F830300BE70649D1F80039AD
:10DC80000133C1F80039002F00F0DA804FF6FF733E
:10DC9000BFE700BF040000101F85EB51CDCCCCCCFA
:10DCA000D4E70608C81A0020794AD9F89010C2F8BB
:10DCB0001456012382F8003A0A68487999F89810B6
:10DCC000890748BF0423118C83409BB289B221EAA3
:10DCD00003011184118C89B20B431384039B012B24
:10DCE0003FF4A8AED9F81C211368517999F8242182
:10DCF000970754BF012204228A40198C92B289B23C
:10DD000021EA02011984198C89B20A431A84039BFF
:10DD1000022B3FF48FAED9F8A8211368517999F8F6
:10DD2000B021960754BF012204228A40198C92B276
:10DD300089B221EA02011984198C89B20A431A8432
:10DD4000039B032B3FF476AED9F834221368517944
:10DD500099F83C22950754BF012204228A40198C6D
:10DD600092B289B221EA02011984198C89B20A435C
:10DD70001A84039B042B3FF45DAED9F8C0221368CC
:10DD8000517999F8C822940754BF012204228A408D
:10DD9000198C92B289B221EA02011984198C89B2D4
:10DDA0000A431A84039B052B3FF444AED9F84C2355
:10DDB0001368517999F85423900754BF0122042223
:10DDC0008A40198C92B289B221EA02011984198C15
:10DDD00089B20A431A84039B062B3FF42BAED9F871
:10DDE000D8231368517999F8E023920754BF012290
:10DDF00004228A40198C92B289B221EA0201198464
:10DE0000198C89B20A431A84039B082B7FF412AE43
:10DE1000D9F8642499F86C141368507911F0020F42
:10DE200018BF0422198C08BF0122824092B289B225
:10DE300021EA02011984198C89B20A431A84F9E58E
:10DE40001146144858225FF0B5F9DAF800404FF651
:10DE5000FF73DEE6002009B0BDE8F08F99F8E924F1
:10DE600002EB420209EBC2023A4492F8F9240D2A6D
:10DE70007FF4CDAE029980228A77CAE6044A012354
:10DE800082F8003A1346039AC3F81426D2E500BF7D
:10DE900004000010AC09001008B9002070472DE9FB
:10DEA000F04F002299B02F21054610F0FFFC81466B
:10DEB000C8B1DFF84C830668C8F8D06EFDF782FC65
:10DEC00088B1D0E9014AC8F8CC4E64B1BE4F0022F7
:10DED0003946384643689C4200F1240002F10102B1
:10DEE00005D0102AF6D1002019B0BDE8F08FD2B2CB
:10DEF000B64B013A02EBC202900003EB820292F8A9
:10DF00004CB1BBF1000FEED10A182F2128469183A6
:10DF10000FF09CFEAE4D2F21C5F8940528B1C180AD
:10DF200099F807202A21FDF771FFAA4B002203F57B
:10DF30004F6050F832108E4200F0148101320E2AE8
:10DF4000F7D100205AF0B2F93188D8F8C02721F073
:10DF500001010904090C31809F498E4200F0E980DB
:10DF6000A1F580618E4200F0E48001F580418E428F
:10DF700000F0DF8001F580618E4200F0DA8001F56B
:10DF800080618E42954900F00C81B1EB520F4FEA4F
:10DF9000520040F2FA8001220021B0FBF2F2ADF80B
:10DFA00004108F498F48120AA1FB02210A09A0FB25
:10DFB00002025208A5F89A2509095200A5F89825E9
:10DFC0000291002501A93046ADF80C50ADF806507D
:10DFD0008DF80E5055F048FD99F80620ADF8145014
:10DFE00060219307CDE906550895049199F80550ED
:10DFF00040F1A480D20002F008024FF00408ADF80E
:10E000001E20ADF8148004AA29463046FFF742F8D6
:10E0100008222946FFF7D8FCB6F844206FEA4242AE
:10E020006FEA524292B2A6F84420328892B242F08D
:10E0300080023280328C08FA05F39BB292B222EA57
:10E0400003023284328C92B21343338433889BB2FE
:10E0500043F0010333803A46002351688C4202F1B9
:10E06000240203F1010377D0102BF6D14FF0FF33D8
:10E07000564A5D4903EBC30302EB83095B4AD9F8B7
:10E0800030318B4214BF4FF480034FF40013116BF7
:10E090000B43136300237A68944207F1240703F1CA
:10E0A00001035CD0102BF6D1514960220023584661
:10E0B000FDF784FC204655F0BBFA236823F00103EA
:10E0C0002360204655F0B4FA06F134032B440A933A
:10E0D00040F22A430D934FF480630F93454B0B930B
:10E0E00040230C934FF480504FF480430027CDE938
:10E0F000100309A94FF440332046CDE91477CDE948
:10E100001677CDF824A00E971297139355F026FB9F
:10E110000C2D04D8384B03EB4503B3F8DC70B389FE
:10E120009BB23B43B381236843F01003012023607B
:10E13000DAE62A498A421AD2002130E7520002F078
:10E1400002024FF001084FF48073ADF81C20ADF8C7
:10E150001280ADF8203056E7DBB2013B88E75FFA6A
:10E1600083FBA1E703EBC20C9CF8F40CEAE623481E
:10E1700002F1B77101F55851A0FB0101890D013978
:10E1800089B2481CB2FBF0F209E71C4900F1B772F2
:10E1900002F55852A1FB0221890D013989B24A1CAE
:10E1A000FBE68A4204D201200021B2FBF0F2F6E63F
:10E1B000124802F1B77101F55851A0FB0101890D18
:10E1C000013989B2481CF0E7B8020020880100201C
:10E1D000C02B0020DCD6060800040140006CDC02E5
:10E1E000598B4F01ABAAAAAA006002400038024036
:10E1F000BD870008C8970020D4E70608819F5E16F7
:10E20000C81A00202DE9F043013B87B00E683C4F4F
:10E21000BDF838809DF83C909BB20293394B0C4678
:10E22000BE424FF00001D3F8C037ADF80C100546E0
:10E23000ADF806108DF80E100FD033498E420CD079
:10E2400001F580418E4208D001F580618E4204D0F4
:10E2500001F580618E4218BF5B08B3FBF2F301A9A0
:10E26000013B3046ADF8043055F0FEFB6779A379E9
:10E27000B9F1000F01D083F001030022CDE904229F
:10E28000ADF80820602201929A072BD5DB0003F03D
:10E290000803ADF812300423ADF80830304601AA67
:10E2A0003946CDF80C80FEF7F5FE39460822FFF717
:10E2B0008BFBB6F844306FEA43436FEA53439BB29B
:10E2C000A6F84430338832469BB243F0010322F86B
:10E2D000343B63796E60D01800212860D15007B0BC
:10E2E000BDE8F0835B0003F00203ADF810300123BA
:10E2F000ADF806304FF48073ADF81430CEE700BFB0
:10E3000000040140C81A00200000014010B4104A67
:10E3100092F8B83703F0FF01002BF9D10D4B0E4CEA
:10E32000D3F89C052468B3F8B0354FF0010C82F89F
:10E33000B8C74360616223889BB243EA0C03238021
:10E3400003685DF8044B43EA0C030360704700BFA9
:10E35000C81A0020C02B0020B83C002030B58BB07C
:10E360004FF0010C00910021CDE90123CDE904110A
:10E37000CDE9061105688DF80CC004468DF820C063
:10E380000991EFF3118C102383F3128803681B6A41
:10E390000BB3029B684602461BB1D3691432002BB3
:10E3A000FBD12B6A6BB1996839B99A4209D01968C7
:10E3B00029B15B6899680029F7D01433F3E7C3E902
:10E3C00000405FFA8CFC8CF311882268136A002BE2
:10E3D000FCD10BB030BDC5F820D05FFA8CFC8CF3BB
:10E3E0001188FCF711FDF0E738B590F82830012BC3
:10E3F000044606D0407F08B9012038BD002363776A
:10E4000038BD406A03681A7B82B9637F002BF3D062
:10E41000094D0A4902232A1DFFF7A0FF6B79D84353
:10E4200003F0010300F001006377E9E71B6A002BAA
:10E43000EBD0002038BD00BFB83C0020F80400201D
:10E4400038B5044694F82830012B07D0637F0BB110
:10E4500000236377012038BD1B6A23B1606A03681B
:10E460001A7B002AF8D1637F002BF3D0064D0749B1
:10E4700002232A1DFFF772FF6B7903F00102DB070D
:10E480006277E7D5DEE700BFB83C0020F804002043
:10E4900030B593B000238DF807108DF806200DF1EC
:10E4A00006010122CDE90332CDE90631CDE908327A
:10E4B0000DF107058DF814308DF828208DF83C20DB
:10E4C0000B930E93109300220023CDE90C230168D7
:10E4D00002950446EFF3118C102383F3128803682E
:10E4E0001B6A0BB3049B02A802461BB1D36914320A
:10E4F000002BFBD10B6A6BB1996839B99A4209D0EC
:10E50000196829B15B6899680029F7D01433F3E7DB
:10E51000C3E900405FFA8CFC8CF311882268136A0F
:10E52000002BFCD113B030BD02AB0B625FFA8CFC48
:10E530008CF31188FCF768FCF0E700BF30B593B0AE
:10E540000DF1070508920022CDE90252CDE906221D
:10E550008DF807108DF81420012109930B920E926B
:10E5600010920023002204918DF828108DF83C10A1
:10E57000CDE90C2301680446EFF3118C102383F3DB
:10E58000128803681B6A0BB3049B02A802461BB1E6
:10E59000D3691432002BFBD10B6A6BB1996839B97E
:10E5A0009A4209D0196829B15B6899680029F7D0A7
:10E5B0001433F3E7C3E900405FFA8CFC8CF3118855
:10E5C0002268136A002BFCD113B030BD02AB0B6282
:10E5D0005FFA8CFC8CF31188FCF716FCF0E700BFA7
:10E5E00030B595B000230122CDE90532CDE90833DD
:10E5F0008DF81C300D93109312930DF10F030DF154
:10E6000007050B928DF830208DF844200A930022E4
:10E6100000238DF80710CDE90E2301680495044608
:10E62000EFF3118C102383F3128803681B6A1BB36A
:10E63000069B04A802461BB1D3691432002BFBD100
:10E640000B6A6BB1996839B99A4209D0196829B136
:10E650005B6899680029F7D01433F3E7C3E90040F9
:10E660005FFA8CFC8CF311882268136A002BFCD1B2
:10E670009DF80F0015B030BD04AB0B625FFA8CFC47
:10E680008CF31188FCF7C0FBEEE700BF144BD3F806
:10E69000C037B0EB930F14D2B0EBD30F13D2B0EB63
:10E6A000131F12D2B0EB531F11D2B0EB931F10D235
:10E6B000B0EBD31F0FD2B0EB132F0ED24FF48070FC
:10E6C00070470220704704207047082070471020D0
:10E6D000704720207047402070478020704700BF5F
:10E6E000C81A002011F001020ED170B590F8281060
:10E6F000C568012982B0044607D0B5F1807F01D9F1
:10E700000123037702B070BD7047094B466A9868D1
:10E71000FFF7BCFFB5F1807FB080F3D9B725217733
:10E720000B46304601A98DF80450FFF717FEE9E7C4
:10E73000B83C00202DE9F0410546406A94B01446EB
:10E7400000681F460E465CF0A1FA0B94264C0C970D
:10E7500004F55F730093254B01930223002202937B
:10E760000123CDE90922CDE90E22CDE910228DF851
:10E770000C308DF834308DF8483006922B7F8DF8B0
:10E78000202013921A4A049204F55D7205921A1D14
:10E79000079223B3330E84F8753304F27634330CC6
:10E7A000DFF850802370330A6370A670D8F8080031
:10E7B0006A6AFFF76BFF6B7F90809BB169461046DA
:10E7C000FCF72AFC6C6A20685CF060FAD8F810004C
:10E7D000FFF75CFFA080384614B0BDE8F08104F27A
:10E7E0007534DCE705A9EAE788010020C43C002075
:10E7F000698E0008B83C0020013902292ED81B4A36
:10E80000282310B401FB03F302F561641C44134494
:10E810000460012480F8884093F8104E022C03F520
:10E82000616C1DD0C9B202EB0112D2F8982EC3F868
:10E83000142E8AB14FF48072022183F8101EACF8B6
:10E840000C2000F110024C30C3F8282EC3F82C0E17
:10E8500001205DF8044B70470020FAE70020704764
:10E8600093F81D2E013283F81D2EF1E7C81A0020FF
:10E870002DE9F0410C4D0646D5F8148000241835DA
:10E88000A04501DCBDE8F08104EB4407E85D0FF032
:10E89000DDF9864205D12146E819BDE8F041FCF7D3
:10E8A00098BA0134ECE700BFB83C00202DE9F041F4
:10E8B00091F80380B8F1000F03D100273846BDE876
:10E8C000F08100F110060C46054689783046FFF7C6
:10E8D00093FF07460028F0D040460FF0B7F9A86133
:10E8E000237801338046DBB210B1C37122238371D8
:10E8F00040460921FCF78EF84046FCF755FA104ACD
:10E900001368632BFCD90F48DFF84080FFF7BEFE89
:10E910000D4BA88202E058F8043F53B130469847A7
:10E9200003460028F7D0286985F8D8305BF008FC4A
:10E93000C4E7E0780FF08AF9FFF79AFFBDE700BF60
:10E94000C81A002040420F0081CF05084CE9060894
:10E9500037B590F85F38032B04462DD100231F4DA7
:10E960008DF807309DF8073094F860289A4201D856
:10E9700003B030BD9DF8073005EBC30393F84C306E
:10E9800083B181F001037BB19DF8073005EBC30330
:10E99000986CFCF709FA9DF807300133DBB28DF86B
:10E9A0000730DFE70B46EEE79DF8073005EBC303C2
:10E9B000986CFCF709FAEEE7D0E910039B7903F0B5
:10E9C0000103994204D003B0BDE83040FCF7ECB934
:10E9D00003B0BDE83040FCF7F7B900BFB83C0020F9
:10E9E00010B50446222100795BF006FF63792168A7
:10E9F00002229B0802FA03F3DB439BB20B8263798A
:10EA00008889D3409A40024392B28A8110BD10B5E2
:10EA10000446012100795BF0EFFE2068617983896B
:10EA2000890802229BB28A4023EA0203838110BD37
:10EA300038B510F8133CA0F664041BBB94F85038AA
:10EA40008BBBD4E909239A421CD05A1CA169A2624B
:10EA5000CB5C21695B0043F40073A4F854380A23AB
:10EA600084F85238012384F8503894F85F388A4289
:10EA700028BF0022012BA26201D0042B02D1606CBE
:10EA8000FFF7C5FF94F84C38002B6DD194F84D3842
:10EA90000133DBB2092B84F84D3825D12046BDE87F
:10EAA0003840FAF705B894F952586DB1B4F85418D3
:10EAB0004B08A4F8543801F001012046013DFFF74E
:10EAC00047FF84F85258DDE7D4E909239A4284F8D5
:10EAD0005058D7D194F85F38012B01D0042BD1D1F5
:10EAE000606CFFF77DFFCDE70A2B3DD194F84F38DE
:10EAF0002BB9B4F8563843F00103A4F856382379FB
:10EB0000D9070AD5B4F85608820501D4C30718D42A
:10EB1000B4F85C380133A4F85C38012284F84C283E
:10EB200094F84F280023012A84F84D381CD16179CC
:10EB300084F84F38606C01F00101BDE8384059F0AD
:10EB4000BBBAE36AC0F3470013B1216B9847E4E70F
:10EB5000E3696269D054E369E2680133B3FBF2F11F
:10EB600002FB1133E361D8E738BD2DE9F84310F813
:10EB7000133CA0F664047BB1B4F8583801339BB25F
:10EB8000082BA4F858381BD90021606C84F8511860
:10EB9000A4F8581859F090FA384F97F88880B8F1CF
:10EBA000000F03D101212046FFF7D2FE94F8503820
:10EBB00053BBD4E909239A4204D1002387F8883053
:10EBC000BDE8F883B8F1020F12D808F1010814BFAC
:10EBD000FF237F2387F88880A4F85438082384F81B
:10EBE0005238012384F85038606CBDE8F8430EE7D2
:10EBF0005A1CA169A262CB5C21698A4228BF00220B
:10EC0000DBB228BFA262E7E794F952685EB3B4F8BA
:10EC1000549897F8895019F001010BD0012D01D8B3
:10EC2000012103E0AB1E012B09D800212046FFF78C
:10EC30008FFE04E015F0FD03F2D0012BF6D0013574
:10EC4000EDB2032D87F88950BAD9013E4FEA590930
:10EC500076B20023A4F8549884F8526887F8893073
:10EC6000002EA6D0ACE7D4E909239A42A8D184F8B3
:10EC70005068606CBDE8F843B2E600BFB83C0020C5
:10EC80002DE9F84FC56E95F90020D3B2052B00F29F
:10EC90009F80C04B134493F98831002B00F098807B
:10ECA0003F24144114F00104074640F093800126EC
:10ECB0004FF0FF32A446B8484FEA420E00EB420242
:10ECC00092F98C10CAB2012A2AD8DFF8D49208220D
:10ECD000013B4FF00C0818FB0128DBB24A4609F54E
:10ECE000137B02E01C325A4515D092F800A0BAF10D
:10ECF000040FF7D192F801A09A45F3D152F808A079
:10ED0000BAF1000FEED0C7F840A001EB410A02EBC8
:10ED10008A02D268BA64704490F98D2001325ED1C3
:10ED20003A6C002A52D09D4BD3F83411914200F036
:10ED3000E380D3F858118A4200F00F81D3F87C1198
:10ED40008A4200F00E81D3F8A011914200F00D81AB
:10ED5000D3F8C4118A4200F0FC80D3F8E8118A424B
:10ED600000F00981D3F80C128A4200F00881D3F830
:10ED700030128A4200F00781D3F854128A4200F020
:10ED80000481D3F878128A4200F01281D3F89C12E1
:10ED90008A4200F01381D3F8C0128A4200F0128137
:10EDA000D3F8E4128A4200F00F81D3F808138A42A4
:10EDB00000F00E81D3F82C138A4200F00D81D3F8B5
:10EDC00050138A4208BF0F2000F09780F86B08BBF1
:10EDD000BDE8F88F541C0C264FF00B0C6BE7704A03
:10EDE00009F5137902E01C324A4599D010780528BC
:10EDF000F9D150789842F6D152F808000028F2D0A4
:10EE000001EB410102EB8102F863D3683A6C7B6449
:10EE1000002A88D1614BD3F83411884200F09B80DE
:10EE2000D3F85811884200F09A80D3F87C118842B8
:10EE300000F09980D3F8A011884200F09880D3F8B0
:10EE4000C411884200F08380D3F8E811884200F0B2
:10EE50009080D3F80C12884200F08F80D3F83012E3
:10EE6000884200F08E80D3F85412884200F08F80E0
:10EE7000D3F87812884200F09D80D3F89C12884223
:10EE800000F09A80D3F8C012884200F09980D3F83D
:10EE9000E412814200F09A80D3F80813884200F00F
:10EEA0009980D3F82C13884200F09880D3F850133F
:10EEB000884208BF0F228BD102EBC20203EB820310
:10EEC000E4B293F84C21002A82D183F84C6183F894
:10EED0004D413449D3F830316A688B4214BF4FF446
:10EEE00080034FF40013A1F520510432086B034353
:10EEF0000B63FA65BDE8F88F002000EBC00203EB5E
:10EF00008203013093F84C21E1B2002A7FF45EAF16
:10EF100083F84D1183F84CC1234AD3F8303121498D
:10EF20008B4214BF4FF480034FF40013116B0B435B
:10EF3000136395F823201D493B46FCF73FFD6B68A2
:10EF4000F86B0433BB6500283FF442AF62E704224C
:10EF5000B2E70420D1E70022AEE70120CDE701228D
:10EF6000AAE70220C9E70222A6E70320C5E7032299
:10EF7000A2E70522A0E70520BFE706229CE70620BE
:10EF8000BBE7072298E70720B7E70820B5E7082284
:10EF900092E700BFD4E70608B83C002088010020B3
:10EFA00034E50608006002400038024061AA00080B
:10EFB0000920A2E709227FE70A227DE70A209CE7D1
:10EFC0000B2279E70B2098E70C2096E70C2273E7D9
:10EFD0000D2092E70D226FE70E208EE70E226BE7E1
:10EFE00038B5484DD5F8E03AD5F8044B002B4AD057
:10EFF000A289238850069BB201D559061CD4D5F8A6
:10F00000E43A23B3A28A2388D0079BB204D5190718
:10F0100044BF4FF6F7732380A2892388D2069BB2A0
:10F0200009D5DB0607D5D5F8D83A13B19847D5F8F6
:10F03000044B2388A38838BD95F8213B002B34D09E
:10F040004FF6BF732380D5F8E43A002BDAD1A289BA
:10F05000238812069BB2D5D51B06D3D5D5F8CC3A5A
:10F06000D5F8C82A934233D0D5F8BC2AD5F8B41ABB
:10F07000D25C0133D2B2A280B3FBF1F201FB1233B6
:10F08000C5F8CC3ABEE7A289238892069BB2AFD5D9
:10F090009B06ADD5D5F8D03AFBB1A088D5F8D41AE7
:10F0A00080B29847D5F8044BA2E795F8150B0EF0FF
:10F0B000CDFDA38923F008031B041B0CA3810123AE
:10F0C00085F8213B0028BBD02021FBF77DFCB7E76A
:10F0D000E36823F08003E36094E7A388D5F8C02AAF
:10F0E000D5F8B81ADBB28B54D5F8C03AD5F8B02AA7
:10F0F000D5F8044B0133B3FBF2F102FB1133C5F831
:10F10000C03A75E70400001038B5484DD5F8603BAB
:10F11000D5F8844B002B4AD0A289238850069BB295
:10F1200001D559061CD4D5F8643B23B3A28A2388A1
:10F13000D0079BB204D5190744BF4FF6F77323805D
:10F14000A2892388D2069BB209D5DB0607D5D5F85C
:10F15000583B13B19847D5F8844B2388A38838BD12
:10F1600095F8A13B002B34D04FF6BF732380D5F820
:10F17000643B002BDAD1A289238812069BB2D5D535
:10F180001B06D3D5D5F84C3BD5F8482B934233D04A
:10F19000D5F83C2BD5F8341BD25C0133D2B2A28017
:10F1A000B3FBF1F201FB1233C5F84C3BBEE7A28979
:10F1B000238892069BB2AFD59B06ADD5D5F8503BC0
:10F1C000FBB1A088D5F8541B80B29847D5F8844B82
:10F1D000A2E795F8950B0EF039FDA38923F00803FB
:10F1E0001B041B0CA381012385F8A13B0028BBD085
:10F1F0002021FBF7E9FBB7E7E36823F08003E36036
:10F2000094E7A388D5F8402BD5F8381BDBB28B5494
:10F21000D5F8403BD5F8302BD5F8844B0133B3FB00
:10F22000F2F102FB1133C5F8403B75E70400001012
:10F2300038B5484DD5F8E03BD5F8044C002B4AD002
:10F24000A289238850069BB201D559061CD4D5F853
:10F25000E43B23B3A28A2388D0079BB204D51907C5
:10F2600044BF4FF6F7732380A2892388D2069BB24E
:10F2700009D5DB0607D5D5F8D83B13B19847D5F8A3
:10F28000044C2388A38838BD95F8213C002B34D04A
:10F290004FF6BF732380D5F8E43B002BDAD1A28967
:10F2A000238812069BB2D5D51B06D3D5D5F8CC3B07
:10F2B000D5F8C82B934233D0D5F8BC2BD5F8B41B66
:10F2C000D25C0133D2B2A280B3FBF1F201FB123364
:10F2D000C5F8CC3BBEE7A289238892069BB2AFD586
:10F2E0009B06ADD5D5F8D03BFBB1A088D5F8D41B93
:10F2F00080B29847D5F8044CA2E795F8150C0EF0AB
:10F30000A5FCA38923F008031B041B0CA381012384
:10F3100085F8213C0028BBD02021FBF755FBB7E73F
:10F32000E36823F08003E36094E7A388D5F8C02B5B
:10F33000D5F8B81BDBB28B54D5F8C03BD5F8B02B51
:10F34000D5F8044C0133B3FBF2F102FB1133C5F8DD
:10F35000C03B75E70400001038B5484DD5F8603C57
:10F36000D5F8844C002B4AD0A289238850069BB242
:10F3700001D559061CD4D5F8643C23B3A28A23884E
:10F38000D0079BB204D5190744BF4FF6F77323800B
:10F39000A2892388D2069BB209D5DB0607D5D5F80A
:10F3A000583C13B19847D5F8844C2388A38838BDBE
:10F3B00095F8A13C002B34D04FF6BF732380D5F8CD
:10F3C000643C002BDAD1A289238812069BB2D5D5E2
:10F3D0001B06D3D5D5F84C3CD5F8482C934233D0F6
:10F3E000D5F83C2CD5F8341CD25C0133D2B2A280C3
:10F3F000B3FBF1F201FB1233C5F84C3CBEE7A28926
:10F40000238892069BB2AFD59B06ADD5D5F8503C6C
:10F41000FBB1A088D5F8541C80B29847D5F8844C2D
:10F42000A2E795F8950C0EF011FCA38923F00803D0
:10F430001B041B0CA381012385F8A13C0028BBD031
:10F440002021FBF7C1FAB7E7E36823F08003E3600C
:10F4500094E7A388D5F8402CD5F8381CDBB28B5440
:10F46000D5F8403CD5F8302CD5F8844C0133B3FBAB
:10F47000F2F102FB1133C5F8403C75E704000010BF
:10F4800038B5484DD5F8E03CD5F8044D002B4AD0AE
:10F49000A289238850069BB201D559061CD4D5F801
:10F4A000E43C23B3A28A2388D0079BB204D5190772
:10F4B00044BF4FF6F7732380A2892388D2069BB2FC
:10F4C00009D5DB0607D5D5F8D83C13B19847D5F850
:10F4D000044D2388A38838BD95F8213D002B34D0F6
:10F4E0004FF6BF732380D5F8E43C002BDAD1A28914
:10F4F000238812069BB2D5D51B06D3D5D5F8CC3CB4
:10F50000D5F8C82C934233D0D5F8BC2CD5F8B41C10
:10F51000D25C0133D2B2A280B3FBF1F201FB123311
:10F52000C5F8CC3CBEE7A289238892069BB2AFD532
:10F530009B06ADD5D5F8D03CFBB1A088D5F8D41C3E
:10F5400080B29847D5F8044DA2E795F8150D0EF056
:10F550007DFBA38923F008031B041B0CA38101235B
:10F5600085F8213D0028BBD02021FBF72DFAB7E715
:10F57000E36823F08003E36094E7A388D5F8C02C08
:10F58000D5F8B81CDBB28B54D5F8C03CD5F8B02CFC
:10F59000D5F8044D0133B3FBF2F102FB1133C5F88A
:10F5A000C03C75E70400001038B5484DD5F8603D03
:10F5B000D5F8844D002B4AD0A289238850069BB2EF
:10F5C00001D559061CD4D5F8643D23B3A28A2388FB
:10F5D000D0079BB204D5190744BF4FF6F7732380B9
:10F5E000A2892388D2069BB209D5DB0607D5D5F8B8
:10F5F000583D13B19847D5F8844D2388A38838BD6A
:10F6000095F8A13D002B34D04FF6BF732380D5F879
:10F61000643D002BDAD1A289238812069BB2D5D58E
:10F620001B06D3D5D5F84C3DD5F8482D934233D0A1
:10F63000D5F83C2DD5F8341DD25C0133D2B2A2806E
:10F64000B3FBF1F201FB1233C5F84C3DBEE7A289D2
:10F65000238892069BB2AFD59B06ADD5D5F8503D19
:10F66000FBB1A088D5F8541D80B29847D5F8844DD9
:10F67000A2E795F8950D0EF0E9FAA38923F00803A7
:10F680001B041B0CA381012385F8A13D0028BBD0DE
:10F690002021FBF799F9B7E7E36823F08003E360E3
:10F6A00094E7A388D5F8402DD5F8381DDBB28B54EC
:10F6B000D5F8403DD5F8302DD5F8844D0133B3FB56
:10F6C000F2F102FB1133C5F8403D75E7040000106C
:10F6D0001648174A174938B5174C184D121A5DF0DD
:10F6E00069FDD4F88820164B164842F47002C4F81D
:10F6F00088201A68002142F001021A6099601A6895
:10F7000022F0847222F480321A6058601A6822F45F
:10F7100080221A600C4AD960521B28460B495DF0C2
:10F7200049FDA560BDE83840F9F74ABB000000106C
:10F73000040000104F26080800ED00E00000002043
:10F74000003802401030002488010020000000082A
:10F750000548D0F8D03723B1DB6A13B100F5FA6061
:10F7600018470248704700BFC81A002064E906081D
:10F7700038B5174CD4F898301B8843B9154D002381
:10F7800084F8A73085F8C837C5F8C43738BDD4F831
:10F790009C20002AF2DDD4F8A010012A488806D067
:10F7A00001230C4DA4F8A40084F8A630E7E78A886A
:10F7B0000132121A9A42F3D1064DD5F8D037002201
:10F7C0001B69C5F8FC2705F5FA609847D7E700BF25
:10F7D000B83C0020C81A00200748D0F8CC371BB12D
:10F7E000064B93F8A6300BB100207047D0F8D03705
:10F7F00000F5FA605B681847C81A0020B83C002082
:10F8000030B4174A174B92F8C8C703F1A80505EBA7
:10F810000C04C0E9004593F8A73092F8C80783426A
:10F8200092F8C80714D8834206D300231A46184614
:10F8300030BCC1E90032704792F8C8071A1EC0F107
:10F84000800330BC0CBF01200220C1E900327047A8
:10F850001B1A0022012030BCC1E90032704700BFF2
:10F86000C81A0020B83C00200E4B0F4A93F8C81766
:10F8700092F8A70093F8C827904293F8C8270CD8AD
:10F88000904238BF93F8C827D3F8C4373ABFC2F1C3
:10F8900080028018002018447047D3F8C437801ABB
:10F8A00018447047C81A0020B83C002070B51E4CA0
:10F8B0001E4D94F8C83794F8C81784B005F1A80213
:10F8C0001344029395F8A73003928B4220D894F802
:10F8D000C827934214D294F8C8171E46C1F180017C
:10F8E000F3B98C460122CDE9001610B9BCF13F0FE7
:10F8F00006D90023694602A85AF02CFF95F8A730D4
:10F9000094F8C807C01AB0FA80F0400904B070BD7E
:10F9100094F8C8C7A3EB0C0C614600260122E2E76D
:10F9200001EB030C0222DEE7C81A0020B83C0020DD
:10F930002DE9F043164685B0002936D0441E254DEA
:10F94000254F04EB01084FF0000901E0A0452CD041
:10F9500095F8A70014F8013F411C2844C9B280F86B
:10F96000A8300B0648BF002097F8C83785F8A710C5
:10F970004ABF0146084685F8A790994297F8C837CC
:10F9800036BFC3F18003C01AC0183F28DED997F8EC
:10F99000C8379942DAD0114B93F83230002BD5D0CA
:10F9A0000020FFF783FFA045D2D1694602A8FFF7E8
:10F9B00027FF20B1DDE9003213443F2B02D805B008
:10F9C000BDE8F0830246334602A85AF0C3FE05B0F4
:10F9D000BDE8F083B83C0020C81A00208801002050
:10F9E00030B585B0694602A8FFF70AFF58B9094C3F
:10F9F00004F5FA65D4F8D03728465B6898470028A4
:10FA0000F8D005B030BD0246012302A85AF0A2FE8C
:10FA1000EDE700BFC81A002070B5134D134C00234A
:10FA2000C5F8CC3758F024FBC4F8A000FFF790FECF
:10FA3000D4F8A030C4F89800A3B19A885B88D21A91
:10FA4000436802FB0333C5F8CC37F9F741FA95F860
:10FA5000C83794F8A7209A42064601D0FFF7C0FFA6
:10FA6000C5F8C46770BD00BFC81A0020B83C0020AC
:10FA70002DE9F041104ED6F8CC37154682189A423F
:10FA80000E4A88BF1D1A92F8A72096F8C8379A42E6
:10FA900004460F4601D0FFF7A3FFD6F8D027084849
:10FAA0000023C6F8FC372B46956A21463A46AC46F9
:10FAB000BDE8F041604700BFC81A0020B83C0020F4
:10FAC000982200208C461346014662461846CFE72E
:10FAD0002DE9F04F41F62C728BB00021C4485DF047
:10FAE000C1FB042053F0CCFE0446052053F0C8FEB1
:10FAF00050EA040340F02A81BE4B0393039BBE49A6
:10FB0000BB48D3F8B043E4225DF054FBB84BC3E9E3
:10FB10000744C3E91A445C621C67C3F8B4401F463B
:10FB2000C3F8B840C3F8BC4059F080FBFFF774FF3E
:10FB3000002108460EF0DEF8F9F7CAF9B0F1000826
:10FB400040F3A481AD4DDFF8DCC2AD4ECDF808C066
:10FB5000002407F1E40901942746A24605F5947BA9
:10FB600004E00AF5006AD04540F3AF80029A1368BA
:10FB7000C2F81438F9F7E0F9202259465046FFF749
:10FB800077FFA049122258465DF0A9FB0028E8D172
:10FB9000BA4525D001999C4B01EB410203EB82034E
:10FBA00001934A1C184699490592AAEB070304934E
:10FBB00001F05AFE4946019B41F84C3B049B059AD3
:10FBC000C9F80C70C9E90433D9F81C300192C9E9AD
:10FBD00008338F4BC9F828300123C9F8083089460B
:10FBE000039BD3F8B033C9F81C3057461222A9182A
:10FBF000335D91F82811994202F101020BD00024E3
:10FC0000202AF4D12037B8455946384653DBFFF750
:10FC10002FFF0022EBE70134152CF1D1D0197D49DB
:10FC20002022FFF725FF00230A2209A97948CDF8F1
:10FC300024B001F08DFF07460998002301300A2205
:10FC400009A9099001F084FF079009980023013069
:10FC50000A2209A9099001F07BFF06900998002368
:10FC600001300A2209A9099001F072FF0590099854
:10FC700009A9013000230A22099001F069FF0490CC
:10FC80000998002301300A22194601F061FF97B15B
:10FC9000DDE9063243EA4212049B05995B0143EA1F
:10FCA000C123A7F2BC7143EA600342EA412243EA5E
:10FCB0000243C9F81C30019B642B00F0B580574605
:10FCC0000AF5006AD0453FF751AF019B642B00F065
:10FCD000AB80BA451DD0019B4B4C4C490C2202FB1A
:10FCE000034401331A462046019301F0BDFDD9F8C3
:10FCF0001C20C9F80040AAEB0705C9E90822C9E998
:10FD00000375434AC9F828200122C9F81450C9F8DC
:10FD10000820019B002B03F1030100F388804FEAC8
:10FD20004803B3F1805FC0F2B280314B986830B9BC
:10FD30001A461B791BB11368002B40F0DE800021AE
:10FD400008460BB0BDE8F04F0DF0D4BF4FF47A7207
:10FD5000002321465BF096FC2F4BA3FB00231B0CDA
:10FD600040F2B27240F26D1401E05B1A013212F0FF
:10FD7000030514BF21464FF4B7718B42F5DA1D49D4
:10FD8000002D00F0B48003910399D1F880138B42C9
:10FD9000C0F25781214D01245B1A55F8041F994286
:10FDA00004F10104F8DD013343EA4413A2F2BC720A
:10FDB00043EA42231A4A039DB0FBF2F102FB11020F
:10FDC0004FF461603C24B2FBF0F100FB11221C20D7
:10FDD000C5F88403B2FBF4F004FB1022521042EA8F
:10FDE000401242EAC12242EA0343C5F8B03385E635
:10FDF000A87200208801002078E90608B83C00209D
:10FE00003C6A0708186A0708003E00202C6A0708A9
:10FE1000C5FA0008E03D002007452EC20805002075
:10FE200080510100C81A00206423019367214C26E9
:10FE30008548DFF82892854F06FB01F40519324604
:10FE4000002128465DF00EFA3246002128465DF07A
:10FE500009FA7D487E4E40F8049004F110034FF0FB
:10FE6000010AC5F808A02F62AE6240F8038003447F
:10FE7000021DC3F804801834039B0199D3F8B033F2
:10FE80001351A018043143606B6248E703216E4BA5
:10FE9000DFF8CC914C2606FB01F41D1932460021F7
:10FEA00028465DF0DFF93246002128465DF0DAF998
:10FEB000654B664E43F80490039A2E62654ED2F865
:10FEC000B00304F1100104F118020127341FC8F136
:10FED0000063BB404FF0020A85F805A0AF60635095
:10FEE00021444B60B0503244506068621DE70C46BC
:10FEF00003911D21C4F8841346E7534900220023CF
:10FF0000C1E9102388640A46C86305460146D46CDB
:10FF100002F14C03B4B19C689D644E1EB442C2E928
:10FF20002355DD6300F086804E1CB44274D113F873
:10FF3000481C00293FF403AF1A6443F8083C2146EB
:10FF40001A46E4E7404A0226254615E0D36B1663BD
:10FF50005B0118BF03F6FF73C2E9045514BF01EB40
:10FF60001333334653631946916352F84C7FCB1ACF
:10FF70001C444E1C0130CFB11379711E002BE5D10A
:10FF8000136916635BB103F6FF73576901EB133313
:10FF900053634FB107F6FF7701EB1731E4E7576979
:10FFA00033465363002FF5D13146DDE7DFF8B4C0A7
:10FFB000294BCCF8584801390CF50362CCF83C3891
:10FFC0003E2440233F25CCF86408CCF84838C2E9E9
:10FFD0000445CCF85418880F8B00D9B140F2FF14B7
:10FFE0001B1940F100005B0A43EAC0531648C2E9FE
:10FFF0000B0003F14000034403EBC101CCF850387F
:020000040801F1
:10000000CB0D53604B02CCF84C08CCF83818CCF828
:10001000303894E60123E9E78C427FF490AE002962
:100020003FF48DAE146CE66B0136E6631C6493649A
:100030001A466CE700293FF482AE53F80C2C214697
:10004000EDE70124AFE600BFA87200200068214C54
:10005000C5FA0008AC720020706A0708546A0708E5
:10006000646A0708C81A002010B50A4CD4F8D037C3
:100070005B6A13B104F5FA609847074AD4F8C437AD
:10008000D2F898205288013B134452421340C4F8DE
:10009000C43710BDC81A0020B83C00202DE9F04735
:1000A000DFF82881474E92B0FFF762FB98F8C83717
:1000B00096F8A7209A4201D0FFF792FCD8F8CC9787
:1000C0000025C8F8C457B9F1000F29D03E4F6C463F
:1000D0000AE098F8C83796F8A7209A4201D0FFF7AF
:1000E0007FFC2035A9451BD92A463946204601F018
:1000F000BBFB20465AF002FE012201462046FFF7D4
:1001000017FCABB2002BE4D1D8F81C38002BE0D0A0
:100110001A689B8851690B4214BF53831383D8E735
:10012000D6F898309B7B012B45D098F8C83796F8C5
:10013000A7209A4201D0FFF753FC0027C8F8C477E4
:10014000B9F1000F3AD0DFF880A03D466C4602E0DE
:100150002035A94529D92A46514609A801F084FB32
:100160002122002120465DF07DF8202221462846EC
:10017000FFF77EFC2022064609A920465DF0AFF875
:1001800008B9202E00D00137ABB2002BE0D1D8F84F
:100190001C38002BDCD01A689B88516920350B4233
:1001A00014BF53831383A945D5D8B7FA87F0400904
:1001B00012B0BDE8F087FFF757FFB6E7012012B095
:1001C000BDE8F087B83C0020786A0708C81A00200C
:1001D000032108B50546084653F042FB72B60F4AA4
:1001E00052E9023153EA01020AD1002421460420D7
:1001F00053F036FB2146052053F032FBFCF786FC1A
:10020000074804684EF6602202FB05F0E41841F14D
:100210000001041941EBE071E9E700BFB84200209A
:10022000C81A00204FF6FF7200234FF0030C43F270
:100230000111028243F2013280F808C08374018008
:100240008280C0F80A30C381704700BF0F4B4FF661
:10025000FF7200B5A0F803200281A0F80D2003F181
:10026000120E13F9012CB3F800C002EB8202063320
:1002700020F802C0811813F8042C8A7033F8032C7C
:10028000A1F803209E45ECD15DF804FBC9FD0608EA
:10029000014BC0F8053070470001020300234FF402
:1002A000007203808370A0F80320704740F21F3370
:1002B0000380704742F601410222002301808270D0
:1002C000C3707047114B1249124A10B4C361124BEC
:1002D000C0F811304FF4F07C104B114CA0F800C066
:1002E00001624FF00E0C826040F206710222C0F8EB
:1002F00015300723C46080F824C05DF8044BA0F8D3
:100300001910A0F805208370704700BF2602D0079F
:10031000E803A80738391819020000010203040590
:100320001A242021084B09498B4202460AD218465A
:1003300002E01C30884205D20388C3F30B039A42C3
:10034000F7D170470020704790010808300B08086B
:1003500070B58588C5F30B059542A8BF15462A469A
:100360000C46064680685CF025FF62199442B56928
:10037000064B08D0064814F8011B00FB03F3A24209
:1003800083EA0103F7D12B60012070BDC59D1C815C
:1003900093010001014B0360704700BF2829FFFF54
:1003A00043F232524FF0013302604360704700BFA6
:1003B00000230360704700BF00230360704700BF45
:1003C000002306214FF47A72C0E901230170037300
:1003D000704700BF00230372704700BF0023037003
:1003E000704700BF40F23922A0F8032040F21912F2
:1003F000A0F809204FF492724FF40E7C4FF48C71E8
:10040000A0F80F2040F22122A0F800C0C1804FF4D4
:100410008D7C4FF40871A0F815204FF494720023DE
:10042000A0F80CC0418240F2231C40F22921A0F820
:100430001B20FF22837043710372C3728373437462
:100440000375C375A0F818C083764377C18380F81D
:100450002020704703230370704700BF0023036010
:1004600003717047704700BFD0ED007AD0ED016A8C
:1004700030EE677AE6EE877AB0EE670AC0ED007A72
:10048000704700BFD0ED017AD0ED026A30EE677A96
:1004900090ED000AE6EE877A37EEC07AC0ED017A79
:1004A000A6EE870A80ED000A704700BF90ED017A42
:1004B000D0ED036AD0ED027A30EE470AA6EE807ADC
:1004C00090ED000A80ED017A37EE676AE6EE867AF3
:1004D00037EEC07AC0ED027AA6EE870A80ED000AF8
:1004E000704700BFD0ED056AD0ED017A90ED066A45
:1004F000D0ED025A90ED035AC0ED066AB0EE407A94
:1005000026EEA70AD0ED007A80ED057AA7EE870ADD
:10051000D0ED077AA5EE860A90ED086AD0ED045A70
:10052000C0ED087AA5EE670AA5EEC60A80ED070AB7
:10053000704700BFF0EE406AD0ED007A90ED050AFA
:1005400090ED067A90ED016AD0ED035AA7EEA60A67
:10055000A6EE267AD0ED047A90ED026A67EEC07AB4
:10056000A5EEC07AE6EE267A80ED057AC0ED067A31
:10057000704700BF2DE9F047DDF820A055460F4633
:1005800015F8011B002B064614460CBF4FF020093E
:100590004FF0300939B3002A2BDD2B4600E09CB127
:1005A00013F8012BA046013C002AF8D1A8F102085B
:1005B00054B1444649463046B847013CFAD29AF80D
:1005C000001008F1010459B13046B8472B4615F820
:1005D000011B0029F8D1A4EB0A041819BDE8F08723
:1005E0002046BDE8F087002A02F1FF38E1DC08462A
:1005F000F4E70024E8E700BF03685A1C02601970A2
:10060000704700BF024B186803681B68184700BF9B
:1006100070A8002010B500F100440246013C04E03F
:10062000B3EB0E0015D1A24214D012F8013BA3F196
:100630004100192811F8010BA0F1410C98BF20339B
:10064000BCF1190F00F1200EEAD91B1A04D10028C1
:10065000E9D110BD002010BD184610BD884210B56C
:100660004FF001043ED301FB04F4B0FBF4FC8C45D5
:10067000F9D2CCB122BB08E0A14203F801EBB4FBF4
:10068000F1F211D8B0FBF2FC1446BCF1090F0CF1E9
:10069000570E0CF1300204FB1C00EDDCA14203F804
:1006A000012BB4FBF1F2EDD900221A7010BDA1426A
:1006B00003F801EBB4FBF1F2F6D8B0FBF2FC144600
:1006C000BCF1090F0CF1370E0CF1300204FB1C00D9
:1006D000EDDCA14203F8012BB4FBF1F2EDD90022CD
:1006E0001A7010BD8446002AEAD1CEE7002870B502
:1006F00003DA2D2301F8013B4042092886464FF0DA
:10070000010307DD03EB83035B00B0FBF3F2092A6F
:10071000F8D8E3B10F4CA4FB0320BEFBF3F2092A87
:1007200002F1570602F130054FEAD00007DD092B30
:1007300001F8016B03FB12EE09D90346EBE7092B25
:1007400001F8015B03FB12EE01D90346E3E7002346
:100750000B7070BDCDCCCCCC0378202B024600F1C1
:100760000100F9D0092BF7D02D2B28D02B2B03BF5C
:100770005378B7EE000A0246B7EE000AA3F1300143
:10078000C8B209289FED567A10D8F2EE046A07EE37
:10079000901AF8EEE77A12F8013FE7EE267AA3F115
:1007A0003001C8B20928B0EE677AF0D92E2B5ED09E
:1007B00003F0DF03452B07D020EE070A704753787C
:1007C000BFEE000A0246D9E710B451782D2978D03F
:1007D0002B296AD0A1F13003092B02F101026BD859
:1007E0000024002303EB830301EB430312F8011FF2
:1007F000A1F130000928A3F13003F3D9B3F59A7FB2
:100800001A4628BF4FF49A72072B66D9DFED356A76
:100810001346F7EE007A083B072B67EEA67AFAD864
:1008200002F00702DAB1F2EE046A012A67EEA67A54
:1008300015D0022A67EEA67A11D0032A67EEA67AAF
:100840000DD0042A67EEA67A09D0052A67EEA67AAB
:1008500005D067EEA67A062A18BF67EEA67A6CB3B3
:1008600087EE277A5DF8044B20EE070A704753782D
:10087000A3F13001C8B2092802F1010298D8F2EEC2
:10088000046AF0EE665A07EE901AF8EEE77A12F86C
:10089000013F87EEA66AA3F13001C8B2092866EECF
:1008A000A56A37EE067AEED982E79178A1F1300396
:1008B000092B02F1020293D9F7EE007A27EE277A8C
:1008C000D0E79178A1F13003092B02F1020288BF31
:1008D000F7EE007AC4D8012483E7F7EE007AA1E7A7
:1008E0000000000020BCBE4CF0B5067906F0E00325
:1008F000402B03D145794FF0FF3406E0602B4FF0D9
:100900000105F8D1447905FA04F40023012006F02A
:100910000706AB4200D1F0BD052E0FD8DFE806F088
:100920000308101D242448B1C85CD75C78400FE050
:1009300020B1C856D756C71B784278410133E8E743
:100940000028FBD031F8130032F81370784080B2E1
:1009500020420CBF01200020F0E70028EED031F942
:10096000130032F91370E6E70028E7D051F82300AE
:1009700052F82370DAE7037903F01803102B1AD02A
:1009800003D833B9B0F80B007047182BFAD0002009
:100990007047104BB0F80B0093F90030591C06BF9C
:1009A0000D4B1B78DBB2C3EBC302C3EBC20300EBFE
:1009B000830080B27047074BB0F80B0093F9013009
:1009C0005A1C06BF044B5B78DBB2C3EB031300EB8E
:1009D0004300EEE7B8050020B842002070B5054698
:1009E000B0F80900FFF79EFC054B1E790446284627
:1009F000FFF7C1FF16B1E368184470BDA368FBE7B9
:100A000070A8002038B505460C46FFF7E7FF2A79A5
:100A100002F0070302F0E002602A29D1052B0CD86E
:100A2000DFE803F0030B0F0B1B1B6A7901239340D4
:100A3000DBB2027814B11343037038BD22EA03031A
:100A4000FAE76A79012393409BB2028814B11343F9
:100A50000380F2E722EA0303FAE76B7901229A4066
:100A6000036814B113430360E7E723EA0203FAE7DC
:100A7000052BE2D8DFE803F0030305050707047040
:100A8000DBE70480D9E70460D7E7032870B516D800
:100A90000B4BC60003EBC000C943057B427B01F052
:100AA000010181EA0504A24209D082682AB1908836
:100AB0001268A94214BF1083508333445C7370BD25
:100AC00070A8002010B514490446052220305CF0BF
:100AD00018FC1249152204F125005CF012FC104BA1
:100AE00093F82820012184F83A101AB9964684F820
:100AF0003BE010BD03F12C0C8E46BCE80F002060DB
:100B00006160A260E360BCE80F0084F83BE0206114
:100B10006161A261E36110BDFC6A0708006B070810
:100B200070A800200E4B002200B50260828003F105
:100B3000120E13F9012CB3F800C002EB4202063387
:100B400020F812C000EB420113F804CC33F8032C58
:100B50008A80734581F802C0EBD15DF804FB00BFC9
:100B6000DDFD0608092900D001B9704701394A00A6
:100B700002F00802930001F00301A3EB9203C1EB22
:100B80000111C3EB0313C1EB011100229B0089008B
:100B9000026081804380704784B04FF46173ADF888
:100BA00004300199ADF80C10BDF80C1081814FF4A0
:100BB000007C41F201420023A0F800C042804FF4C3
:100BC0000D7C01220093A0F806C08360837302822B
:100BD00004B0704710B53822002104465CF042FB97
:100BE0000D490E4A0E482061C4E905120D480E4910
:100BF000E06101234FF0090C40F20112C4F8261005
:100C000084F808C0A37384F8213062852146074820
:100C1000BDE8104032F0E0B81A046C070019750303
:100C20006400DC0543080E001E1E1E7D0C6B0708C9
:100C300070B50B4C4FF0FF33054603604360836093
:100C400004F10F0614F9010C11F092FC05289CBF69
:100C5000238825F810300334A642F3D170BD00BFBD
:100C6000F1FD0608B5EEC00ADFED347AF1EE10FAB8
:100C7000CCBF30EE270A30EE670ADFED317A20EE86
:100C8000270A30B5FDEEC07A87B017EE904A0546C8
:100C900084EAE470002303A9A0EBE470CDE90033FB
:100CA000029354F0B7F8002CB4BF2D23202303A8DF
:100CB0008DF800305AF022F8012829D0022833D0CC
:100CC00003281DD003A968465CF0D4FA68465AF0A0
:100CD00015F8C41EE4B22246694628465CF06AFA5A
:100CE00000232B5528465AF009F82E232B540130A7
:100CF0000DEB040128445CF0EAFA284607B030BD49
:100D0000302303A968468DF801305CF0B3FADDE7C3
:100D100043F23002302303A96846ADF801208DF874
:100D200003305CF0A7FAD1E743F2300303A9684629
:100D3000ADF801305CF09EFAC8E700BF6F12033ACD
:100D400000007A440CF002BD38B5054658B14C1E7F
:100D500014F8011F284619B9BDE838400CF00ABD47
:100D60000CF0F4FCF4E738BD08B520215CF091FAF2
:100D70000346184623B10278202A03F10103F8D074
:100D800008BD08B5CB0701D4FBF708FF08BD2DE966
:100D9000F341134D134F002305F84C3F044600EB7D
:100DA0008106B44203D1104802B0BDE8F081394653
:100DB00028465CF05FFA214668465CF088FA4FF0FE
:100DC0000008202168465CF064FA28B96946284684
:100DD0005CF050FA0434E4E780F80080F1E700BFEB
:100DE00070A80020D5ED0708BCA800202DE9FF471A
:100DF0001E46C368BDF83070DDF83480044689466D
:100E000092463BB30D29DABF194B5D560025BAF166
:100E1000FF3F21D0CDE9005A164A236831463846B3
:100E2000C047524620795FFA89F1FAF75FFC024623
:100E300000B10288D3B20393C2F30323120BCDE9AE
:100E40000052029323680C4A31463846C04704B02A
:100E5000BDE8F0874D1CDAE77B06F8D40C952368D3
:100E6000064A31463846C44604B0BDE8F0476047FC
:100E7000EC6A07083DDD07084ADD07086EDD070854
:100E80002DE9F043154685B06A1C8946BDF83060EF
:100E90000D9F194625D04FEA101800F00F0408F1F5
:100EA0004008CDE90045164A43463046B847A8B148
:100EB00099F80510D9F800002A46FAF759FC68B1EC
:100EC000038802780392C3F303221B0BCDE900438E
:100ED000029243460B4A00213046B84705B0BDE8B0
:100EE000F0837306FAD40309074A00F00F000C9050
:100EF00040333046BC4605B0BDE8F043604700BF14
:100F00007DDD07088FDD0708B8DD07082DE9F04310
:100F100087B00709DDF8388091461E46403700F05B
:100F20000F0439B30DF080FBC379174ACDE90043B4
:100F300005463B4649463046C047C0B12868FAF7E7
:100F400027FFAA796B79114912F0020F4FEA930338
:100F50000F4A18BF0A46E97900940133CDE903210D
:100F6000CDE901030B4A3B4600213046C04707B09C
:100F7000BDE8F083084A0E943B4649463046C446D5
:100F800007B0BDE8F0436047CCDD07082CDF070859
:100F90005DEA0708DEDD070800DE070870B5858812
:100FA0000B460446C5F30B052A46002118465CF0A3
:100FB00059F90A4A61699142034606D3084A9142A7
:100FC00006D3BDE87040184608470029F9D170BD26
:100FD0002A46BDE870405CF0EDB800BF300B080851
:100FE0000F0D080838B5064C064DAC4206D2A16874
:100FF00020461C34FFF7D2FFAC42F8D338BD00BF07
:1010000090010808300B080800B501EB020E71458D
:1010100016D001390EF1FF3E41F2210C11F8013FCB
:10102000082280EA032003B2002B4FEA4000B6BF3B
:101030008CEA430380B298B2013AF4D18E45EDD1E7
:101040005DF804FB4840082341B240000029C0B2CB
:10105000B8BF5040013BF7D1704700BF30B50568BD
:101060008D42044618D901F1FF3E681E00231EF888
:1010700001CF082183EA0C034FFA83FC5B00BCF12B
:10108000000FDBB2B8BF53400139F5D17045EED146
:101090006A1C22602B7030BD00236A1C22602B70FA
:1010A00030BD00BF07EE901AB8EE677ADFED867AA2
:1010B00027EE000A60EE277ABDEEE77A17EE103AC7
:1010C0002033402B00F2FB809FED807AB4EEC70AFC
:1010D000F1EE10FA40F3A180DFED7D5A9FED7D6ABD
:1010E000B0EE677AF0EE476AF4EEC66AF1EE10FAF7
:1010F00037EE657AF6DCDFED786AB4EEE67AF1EE8B
:1011000010FA00F3A980DFED756AB4EEE67AF1EE2D
:1011100010FA44BFDFED726A36EEC77A27EE075A3F
:10112000DFED705A9FED706ADFED706ADFED704A97
:10113000A5EE256A27EE054AE5EE066AF7EE005AA7
:10114000A4EE267AF0EE656AE7EE646AE7EE245ACA
:1011500086EEA54A9FED607A77EE877ABDEEE77A54
:1011600017EE103A2033402B00F2A2809FED617AF7
:10117000B4EEC70AF1EE10FA73DD9FED556ADFEDAC
:10118000556AB0EE677AB4EEE67AF1EE10FA77EED1
:10119000C67AF6DC9FED507AF4EEC77AF1EE10FADB
:1011A0007ADD9FED557A77EE677A67EEA74A9FED75
:1011B0004D7A9FED4D5ADFED4D6AA4EE875A67EEEA
:1011C000A43AE4EE856AB7EE006AE3EEA67AB6EEDC
:1011D000007A36EE676AB8EE005A67EE857A26EE38
:1011E000077AB7EE005AC5EE256A00238361436192
:1011F0000362C36180ED044A26EE877A26EE866A92
:1012000066EEA76A80ED095A80ED007A80ED016AEA
:1012100080ED027AC0ED036A70479FED387AB4EE34
:10122000C70AF1EE10FAB0EE677A7FF564AFDFED32
:10123000285A9FED336AF0EE476AF4EEC66AF1EE83
:1012400010FA37EE257AF6D4DFED236AB4EEE67AAB
:10125000F1EE10FA7FF757AFDFED276A36EEC77A67
:101260005CE79FED287AB4EEC70AF1EE10FA91D54B
:101270009FED176ADFED226AB0EE677AB4EEE67A88
:10128000F1EE10FA77EE867AF6D49FED137AF4EE4B
:10129000C77AF1EE10FA84DC9FED107AF4EEC77A8B
:1012A000F1EE10FA44BF9FED0E7A77EE677A7CE795
:1012B000DFED157AB6EE007AB7EE006A91E7B7EE89
:1012C000004AF0EE445A45E727D4D2360024F448C9
:1012D000DB0FC940E4CB1641DB0FC93FDB0FC9BFB1
:1012E000DB0F49C092E741B99730083C15A82ABEE8
:1012F000F304353F00247448DB0F49400024F4C850
:10130000E4CB16C1001B37C900000000FDEEC07A17
:1013100017EE903A2033402B50D8DFED2A7AB4EE06
:10132000E70AF1EE10FA2FDDDFED276A9FED277A4D
:10133000F0EE407AF4EEC77AF1EE10FA30EE660A7B
:10134000F6DCDFED237AB4EEE70AF1EE10FA30DCDA
:10135000DFED207AB4EEE70AF1EE10FA44BFDFEDDC
:101360001E7A37EEC00A60EE006A9FED1C6A9FEDA0
:101370001C7ADFED1C7AA6EE867A20EE266AE6EE6F
:10138000877AA6EE270A7047DFED137AB4EEE70AF4
:10139000F1EE10FAD5D5DFED0C6A9FED137AF0EE81
:1013A000407AF4EEC77AF1EE10FA30EE260AF6D45F
:1013B000C7E7DFED047A37EEC00AD4E79FED0B0AEA
:1013C000704700BFDB0F4940DB0FC940E4CB16413B
:1013D000DB0FC93FDB0FC9BFDB0F49C092E741B943
:1013E0009730083C15A82ABEE4CB16C100000000C7
:1013F0009FED327A70EE077AFDEEE76A16EE903ACC
:101400002033402B56D8B4EEC70AF1EE10FA31DD86
:101410009FED2B6ADFED2B6AB0EE677AB4EEE67AC9
:10142000F1EE10FA77EEC67AF6DC9FED247AF4EE50
:10143000C77AF1EE10FA38DC9FED237AF4EEC77A22
:10144000F1EE10FA44BF9FED217A77EE677A27EE2E
:10145000A76ADFED1F5ADFED1F6A9FED1F7AE6EEE8
:10146000256A67EE865AA6EE267AE5EE877AB0EE12
:10147000670A70479FED197AB4EEC70AF1EE10FAC9
:10148000D3D59FED0F6ADFED166AB0EE677AB4EE42
:10149000E67AF1EE10FA77EE867AF6D49FED077AC7
:1014A000F4EEC77AF1EE10FAC6DD9FED0E7A77EE14
:1014B000677ACCE79FED0C0A704700BFDB0FC93F8E
:1014C000DB0FC940E4CB1641DB0FC9BFDB0F49C0BE
:1014D00092E741B99730083C15A82ABEE4CB96C0E4
:1014E000E4CB16C1DB0F494000000000B0EEC07A2B
:1014F000F0EEE06AF4EEC76AF1EE10FAB4BFF0EE77
:10150000475AF0EE665AF5EE405AF1EE10FAF0EE58
:10151000407A44D0F4EEC76AF1EE10FA8CBFB0EE18
:10152000475AB0EE665A85EE256A9FED1E2A9FED5A
:101530001E3A9FED1E4ADFED1E4ADFED1E2ADFED4B
:101540001E3A9FED1E5AA6EE423AE6EE223AA6EE6B
:10155000034AF7EE005AE6EE044AE6EE235AA6EEF8
:10156000245A85EE250AF4EEC76AF1EE10FA48BF58
:101570009FED137AF5EEC00A48BF37EE400AF1EE50
:1015800010FA48BF9FED0F7AF5EEC07A48BF37EEEC
:10159000400AF1EE10FA48BFB1EE400A70479FEDE5
:1015A000070AE0E739094E3DE3B59E3E88FA163E4C
:1015B00045FE7F3F99FB243F69A2163EA7DFA83472
:1015C000DB0FC93FDB0F49402DE9F04F144689B0CE
:1015D0008846217801320392002900F01681002507
:1015E00007461E46A94609E03846C047039C013518
:1015F0002178631C0393002900F08F802529F3D103
:101600006078A31C3028CDE9033923D0A0F1300342
:10161000DBB2092B4FF0000A26D96C282AD0782893
:101620007FD8572878D9A0F15803202B79D8DFE844
:1016300003F0BD7878787878787878787882AF78A1
:101640007878787878787878AA787878789E788AB0
:101650007878BD00A078E31C0393A0F13003DBB2DF
:10166000092B4FF0010AD8D804AA03A956F0DAFCD6
:101670006C28D4D1039C22780134782A0394B7D8FB
:10168000572A40F28E80A2F15803202BB0D801A136
:1016900051F823F0CB170108F1150108F1150108E5
:1016A000F1150108F1150108F1150108F1150108FE
:1016B000F1150108F1150108F1150108F1150108EE
:1016C00039170108E7170108F1150108F11501089C
:1016D000F1150108F1150108F1150108F1150108CE
:1016E000F1150108F1150108F11501088917010824
:1016F000F1150108F1150108F1150108F1150108AE
:1017000071170108F1150108F7170108F115010813
:10171000F1150108CB17010828B9284609B0BDE822
:10172000F08F039C64E72528FBD1039C25213846D4
:10173000C04701355CE7039C56F8041B3846C9B224
:10174000C047013554E70DF1140B56F8040B039C08
:101750005B4600220A21FEF781FF049ACDF800B013
:10176000534641463846FEF705FF054440E7039CD3
:1017700056F8043B0093049A002341463846FEF78E
:10178000F9FE054434E7039C56F8043B1D602FE73F
:101790000DF1140B56F8040B039C5946FEF7A6FFF7
:1017A000DBE7002AB9D0252AC0D021E7A0F15802F2
:1017B000B2FA82F20DF1140B56F8040B52095B4693
:1017C0001021FEF74BFF039CC7E7A2F158020DF171
:1017D000140BB2FA82F256F8040B52095B46102140
:1017E000FEF73CFFB9E70DF1140B56F8040B594610
:1017F000FEF77CFFB1E70DF1140B56F8040B5B46C6
:1018000000220A21FEF72AFFA7E70D4685E7F8B573
:10181000104C0746206F0D461646A0B10E49FFF743
:1018200093FA206F3946FFF78FFA0C49206FFFF7C4
:101830008BFA0B49206F33462A46FFF7C5FE09494C
:10184000206FFFF781FA94F8743013B1012384F804
:101850007530F8BD70A8002012DE0708D1F6070821
:10186000450D01081FDE07080EB400B584B005ABB6
:10187000019053F8042B0649039301A8FFF7A4FE37
:10188000019B00221A7004B05DF804EB03B07047AE
:10189000F90501082DE9F043002483B006460480D1
:1018A00021463046013440F0CBF8082CF8D1002313
:1018B000DFF8608086F8EA30C6F8EC30C6F8F03021
:1018C000C6F8F430C6F8F8309946FC361F464A464A
:1018D000414601A8FFF7C8FF3446032301A802E0F0
:1018E00004F8011B5BB110F8011B1D46013B0029E8
:1018F000F6D120462A4620215BF0B4FC2C4409F1A5
:101900000109B9F1080F277006F10406DFD103B011
:10191000BDE8F083186B0708F7B5114E074630464F
:10192000002300F8763F0C460E4B0F49002F18BFDE
:10193000194615465BF09EFC0C4F04EB45057636C8
:10194000AC4202D10A4803B0F0BD394634F8022B4C
:101950006846FFF789FF694630465BF08BFCEFE78E
:1019600070A8002023DE07082CDE070835DE0708F4
:10197000E6A80020F7B50C4E0C4F002306F8A73F51
:10198000044600EB4105AC4202D1094803B0F0BD6A
:10199000394634F8022B6846FFF766FF6946304641
:1019A0005BF068FCEFE700BF70A80020CDFF0708E0
:1019B00017A90020F8B5084F4E1E054601F11F0477
:1019C00016F8012F28463946FFF74EFFA64205F1CB
:1019D0000205F5D1F8BD00BF3ADE07080246531CE8
:1019E000084605D1034B1A681B790A600B717047D2
:1019F000014939E778DD0708CEFF070810B5013146
:101A000014460CF011FE28B9054B1A681B792260A8
:101A1000237110BDC27903492046BDE8104023E779
:101A200078DD0708D9DD070803685A1C02601970C1
:101A30000368090A5A1C02601970704710B40268E2
:101A40001346511C016013F8021B0360D31C547829
:101A5000036093781B0443EA0423141D0460D078C8
:101A60005DF8044B0B4343EA00607047A0F130037C
:101A7000092B07D920F02000413819288CBF0020FD
:101A80000120704701207047303809288CBF0020A2
:101A900001207047413819288CBF00200120704771
:101AA000613819288CBF002001207047202805D0FC
:101AB000093804288CBF002001207047012070479E
:101AC000A0F14103192B98BF20307047A0F16103AA
:101AD000192B98BF2038704702B310B5844684187C
:101AE00003E0981A15D1A44514D01CF8013BA3F1CA
:101AF0004100192811F8010BA0F1410E98BF2033C5
:101B0000BEF1190F00F12002EBD91B1A04D10028F5
:101B1000E9D110BD002010BD184610BD1046704719
:101B200070B5044608460D4659F0E8F8064602E04E
:101B300014F8013F43B1324629462046FFF7CCFF57
:101B40000028F5D1204670BD1C46204670BD00BF60
:101B50002DE9F043064686469EF800C0BCF1200FF2
:101B60007446ACF109050EF1010EF5D0042DF3D940
:101B7000BCF12B0F64D0BCF12D0F26D10127102A08
:101B800094F801C004F1010423D04FF0FF35B5FBF8
:101B9000F2F502FB05FE6FEA0E0E5FFA8EFE90462E
:101BA000002014F801CBBCF1390F4CF02009ACF146
:101BB000300C29D85FFA8CFC944528DAA8422646D6
:101BC0001ED81BD000FB08C0EBE7102A4FF000071F
:101BD000DBD1BCF1300F0AD16078A0F14105192D9D
:101BE00098BF2030661C78280CBF023434466FF052
:101BF00070454FF00F0E4FF01008D1E7F445E1D9D2
:101C00004FF0FF301F40CCE7B9F1600F0AD801B1A7
:101C10000E6067B923B16FF00043984228BF1846A1
:101C2000BDE8F083A9F157095FFA89FCC4E723B145
:101C3000B0F1004F28BF4FF000404042BDE8F083B4
:101C400000279CE773B50E4610490546FEF7E2FCF7
:101C500018B93070012002B070BD2C78602C8CBF98
:101C6000613C413C072C0FD8013501230A2201A910
:101C70002846FFF76DFF019BAB4205D00F2803D824
:101C8000013440EA0410E4E70020E4E778DD0708C7
:101C900001230A2200215BE770B50D461446FFF7C9
:101CA00063F80646A0B1FFF7F3FF40F6340398420D
:101CB000A8BF1846B0F5617FB8BF4FF46170A0F5BA
:101CC00061731922B3FBF2F32B7023780133237075
:101CD0003046FFF749F80646A0B1FFF7D9FF40F6B6
:101CE00034039842A8BF1846B0F5617FB8BF4FF4DF
:101CF0006170A0F561731922B3FBF2F36B70237866
:101D000001332370304670BDF8B516461F460446B1
:101D1000394630464FF47A72002359F0B3FC3C4DFB
:101D20003C4B054483FB05602844E917C1EB601177
:101D300083FB01030B44384EC817C0EB631086FBCE
:101D4000003CC317354EC3EBAC0386FB03764FEA6A
:101D5000E37ECEEBE61EC1EB0116A5EB860CC0EBD5
:101D60000015A1EB8501617103EB4301A0EBC100FC
:101D700040F2B55101FB1E33B3F5896F84F806C0FC
:101D800020714FEA8E0636DA40F2DA218B4238DCD7
:101D9000B3F5B77FB4BF4FF0000E4FF0010E2049EE
:101DA0000EEB4E0001EBC0017546B1F84E004FEA54
:101DB0004E071C4907EB0E0C01EBCC0C0CF1160C7A
:101DC0000B2101E03CF8020D984211DD0139F9D1F7
:101DD0001349774401EBC701088F0121013306F550
:101DE000FA6E1B1A7544A170E37022812580F8BD3C
:101DF0000131C9B2F2E7032540F29650AE460627FC
:101E0000D7E7022540F22940AE460427D1E700BFBC
:101E100080BC92C789888888ABAAAA2A73B06D163D
:101E2000C8FD060800FE06080C4B10B5D3E90043B8
:101E300054EA030209D1014640F201130020C1F81F
:101E4000023088710880088110BD054A1268121995
:101E500043F10003FFF758FF012010BDB0420020FE
:101E6000C81A00202DE9F041044694421546084660
:101E700009D2B4FBF2F6154B05FB16441B5D00F8C6
:101E8000013BBDE8F081B4FBF2F69642B6FBF2F7F7
:101E90000CD20E4B05FB176705FB1644DA5D00F804
:101EA000012B1B5D00F8013BBDE8F081BA42B7FB96
:101EB000F2F807D9054B05FB187813F8082000F84D
:101EC000012BE7E74046FFF7CDFFF3E7206B07085C
:101ED000844B30B59A8819899889DC89B2F57A7F64
:101EE00088BF4FF47A7283B088BF9A80DA88B2F5DF
:101EF0007A7F84BF4FF47A72DA805A89B1F57A7F9B
:101F000084BF4FF47A711981B2F57A7F84BF0022C1
:101F10005A81B0F57A7F52D94FF47A708442988111
:101F20005FD891429CBF00221A81A0429CBF002230
:101F30009A819A8B598B6C4C914284BF00225A83B0
:101F40006A4B1B880BB36179694D0129AA784ED978
:101F5000062A5BD92979002940F09D809FED657A9A
:101F600065490A7807EE903A06EE902AF8EEE77A8D
:101F7000B8EEE66AAB79C6EE276A002B40F08280A5
:101F8000B4EEE67AF1EE10FA4EDC6378032B24D837
:101F90005A49C3EB031301EB43012278584B032A40
:101FA000C3F8B81411D8C2EBC201C2EBC10203F5E9
:101FB000A47303EB8203534A136003B030BDB4F53E
:101FC0007A7F84BF0024DC81ABE7002222704D4A77
:101FD00003F5A473136003B030BD00234749637059
:101FE000DBE700209142D881A3D81881A1E7A97925
:101FF0000029ADD0072A62D0B3F57A6FA8D93E493F
:1020000008780228B8BF02200870A1E73E4901EB1A
:10201000820191ED267A29790029A1D0531F032B43
:10202000B3D9002AB1D03CE027EE277AFCEEC77A7C
:10203000CDED017A9DF8043007EE903AF8EEE77A9C
:10204000B4EEE77AF1EE10FAC4BF0133DBB2A3B30A
:10205000102BA8BF1023DBB2934238BF13460B707E
:1020600093E72A79002A90D123499FED287A0A78AC
:1020700007EE903A06EE902AF8EEE77AB8EEE66AB6
:10208000C6EE276A37EE077AB4EEE67AF1EE10FA7A
:102090007FF77BAFC8E7053A032A7FF676AF9FED5F
:1020A000157AB7EE000A80EE070A5AF04BFC2B882F
:1020B000834228BF03462B8067E70123CBE7062234
:1020C000B3F57A6FAA70CCD90B490A78022AB8BF47
:1020D00002220A702A79002A7FF457AF9FED0B7A0B
:1020E0003FE700BF3C450020B84200202C0F001005
:1020F000AC2800206F120338E844002040A90020DB
:1021000070A80020F0440020C8FD060817B7D13899
:102110002DE9F04FAA4B83B01B78A3F11702022AD6
:1021200000AF13D9A74A12F83310002940F0B1824A
:10213000DB001A4452784AB1A34A3A60134493F838
:10214000B4302BB99E4A1823137001E09E4B3B60BC
:102150009E4B9F4E93F808809E4B4FF0000A03F170
:1021600054059B461FE09BF90430142B00F00883B4
:1021700020465BF00BF9A20323D5012800F0008371
:10218000082800F3FD82B9F1000F01D0344206D1D6
:102190004146204657F0ACFD002800F0F1820BF1DB
:1021A0000C0B5D4513D0DBF8004014F00109DAD0C8
:1021B00020465BF0EBF80AF1010AA2035FFA8AFA03
:1021C000DBD40128DCDC0BF10C0B5D45EBD10AF113
:1021D000FF33022B00F2D4827F4DDFF818920023E8
:1021E000022085F8143510F00BF995F81835D9F858
:1021F0000040022B00F0CD82002800F02C83DFF895
:10220000F8A1764B95F871C5C7F804C003F55C7B5F
:102210004FF47A784FF0000E6422264633F8081CFB
:10222000B1F57A7FB3F8461088BF23F8088CB1F572
:102230007A7F33F8061C88BFA3F84680B1F57A7F11
:1022400033F8041C88BF23F8068C33F8060CB1F56C
:102250007A7F84BF002123F804EC8842B3F85A0047
:10226000B3F85C1098BF23F806EC884293F86B1023
:1022700088BFA3F85AE00139632993F86C1088BF2E
:1022800083F86B200131C9B2092988BF83F86CE05B
:1022900003F16500002113F8314010F801CF01313E
:1022A000A44538BF80F800E00329F4D179680129FA
:1022B00018BF83F886E0DC339B45AFD13446484EE7
:1022C000B378042B00F0A18233B93388B3F5F07FE3
:1022D00084BF4FF4F0733380FFF7FAFD414895F85F
:1022E0008415FEF73FFC95F8A3151030FEF73AFC75
:1022F00095F8B3151030FEF735FCB5F8C215B5F8F2
:10230000C0350B43B5F8C4150B431BB213B1012301
:10231000A5F8C635344B2340002B00F0A982E30713
:1023200000F16E82600400F1BF81210740F12C8230
:102330002E49DAF800300C400B40C9F80040CAF8CA
:102340000030230440F1B681204A0023D373D377B1
:10235000E00440F1BA8195F8D335DFF89480022B80
:1023600004BF012385F8D33508F17804434602E021
:1023700006339C420CD01A78082AF9D19978DA7879
:10238000914202D35A79002AF2D0082023F04EF964
:1023900000234FF4806085F8143510F031F80028E0
:1023A00000F046821249C7F804A08B468A469AF884
:1023B000050078B39AF8001049B3434621E000BF06
:1023C0007443002034EC0608C8FD0608D042002003
:1023D000BC0202002CAD002070A80020C2A9002081
:1023E000AC28002004AE002009600002FE9FFFFD23
:1023F00048AE0020B4490020CC42002006339C4265
:1024000008D01A788242F9D15A79002AF6D00846C3
:1024100023F00CF90AF1060A5445C8D196F8028057
:10242000D7F804A0B8F1080F594600F0C28195F81A
:102430007105AE4BDAF800C0A0F10100B0FA80F0EF
:10244000400985F8500695F87205A0F10100B0FA30
:1024500080F0400985F854065878032884BF00208E
:102460005870A34BA3489A7BD9F80030CCF3C03EF8
:1024700003400CEA000085F852E6C9F80030CAF8BB
:102480000000002A00F0B381B5F86836002B40F058
:10249000A281994A1368B3F1807F24BF002313609F
:1024A000936823F4007323F0020313B140F2022374
:1024B00093601379013B042B84BF01231371A8F1AE
:1024C00005088E4BB8F1030F93F800B040F232814B
:1024D0004FF00008BBF1000F25D0DFF850927C6070
:1024E0005C46CB46894606E0AAF1060AAAEB060A34
:1024F000544540F2DB80DA461BF8010F0028F3D088
:102500000CF0BAF80028EFD082799307ECD57C68FC
:1025100049460122B8F1000F05D0737C3BB97379AD
:10252000012B00D01AB1B3790BB10023B371744BF6
:10253000DA8812F00C0F03D1C2F30312022A02D977
:102540004FF42062DA801A8912F00C0F03D1C2F323
:102550000312022A02D940F601221A8195F86D066B
:1025600095F8792695F86C36904205D9002285F8C1
:102570006D2653B1A5F8702695F878269A4204D2B4
:10258000002385F86C36A5F8703695F8623795F813
:102590006E265C4ED7F800A09A4284BF002385F8CF
:1025A0006E3606F178093346002013F8022F02EB4D
:1025B0004202524492F88C8192F88DE192F88EC1D9
:1025C00013F8012F4245A8BF42461A709A79724506
:1025D000A8BF72469A71DA7801306245A8BF624698
:1025E0000328DA70ECD11E364E45DCD1464B1A6B0F
:1025F000002A00F0E880002601200B78292B07D163
:102600004B78043300FA03F313421CBF9A430126AC
:1026100006318C42F1D10EB13B4B1A633B4C6E46F6
:1026200004F10808234602E0434500F0948013F8C3
:10263000012F072AF8D9002304F8013F0133082BA2
:10264000FAD1B5F86A25B5F868359A42B54602D38D
:102650002F4BC5F868352F4B2F4CFF2285F8942758
:1026600003F1540013F9082C142A05D053F80C1C5C
:1026700034EA010100F0C6800C339842F2D1274BB6
:102680005A79022A01D100225A710C37BD46BDE8A1
:10269000F08F02EBC301DB00496800297FF449ADEC
:1026A0001F481721017044E51E4942E67C684946EF
:1026B00000222FE7144BDB7B002B00F0C680124A70
:1026C0000023E004D3773FF546AE21067FF543AE05
:1026D000134B1978182904D8134BCB40DA073FF570
:1026E0003AAEDFF84C8008F1780451E63C45002012
:1026F000B8420020BCD67718F8440020A80D00107E
:102700009048002040A90020D0420020BE28002090
:10271000AE014A0138AD0020010002003C28002033
:1027200074430020F6DFFFFD00410001B3280020C4
:1027300048AE0020002333714FF00108BBF1000FB9
:102740007FF4CBAE737C002B7FF4F1AE7379012B59
:102750007FF4EDAEE7E688B0E9462022FF21484647
:102760005AF080FD474A04E0424549F823303FF4DF
:1027700068AF12F8013F59F823100131F4D05AE73D
:1027800041480FF00BFB27E5A2047FF5DAAD3F4986
:10279000CFE500283FF433AD90F904604FF0FF0817
:1027A00001E080F8088030460FF01AFE0028F8D1CA
:1027B00025E5B379002B3FF43AAE737C012B04BFBF
:1027C0000223737433E62920796022F02FFF304B07
:1027D00079681A6B0FE795F8640679600BF04CFF87
:1027E000796800287FF455AEA5F8680651E643F4F1
:1027F000A02340F4A020C9F80030CAF8000043E646
:10280000244996E585F8942739E7DAF8003023F46F
:102810008053CAF80030338C24F48054B3F57A7FA7
:10282000C9F80040BFF458AD4FF47A73338453E5D0
:10283000D9F8003023F00063C9F80030DAF800302E
:1028400023F00063CAF80030ACE542F201031C42F9
:102850007FF435AF7CE5DFF840A0DAF8003024F0F3
:10286000800423F08003C9F80040CAF80030C8E4AF
:10287000DAF8003043F0080344F00804CAF80030E6
:1028800056E500BFBE2800202CAD0020F6BFFFFD9E
:10289000D0420020F79FFFFDCC4200202DE9F04FF1
:1028A000834B93F89837013B012B83B040F2E780CC
:1028B000DFF828827F4ED8F80C30DFF8249203F23C
:1028C000DC534E45C8F80C3080F0EE8001230193B4
:1028D000794BDFF810B206F11C059F1C764B598826
:1028E000002900F0B7807A185A4580F0B3803C4642
:1028F00008E0118814460A44002900F0AB805A45CC
:1029000080F0A880052940F2A58035F81C3C61883C
:10291000C3F30B039942ECD163799B07E9D1238878
:1029200055F8141C94F804A000933046FEF736FBCB
:1029300035F81C1CBAEB113F00F092800023019384
:1029400035F8181C55F8140C55F8044CC1F30B015C
:1029500054F0F2FB1C364E45206005F11C05BDD33A
:10296000564A574B574E12681A60FFF7D1FB33781F
:10297000554C564D7278C3EBC301C3EBC10304EB56
:102980008303C2EB02122B60A4F1780303EB420332
:10299000C4F870331DF0F2F928684D4D4FF0FF3345
:1029A0006B602EF023FB22F089FE04F5926304F5A0
:1029B000A16102E0063399425CD01A78002AF9D16D
:1029C0009C78D878844202D358790028F2D0384CC9
:1029D0002A7294F8D035B4F8D42503EB830303EBC3
:1029E00083039B00642BB8BF6423C8F804306423BE
:1029F00003FB02F2642AB8BF64220023C8E9022361
:102A0000C8F82020334AA8F82430C8E90433C8E9BC
:102A1000063388F8263004F5B863936232F0B2FBCF
:102A200094F8BE17B4F8BC0725F0DCF840F05EF867
:102A300017F05EFD94F89837013B012B2CD9264AFC
:102A400001981268C8F80C20012388F8253003B0DB
:102A5000BDE8F08F55F8141C3046FEF79FFA6DE77D
:102A6000009BA11D9A1F3046FDF772FC00287FF4E1
:102A700067AF63E7F27B003A18BF0122A7E7F7F7D9
:102A8000E9F80B4B00F5B71000F558700222C3F8B7
:102A9000B40783F8B8270BE7F7F7DCF80223C4F88C
:102AA000B40784F8B837CAE70123019358E700BF99
:102AB00070A800209001080800400008B4490020D8
:102AC000CC420020B8420020B8A90020F0440020E9
:102AD000B8050020BC140010C81A002004450020CE
:102AE000300B08080080000801211B4A10B503289C
:102AF00000EB010403461170E4B218D9FF2828D076
:102B0000164A002341F2024100E034B10233402B67
:102B100022F8021B04F1FF34F7D1114A1344FF21BC
:102B200083F8C017BDE810400E200FF0A3BDC3EB23
:102B3000C3020C480C49C3EBC20200EB82000B4AF3
:102B40000B7010602EF052FA2BF0BAFB2BF094FCB5
:102B5000D6E70023E1E700BFF014001030B00020FA
:102B600070A80020B8A90020B8420020F04400203E
:102B7000044A05491368012043F4001381F8010851
:102B800013607047E444002070A800207047F8B537
:102B9000164D6B78BE2B26D1022229464FF6FF70C8
:102BA000FEF732FA124FAC1C22884AB1A618BE4278
:102BB00019D2052A17D92146FEF726FA3446F3E73B
:102BC00021460222FEF720FA0222A118FEF71CFA83
:102BD0000634084B641BA3F8024841F60F53C31A8E
:102BE00058425841F8BD0020FCE700BF00400008F3
:102BF0000080000870A800202DE9F0410768C7F3A5
:102C00000D04064688460CB3D8F8005050F0D4FDA9
:102C1000092840F08880454C236923F440732361E0
:102C2000236943F400732361236943F001032361A3
:102C30003D6050F0C1FD2369092823F001032361A1
:102C400071D1336804333360002034E0384B394AA3
:102C500093422AD302F58042934225D302F5804263
:102C600093422AD3344A934229D902F580329342BF
:102C700027D902F50032934225D902F5003293425A
:102C800023D902F50032934221D902F50032934252
:102C90001FD902F5802293421DD9B3F1016F1CD3D5
:102CA0000520F7F75FFDFBE7082450F085FD0928B4
:102CB00015D04FF0FF30BDE8F0811024F5E718245F
:102CC000F3E72024F1E72824EFE73024EDE7382468
:102CD000EBE74024E9E74824E7E75824E5E7134D0C
:102CE0002B6923F440732B612B6943F400732B6130
:102CF0002B6923F0F8032B612B691C4344F0020479
:102D00002C612B6943F480332B6150F055FD2B6906
:102D100023F002032B612B69092823F0F8032B61B0
:102D20003FF472AFC5E76FF00100C4E7003C02401A
:102D30000040000800400008FFFF00082DE9F041B6
:102D4000584E3378B12B8AB071D1FFF720FF80F055
:102D50000104E4B2544B554DB3F89B31544FADF8D8
:102D6000003004F00104BD4263D3002C00F09780D2
:102D70001022002106A85AF075FA4E4B04969B1BB0
:102D800005934D4B1A69002A04DA4C4A5A6002F145
:102D900088325A6001228DF82420F322DA606946D5
:102DA000022204A84FF00008CDF8208057F06EFAF8
:102DB000022269464FF6FF70FEF726F93B4D0446A6
:102DC000BD4244D3022201A904A80025ADF8045055
:102DD00057F05CFA022201A92046FEF715F940BA25
:102DE000C043ADF80800022204A802A957F04EFA29
:102DF000079868B106ABC0F10402294618445AF09E
:102E000031FA089818B906A904A8FFF7F5FE08904A
:102E10009DF8243023B1284A136943F0004313611D
:102E20000898B0FA80F040090AB0BDE8F0810124AA
:102E300090E7A988AB69A868D3F80080C1F30B01BB
:102E400054F07AF91C35804518BF01248BE7AE8811
:102E50008DF80D80C6F30B06B31DADF808302B8836
:102E6000C3F30B02ADF80A201B0B062202A904A82B
:102E70008DF80C3057F00AFA062202A92046FEF718
:102E8000C3F8A9680446324604A857F0FFF9A968B8
:102E900020463246FEF7B8F81C35044690E701207C
:102EA000C2E700BF00400008C8FD060890010808FE
:102EB000300B080800800008003C024023016745F1
:102EC000F8B5264DFFF724F995F89837013B012B0B
:102ED0002FD9234E234FF36803F2DC530324F3600E
:102EE000FFF72CFF58B13B78B12B08D1FFF74FFE0D
:102EF000013C1BD040B9FFF721FF0028F3D1013C72
:102F0000EED10520F7F72EFC95F89837013B00220B
:102F1000012B85F8042818D9134B0122196886F86B
:102F200025200023F16085F80538F8BD0028EBD195
:102F3000E7E7F6F78FFE00F5B71000F558700223AB
:102F4000C5F8B40785F8B837C3E7F6F783FE022360
:102F5000C5F8B40785F8B837DEE700BF70A80020D1
:102F60000445002000400008C81A002008B50B499D
:102F70000B4A01230B709373FFF7A2FFFFF78EFC40
:102F8000084B41F20241FF22A3F8C01783F8C22781
:102F9000BDE808400E200FF06DBB00BFF01400101C
:102FA000B842002070A8002090F89230DFED6B6AE4
:102FB0006B4A07EE903A90F8963005EE103A90F88A
:102FC000943004EE903A90F8953005EE903A90F8EF
:102FD0009830F8EEE77AB8EEC55A04EE103A67EE8C
:102FE000A67A25EE265AF8EEE44AF8EEE55AB8EE4F
:102FF000C44A25EE275A64EEA64A65EEA65A24EE88
:10300000264AF0B5B7EE007A90F8917064EE854AE2
:1030100065EEA75A24EE274A00F16F06014602F139
:103020001A050024B0EE476AB0EE473A137807EE6F
:10303000903AF8EEE77A67EE857A67EE867AFDEEEB
:10304000E77A17EE903AFA2BA8BFFA2323EAE37344
:103050000B72537807EE903AF8EEE77A67EEA47AAF
:1030600067EE867AFDEEE77A17EE903AFA2BA8BF64
:10307000FA2323EAE3734B72937803EE903AF8EE67
:10308000E33A63EEA57A67EE877AFDEEE77A17EE0C
:10309000903AFA2BA8BFFA2323EAE3738B72938842
:1030A00007EE903AF8EEE77A67EE847A67EE867A72
:1030B000FDEEE77A17EE903AB3F57A7FA8BF4FF4AA
:1030C0007A7323EAE3738B812B68D5ED007A002BAA
:1030D000F8EEE77A3FDD90F8973002EE903AF8EE9E
:1030E000E22AB0EE436AA2EEE66A63EE863A83EE27
:1030F000A76AA2EEA66A013465EEA77A67EE877A20
:1031000067EE867AFDEEE77A17EE903AFA2BA8BFC3
:10311000FA2323EAE373BC4206F8013F00DDF0BD69
:10312000012C13D190F8933007EE103A90F89B30B1
:1031300006EE103AB8EEC77AB8EEC66A27EE267ADF
:1031400026EE266A0435083208316FE7B7EE007ABA
:10315000B0EE476AF6E7B7EE006ACCE70AD7233C41
:1031600066FF060890F899306BB3B0F864308BB105
:1031700090F89A2002EB82036421C3EB0313B3FBA4
:10318000F1F3A0F86430962312FB03F3B3FBF1F3E1
:10319000A0F8663043884BB190F89A3003EB830374
:1031A000C3EB03136422B3FBF2F34380B0F8503057
:1031B0004BB190F89A30962213FB02F36422B3FBD2
:1031C000F2F3A0F85030704790F821304BB3438BA6
:1031D00083B190F82230FA2213FB02F203EB83034F
:1031E000B3F57A7FA8BF4FF47A7364218383B2FB6F
:1031F000F1F24283838843B190F82230FA2213FB24
:1032000002F36422B3FBF2F38380C3884BB190F8DE
:10321000223003EB8303B3F57A7FA8BF4FF47A73B0
:10322000C380704770B50A4C0A4E002594F891305F
:1032300013B12046FFF7B8FE2046FFF793FF013594
:103240003046FFF7C1FF042D04F1DC04EED170BD60
:10325000B8A900203C45002010B5064C4FF4807200
:10326000002104F6060059F0FDFF0023C4F80839D8
:1032700010BD00BF70A80020034BD3F80C0908B1A3
:103280000AF078BA704700BF70A8002008B50B4656
:1032900005490246D1F80C0928B10449FEF794F912
:1032A000BDE80840E8E708BD70A80020450D01080A
:1032B000024B0146D3F80C09FDF746BD70A800206B
:1032C0000048F5E75BEA07080CB4C30607B500D56C
:1032D00061B9049805A90191FFF7D8FFFFF7F0FF46
:1032E000012003B05DF804EB02B070470020F8E75E
:1032F00008B5FFF7DDFFBDE80840E1E710B504467B
:103300000348FFF7D5FF2046BDE81040F0E700BFB7
:103310003FDE070810B508460749FDF77BF900288E
:1033200015BF0124002405480548FFF7E7FF2046A4
:10333000BDE8104009F058BC44DE07084DDE070820
:1033400074DE0708034B0146D3F80C0908B10AF0F4
:10335000FDB9704770A800200CB407B510F020002C
:103360000BD079B92320FFF7EDFF049805A901914F
:10337000FFF78CFFFFF7A4FF012003B05DF804EB1B
:1033800002B070470020F8E70FB407B504A951F860
:10339000040B0191FFF77AFF03B05DF804EB04B072
:1033A0007047F8B5154B1B6833B31548154FFFF739
:1033B0009FFFFFF761FFFCF7DBF90025FCF70CFA34
:1033C000044640B113200FF055F9FFF779FFBDE82F
:1033D000F8400D488CE73846FFF7D6FF792D05F108
:1033E000010602D1FFF76CFF2646FFF745FF642078
:1033F000F7F738F83546E1E7F8BD00BF9422002022
:1034000090DE070826F90708AADE070838B50B4B37
:1034100003EBC0050C4695F83823094803EB8203FB
:10342000D3F8C411FFF7B0FF95F83E332BB1611C00
:103430000448BDE83840C9B2A6E738BDC8FD060853
:103440008EF60708CDFF07080FB407B504A951F899
:10345000040B0191FFF71AFFFFF732FF03B05DF88D
:1034600004EB04B070472DE9F041037903F0E0026A
:10347000402A4AD009D82ABB03F00703052B1CD8E1
:10348000DFE803F0161B161B090F602A44D0802AC0
:103490003ED0BDE8F081D0F805102148BDE8F041EC
:1034A000D2E7D0F8052051421E48BDE8F041CBE7F5
:1034B000B0F80720B0F80510F6E7B0F90720B0F92A
:1034C0000510F1E74679184D184805EBC605FFF7DA
:1034D000EFFE95F8947400240123A74202D8BDE8BA
:1034E000F041EDE6D5F8906456F824204FEA8408C0
:1034F0004AB113B90E48FFF7DBFE56F808100D4825
:10350000FFF742FF00230134E7E741790A48C5E7A6
:10351000827941790948C8E7BDE8F041084893E756
:10352000B0DE0708C6DE0708C8FD0608DDDE0708AE
:103530004BE207088EF60708EEDE0708FFDE0708F5
:1035400016DF07082DE9F04385B0FCF701F90269A1
:1035500083890188029282680192428800924268BF
:103560001B4EDFF88080DFF880901A4F04461A481F
:10357000FFF76AFF002515B91848FFF7B9FED8F81C
:1035800000309D4213DA3378052B96BF09EB830395
:103590000022D3F85826B38800937388294638460A
:1035A0000135FFF751FF062D06F10606E3D154F071
:1035B0005FFD4288838864689B1A03FB0444FCF720
:1035C00053F902460648214605B0BDE8F0433BE703
:1035D00080B1002098DF07082EDF07088CDF07087E
:1035E000A7DF0708543D0020C8FD0608024903482C
:1035F00001F521610EC927E70070FF1FC4DF07082E
:1036000010B57521044632F099F801460948FFF7D4
:103610001BFF1A21204632F091F801460648FFF7B9
:1036200013FF1B21204632F089F8BDE81040014607
:10363000024809E7D8DF0708EBDF0708FEDF0708C5
:1036400038B50B4DE87810F0FD0405D10948FFF7B7
:10365000FBFE2046FFF7D4FFEB78013B012B06D899
:103660000548FFF7F1FEBDE838400120C8E738BD46
:103670003C45002011E007081CE007082DE9F04F49
:10368000764B77491A687748774BB2FBF3F297B0DD
:10369000FFF77AFE754BDFF84CC2DFF84C82DCF89E
:1036A0000870DFF810920FCB0AAD85E80F003907DC
:1036B00048BFDCF804406E4B05934FEA970E6D4B04
:1036C000069348BFC4F3805416AB1EF0020F18BF18
:1036D00003EB8404C7F3810603EB860618BF54F896
:1036E000442C654C08BF654A56F8301C6448654E4A
:1036F000654FFFF749FEB4F834294FF47A73B2FBF3
:10370000F3F103FB11220A20B4F9363992B2B2FB6D
:10371000F0F25E48FFF798FE5D4A5E495E48FFF7AB
:1037200033FEFFF7CDFD5D4B5D4A997B5D4B5E48F7
:1037300006EB8101D31AD1F88016B4F80228FFF7FE
:1037400083FE5A48FFF7B4FD94F838195848FFF73C
:103750001BFE5848FFF7ACFD94F839195648FFF79F
:1037600013FEFFF7ADFD5548FFF7A2FD00210A4605
:10377000FB7F0B4113F0010F01F1010508D012B1DD
:103780004846FFF795FD29464046FFF7FDFD01221B
:10379000072D2946ECD14A4D95F86A1505F13C03F1
:1037A00005F5EC72012908BF134693F8DC30032BB2
:1037B00002D04448FFF7E8FD434A95F86A1502F540
:1037C000CE73012918BF134693F8DC30012B02D1C8
:1037D0003E48FFF7D9FD3C4A95F86A1502F5CE73CD
:1037E000012918BF13461B695B7B012B02D938489E
:1037F000FFF7CAFD374FDFF8F4A0DFF8F4B0FFF7AA
:103800005FFDD4F83C89002507F1200957F8041B17
:1038100000296FD00123AB4013EA080F1BD0DA0652
:1038200019D01AF8052059F8253053F8222035B15F
:103830002948CDE90212FFF73BFDDDE902125846A7
:10384000FFF7A2FD012D06D1244B93F8211011B1F1
:103850002348FFF799FD0135D8E700BF88220020F3
:103860002FE0070834E0070840420F00380407083B
:1038700047E007084CE0070870A800205DEA070849
:1038800051E00708C8FD06083C45002059E007083C
:10389000F0FF0010000800007AE00708B84200209E
:1038A00000800008004000089EE00708CDE00708FF
:1038B000DFE00708E7E00708E9E00708F1E00708AC
:1038C0002C0F00100AE10708680F001012E107082A
:1038D00017E10708500407084BE20708F01400102E
:1038E00025E107080038024001E10708C40500206F
:1038F0001FE10708FFF7E4FC784B79481A68794B19
:103900001978137A527A06EB8101D1F8BC16FFF7C9
:103910009BFD754B754819684FF47A73B1FBF3F151
:10392000FFF732FD07A8FEF77FFA38B107A90EA806
:1039300056F030FE6E480EA9FFF726FDFFF7C0FCDB
:10394000D4F8C829002A00F0858007EE902ADFED20
:10395000696AB8EEE77AC6EE877AFDEEE77A17EE87
:10396000903A654D95F8C80030B1D5ED337AFCEE4C
:10397000E77A17EE901A88B2D4F848795FB107EE6B
:10398000907ADFED5C6AF8EEE77A86EEA77AFDEED4
:10399000C77A17EE907A5949B1F870106429A8BF18
:1039A0006421CDE900075648FFF74EFD95F8D03069
:1039B00095F8D120B5F8D410524806EB8303D3F81C
:1039C000D036FFF741FD504B5048198889B2FFF7B8
:1039D0003BFDFBF7BDFE016921B182684C48120D29
:1039E000FFF732FD4B48FFF763FC4B4B1B681B0690
:1039F00060D595F80031032B8CBF48484848FFF745
:103A000057FC94F81835022B26D14648FFF750FC96
:103A100095F80031042B44D84348FFF749FC95F84A
:103A20001031002B44D006EBC303D3F828173F48CE
:103A3000FFF7AAFCFFF744FC3D483E4FFFF738FC78
:103A40003D4B1C680125002C38D1FFF739FC17B01D
:103A5000BDE8F08F134684E702200EF0F1FC074624
:103A600008B93648D2E73FF02BF897F9041006EB77
:103A700080000131D0F8E4263148FFF785FC94F846
:103A80001B35012B04D12F48FFF712FC2E48BDE750
:103A9000BB792E4806EB8303D3F8E416FFF774FCDA
:103AA000F4E794F81A350BB92948B6E72948B4E782
:103AB0002949BCE72948FFF7FBFBBBE794FAA4F3CD
:103AC000B3FA83F305FA03F206EB83033846D3F81F
:103AD0005C1724EA0204FFF757FCB4E70C49002006
:103AE00029E1070808490020C81A00203BE107081F
:103AF00055E107080024744968B90020F01400104B
:103B000068E10708AEE1070890290020D5E1070821
:103B1000E4E10708FFE10708CC42002005E20708BE
:103B200011E2070821E20708A6FB070869E2070877
:103B300085E2070875E20708E444002027E2070849
:103B400031E2070845E207084AE20708CBEC07081C
:103B50004EE207085EE2070827E0070879E2070857
:103B60002DE9F04FDFF8708198F8033099B0002B01
:103B700000F094804F48504EDFF860B1DFF860915C
:103B8000DFF860A1FFF7B4FB00252F460BA9E8B2D0
:103B900016F028FF9DF83430002B53D0139C54B1FD
:103BA00007EE904A9FED450AF8EE677A80EE270A05
:103BB00058F0C8FE04460B9A29465846FFF7E4FB26
:103BC000109A002A6CD002FB04F04FF47A73B0FB19
:103BD000F3F30993DDF848C0BCF1000F62D00CFB91
:103BE00004F142F21073B1FBF3F198F80330082DA1
:103BF00018BF7F18002B57D017980790159806907C
:103C0000169805900A2311984FF47A7EB0FBFEFEB9
:103C10000998CDF810E0B1FBF3FE03FB1E11CDE9CE
:103C200002E10999B1FBF3F103FB1100CDE90010AA
:103C3000BCFBF3F321465046FFF706FC0023C6E920
:103C40000D33B3620135222D06F140069ED198F85E
:103C5000033003B31A4C1B48D4E945124FF47A736E
:103C6000D208B1FBF3F3D4F81C11FFF7EDFB0A22E5
:103C7000154897FBF2F102FB1172FFF7E5FB134BBE
:103C80001B78422B04D1D4E948211148FFF7DCFB13
:103C90000023C4F81C3119B0BDE8F08F0D486AE765
:103CA000099297E76146A0E721464846FFF7CCFB1B
:103CB000C4E700BF9BE20708B0B100208096184B14
:103CC00068B9002042E3070862E307084C28002097
:103CD00086E30708F9E20708B842002003E3070873
:103CE0002AF6070812E3070810B52948FFF7E0FA9B
:103CF000284B93F82130002B48D0274C2748FFF75A
:103D0000F7FA94F808312BB194F80A3113B194F80A
:103D1000093173B92248FFF7CBFA224B93F8C83028
:103D200053B394ED450A58F00DFE01461E48FFF7C7
:103D30008BFBB4F80C111D48FFF726FB94F80831F3
:103D4000F3B11B48FFF7D4FAB4F810111948FFF784
:103D50001BFB94F80A31ABB11548FFF7C9FAB4F868
:103D60000E111548FFF710FB94F8093163B11048A4
:103D7000BDE81040FFF7BCBA1048FFF7B9FAD8E722
:103D80000F48DFE70E48E8E70D48F1E70D48EFE799
:103D9000B0E30708D0420020F0140010C6E3070883
:103DA000CDE3070868B90020E7E30708F6E3070852
:103DB00016E4070826E4070840E40708ECE30708D0
:103DC0001FE40708A40008080EB403B503AA52F8BC
:103DD000041B0192FDF71BFD064BD3F80C291AB901
:103DE0000549186FFCF7B0FF02B05DF804EB03B0B3
:103DF000704700BF70A800205BEA07082DE9F04774
:103E000098460B7903F0E005402D81460F46164693
:103E100032D1644DDFF8A881DFF8B091002416E0BC
:103E20003B7903F00703013B042B04D8DFE803F0E0
:103E300014171A1D2100315D5A48FFF7A5FA7B7946
:103E4000013BA34202DD4846FFF732FA01347B7999
:103E5000A342E5DCBDE8F08731572846EDE736F8A8
:103E60001410FAE736F91410F7E756F82410404614
:103E7000E3E756F82410F0E703F00703052B57D8C3
:103E8000DFE803F0031F27292C3E3478602D55D03E
:103E90002CD8002D75D1B7F80550B7F80760414808
:103EA0002146FFF771FAAC4239DBB44237DCB8F196
:103EB000000FCFD0324629463B48BDE8F047FFF718
:103EC00063BA96F90040602D38D00FD8002D58D134
:103ED00051E03488DAE7B6F90040F4E7D6F800A0FC
:103EE000202D54464DD034D9602D27D0802DB1D10E
:103EF00032782E4B2E48002A14BF3146194635E041
:103F0000202D34683DD0EFD821462648FFF73CFAF3
:103F1000D7F80510A14202DB4B42A34221DDFFF797
:103F2000CFF93A68234923464846BDE8F0474BE7B6
:103F3000202D25D01ED9602DD8D100247B7944FABC
:103F400003F3DB07BDE8F0474CBF1B481B48FFF7F6
:103F50001BBA51461A48FFF717FAD7F805108A45D9
:103F6000DDD8B8F1000F3FF475AF1648BDE8F04753
:103F7000FFF70ABA0024B7F90550B7F907608EE7D2
:103F800000247A79104B03EBC20393F89424A242E5
:103F9000C5DDD3F8903453F82400BDE8F047FFF7AF
:103FA00087B900BFCEFF0708BDED070817FA07085D
:103FB0008EF6070866E407082BDF0708A400080848
:103FC000C3DE070860E40708C8FD0608E7E0070845
:103FD00070B50546084616460C46FCF7FFFC33460E
:103FE000024621462846BDE8704007E70EB403B5F7
:103FF00003AA52F8041B0192FDF709FC044B054982
:10400000186FFCF7A1FE02B05DF804EB03B0704737
:1040100070A800205BEA07080049E7E780E407088A
:1040200038B50C46054615492046FCF7F3FA30B979
:10403000FFF7F8F81248BDE83840FFF759B91149C1
:104040002046FCF7E7FAA8B90F4B83F8D90183F8AB
:10405000E10183F8B50283F8BD0283F8910383F888
:10406000990383F86D0483F87504084B83F82100E5
:104070000748E0E72846BDE83840CDE78FE4070869
:1040800095E40708B0E4070870A800203C4500202C
:10409000B8E407080049A9E7D4E40708F8B50646DC
:1040A00008460C46FDF7F4FD20210546204659F050
:1040B000F0F8044618B93046BDE8F840EAE7114F79
:1040C000114E3B7832789A4201D0FBF789FC0F4BB6
:1040D00020461D6056F012FE012201462046FBF7E5
:1040E00027FC3B7832789A4201D0FBF779FC2046D6
:1040F00056F004FE2A460146BDE8F8400448FFF7A2
:10410000A3B900BF902200205F3D00208C22002038
:10411000EBE407082DE9F041064688B008460D4655
:10412000FDF7B6FD20210446284659F0B2F820B923
:10413000304608B0BDE8F041ACE7FDF7A9FD2246E6
:10414000054601460F48FFF77FF985B1202D2A4625
:10415000694628BF20222046FBF78AFCE84606462F
:104160000027B74208DBAD1B3444002EEDD1FFF72A
:10417000A7F808B0BDE8F08118F8010BFFF7E2F8E6
:104180000137EEE701E507082DE9FF470746084636
:104190000D4656F0B3FD082845D105F1FF3801AEB4
:1041A000073531464246B14612F8010FFDF78EFC45
:1041B000AA4201F8010BF7D10023DFF87CA08DF8AB
:1041C0000C30A84517D11B4948462EF005FE19486A
:1041D0001949082310F8012B11F8014B10326A44D9
:1041E000013B02F80C4CF5D114488DF80C3001A9B4
:1041F000FFF72AF914E018F8010FFDF767FC06F83D
:10420000010B04460146504659F043F828B12146B7
:10421000304659F03EF80028D3D03846FFF7FCFE70
:1042200004B0BDE8F0870028D1D0384604B0BDE81E
:10423000F0472FE7D0420020587E070819E507080D
:1042400007B5009313460A460249FFF7CFFE03B0B5
:104250005DF804FB20E5070810B504460748FFF7A2
:1042600047F8FBF71BFF20B1BDE810400448FFF7FB
:104270003FB820460349BDE81040B7E639E50708D6
:1042800043E507084BE507082DE9F041144B1B688F
:1042900088B00446F3B11A6804A9D56A18466A467C
:1042A000A847064688B1DFF8448004AC6D46002775
:1042B00035F8022B34F8021B40460137FFF7C4F8EB
:1042C000BE42F5DC08B0BDE8F08106492046FFF7A4
:1042D0008DFEF7E7044908B0BDE8F04186E600BF6F
:1042E000884500206CE5070884E5070852E50708C3
:1042F00070B5054608460C4656F000FD024668B10A
:104300000B2804D10848214658F0E9FF30B128466F
:10431000054B064A0649BDE8704067E6BDE87040B7
:1043200001490448FFF790B8006B07088BE50708C0
:1043300096E50708C0E5070870B5054608460C462F
:1043400056F0DCFC024668B1032804D10848214637
:1043500058F0C5FF30B12846054B064A0649BDE86E
:10436000704043E6BDE8704001490448FFF76CB86F
:10437000FC6A0708CEE5070896E50708DEE50708AA
:104380002DE9F04306469BB008460C4656F0B6FCB5
:1043900020220546002101A858F064FF2DB3402DCE
:1043A00007D03A4940232A4630461BB0BDE8F043C7
:1043B0001CE601AF04F140084FF00009022221463B
:1043C000684658F09EFF0023102209A968468DF820
:1043D0000290FDF7BDFB099B0DF10202934222D131
:1043E0000234A04507F8010BE8D14122002109A8B9
:1043F00058F038FF002D3AD0254C94F82850D5B10C
:10440000202204F12C0101A858F0B0FF98B104F16A
:104410002C0109A8FDF7CEFA1E4A1F4909AB304608
:10442000FFF7E4FD04E01A781C493046FFF7DEFD93
:104430001BB0BDE8F0832379CBB9C5B901AC0FCC73
:10444000174D0FC594E80F0085E80F00154B0122AA
:1044500009A8A5F1100183F82821FDF7ABFA12484D
:10446000FEF74CFF114809A9FEF7EEFFE0E70D4B00
:1044700093F8283123B9064B93F82830002BF1D05C
:10448000074909A8FDF796FAECE700BFF1E5070830
:1044900070A800202FE6070896E5070813E607082E
:1044A0009CA8002068B9002039E6070848E60708FC
:1044B0002DE9F74F834608460C4656F01FFCDFF8FF
:1044C00018810646D8F8007028B1024633492046C4
:1044D000FDF702FB80B93946314850F0ABFB31495A
:1044E000314821EA070150F0A5FB3049304803B0BC
:1044F000BDE8F04F50F09EBB23782D2B2D4B03BF12
:10450000013406F1FF364FF0010A4FF0000A4FF078
:1045100000094FF0FF3553F8041B51B132462046D5
:104520000193FDF7D9FA019B00280ABF4D460021EF
:10453000012109F1010989B9B9F11D0FEBD11E491A
:104540002246584603B0BDE8F04F4FE53B43C8F85C
:1045500000301A491A4B12E01A4913E0114A01239C
:10456000AB401A40002AF7D007EA0302BAF1000F65
:10457000ECD027EA0303C8F800301349134B002A94
:1045800018BF1946124B134803EB8503D3F8C8270D
:1045900003B0BDE8F04FFEF757BF00BFFEE20708CB
:1045A00080E60708BCD677188AE60708432988E71B
:1045B00096E6070890050708A4E6070878E60708C6
:1045C00071E6070855E6070861E6070868E6070888
:1045D000C8FD060800ED0708B44900202DE9F74F93
:1045E000019008460E461746984656F087FB04464B
:1045F000E8B93F483F4DFEF7C7FE20460DF0D0FE1C
:104600003B68184206D020460DF0DCFE01462846E5
:10461000FEF7BAFE0134182CEFD13B6813B93648C7
:10462000FEF746FE03B0BDE8F04FFEF749BE024676
:1046300032493046FDF750FA0546A8B93048FEF732
:1046400037FE2C462F4D20460DF0AAFE10EA080F2B
:1046500006D020460DF0B6FE01462846FEF794FE31
:104660000134192CEFD1DDE733782D2B03BF013650
:1046700004F1FF34012500254FF0000948F0807B4C
:1046800048460DF09FFE2246824601463046FDF721
:1046900023FA00BB48460DF083FE1BEA000F1AD038
:1046A0008DB1B9F1180F1CBF3B6840EA03081648EA
:1046B000C7F80080FEF7FCFD1248514603B0BDE884
:1046C000F04FFEF7C1BEB9F1180F1CBF3D6885431E
:1046D0003D600E48EEE709F10109B9F1190FCFD19C
:1046E0000B490198324603B0BDE8F04F7EE400BFAD
:1046F000B5E6070874E20708BFE60708FEE2070808
:10470000C6E6070875E2070868E6070878E60708BE
:10471000A4E60708014A40F202235FE700450020B3
:10472000014A6FF07F4359E7F844002010B5044672
:1047300001202EF0C1FB20B920460449BDE81040FD
:1047400054E4BDE810400248FEF77EBED1E60708FB
:10475000E0E60708064B10B50446D3F82C013EF0FE
:1047600013F920B920460349BDE810403EE410BDCE
:1047700068B90020EBE6070870B5054608461646FE
:10478000FDF786FA0D4B041E1A780EDB944205DA0B
:104790000B482146FEF758FE204670BD2EB1FF2C77
:1047A00003D10848FEF750FEF6E70749013A2846CC
:1047B000FFF71CFC4FF0FF34EEE700BFA80D001020
:1047C00001E7070812E7070825E707082DE9F04F7A
:1047D000074691B08248834D0E46FEF735FE82496A
:1047E000C5F830D1002385F8343106220123097839
:1047F0003046402485F8354108F070FF0A20F5F76F
:1048000031FE95F834310C2BDAB240F2E4809DF899
:104810000C60FE2E2CD0FF2E15BF0F241524002572
:104820000125944240F0D780611EC9B268464BF022
:1048300099FE04F140030DEB030414F8413C83425C
:1048400040F0C4806A1E012A9DF80D3012D903F091
:104850001F0761375C096548FEF72AFD022D39D034
:10486000013C042C34D8DFE804F00B2D2F33310049
:104870000225D6E79DF80E709DF80F401E46EAE728
:104880005B48DFF8C491DFF8C4A1DFF8C4B1FEF7DC
:104890002FFD5848FEF70CFD6C464FF0000814F849
:1048A000011B484608F10108FEF76EFDB8F10C0F38
:1048B00016D00AFB08F3B3F1553FF0D85846FEF77F
:1048C000F7FCECE74C48DCE74C48DAE74C48D8E723
:1048D0004C48D6E700238DF83F300DF11F00D0E79C
:1048E000FEF7EEFC022D3AD06422B6FBF2F102FB99
:1048F00011623B464448D2B2C9B2FEF7A5FD85F02D
:1049000001035B42DBB2012B59D8404A404B9DF872
:1049100010104048404E00290CBF11461946FEF7C2
:1049200093FD9DF811103D4B3D4800290CBF3146C9
:104930001946FEF789FD022D41D19DF812403948F4
:10494000FEF7B6FC8CB1FF2C1FD00A23B4FBF3F1A9
:1049500003FB11423448D2B2FEF776FD08E033483B
:104960003A463146FEF770FDCFE73046FEF7C0FC11
:104970009DF813402E48FEF79BFC44B1FF2C21D03C
:104980002C482146FEF760FD04E02B48EEE7224864
:10499000FEF7AEFC204E214FDFF89C800DF1130591
:1049A000002415F8013F7BB1FF2B14BF3A46424665
:1049B000214622480134FEF747FD042CF1D111B005
:1049C000BDE8F08F1C48E3E73246F1E71C49384662
:1049D000FFF70CFBF3E71B48FEF78AFCEFE700BF8D
:1049E0006BE7070868B90020A80D00107CE70708EE
:1049F00087E70708ADE707088EE7070896E7070887
:104A00009EE7070827E00708BFE7070854E70708FD
:104A10004BE70708F6E707085BE70708F5F707081D
:104A20000DE8070814E8070828E80708DBE7070887
:104A300030E80708CEFF07085FE7070840E80708E7
:104A40004BE807085BE807083ADE0708ABAAAAAA02
:104A500017FA07082DE9F843DFF8A49007460C463B
:104A6000204656F04BF9064658B91D4B1D481A789A
:104A70001D4B03EB8203D3F83818BDE8F843FEF76B
:104A8000E3BC024649462046FDF726F860B1DFF850
:104A90006480002558F8041BB1B9224638461349F2
:104AA000BDE8F843FFF7A2BA1148124C124DFEF7C9
:104AB000FFFB54F8041B19B12846FEF765FCF8E724
:104AC000BDE8F843FEF7FCBB32462046FDF704F88C
:104AD00001350028DED1024B084C1D70C0E700BF35
:104AE0007443002064E80708C8FD0608A4E6070828
:104AF000C6E607080406070875E207085DEA070826
:104B0000FEE2070838B50D4604461A490522284634
:104B1000FCF7E2FF68B9184B93F8742022B9012121
:104B200083F8741083F87520BDE838401348FEF709
:104B3000DFBB134903222846FCF7CEFFA0B90E4D78
:104B400095F8743063B195F875304BB10D49204636
:104B5000FFF74CFA002385F8743085F8753038BDBE
:104B60000948FEF7C5FBF5E720460849BDE838408F
:104B7000FFF73CBA3CF7070870A800206EE807086A
:104B80009EF8070884E80708BBE80708CFE807088D
:104B900070B5164C94F8743005467BB194F87530B6
:104BA00063B11349FFF722FA28461249FFF71EFAAC
:104BB000002084F8740084F8750070BD0E4E96F8DD
:104BC000283183B194F828306BB90C4D0FCD06F520
:104BD0009C740FC495E80F0084E80F00012386F849
:104BE000733109F0ABFE0120E7E700BF70A8002099
:104BF00084E80708DEE8070868B900209CA80020C0
:104C000008B5034610460AB9002008BDDB0601D5E9
:104C10000029FAD0FEF772FBF6E7F8B50C4E3379AF
:104C200005468BB9F8BD25B12388C3F30B039D421C
:104C300004D0D4E90201A28858F0BCFA1C34BC426A
:104C4000F1D300233371EDE7024C034FF7E700BFC8
:104C500070A8002090010808300B08082DE9F04FDB
:104C6000164685B0CDE901011A4600213046FFF70E
:104C7000C7FF314C009006F010034FF00009A24628
:104C80000393FEF7F9FA2379029A03F0180393428B
:104C900003D0002A44D1182B42D14FF00D0B0BFB4F
:104CA00009A3B3F80900FBF73DFB80462046FBF75C
:104CB00062FED8E902210746024401442046FBF780
:104CC00013FE80F00101009A0546C9B23046FFF795
:104CD00097FF039B009003B115BB0BFB09FBB306C9
:104CE0005AF80BB00ED56DB914485946FEF74CFB77
:104CF000D8F8082001982B463A442146FFF77EF861
:104D0000FEF7DEFA0E485946FEF73EFBD8F80C20B7
:104D1000019800233A442146FFF770F8FEF7D0FAD5
:104D200009F1010940F27D23994504F10D04A8D150
:104D300005B0BDE8F08F00BF080F0708FCE80708C2
:104D4000FDE8070820B10078B0FA80F0400970470C
:104D5000012070472DE9F74F81460846FFF7F2FF23
:104D60000E46054670B1002401A9204650F052F8C5
:104D7000013401464846FFF7EDFF122CF4D103B091
:104D8000BDE8F08F0846FCF783FFC4B2112C71D840
:104D9000701C3D4D3D4EFBF7E7FF05EB44086700F7
:104DA00098F874A18346B8B9AAF102014B424B416D
:104DB0003D4495F87421B25C002B54D095F87531C0
:104DC000192040F2EE2100FB03133148214603B0C5
:104DD000BDE8F04FFEF738BB0178304658F059FA7D
:104DE00078B1032C94BF002201222A4902EB42022F
:104DF000831B0A4452FA83F393F8A8A8BAF1030F6D
:104E000005D1484603B0BDE8F04FFFF705B9584655
:104E1000FBF7AAFFF0B1BAF1020FF2D1FCF738FFAD
:104E200040F6CA0380B29842A8BF184640F2EE236B
:104E30009842B8BF1846A0F2EE201923B0FBF3F059
:104E400088F87501AAF1020253425341EA1982F827
:104E500074A1ADE7BAF1020FF4D1484603B0BDE842
:104E6000F04FFFF717B90C48214603B0BDE8F04FEB
:104E7000FEF7EABA094911232A46484603B0BDE8BD
:104E8000F04FFFF7DDB900BF68B900207880070850
:104E900007E90708C8FD060817E9070824E9070815
:104EA0002DE9F04F0346A1B00846FFF74BFF05463A
:104EB00028B1184621B0BDE8F04FFFF7EBB8DFF896
:104EC0000CA30B90FF238DF82830DAF82C31ADF8C5
:104ED0003000CDE9050093F838200D908DF838208A
:104EE0000F90ADF840001193099107464FF0FF383D
:104EF000A34909A858F06CF9044658BBA14E0346D3
:104F00000AAC1A01A04912570F46002017F901CB2D
:104F1000624540F0EC805F1C002311F9010B8242D6
:104F200040F0EC80994A02EB8303D3F8B02898480C
:104F30003946FEF789FA022F4FF00103E1D19DF9BE
:104F400038A09DF92830534540F0DE809148FEF7A7
:104F50007BFA57E02378002BCAD0032FD4BF00265A
:104F60000126062F00F2BC80DFE807F0045760A29C
:104F700004576000042F10D087492046FCF7D0FD6D
:104F800058B14FF480600DF05BFA002800F0D38137
:104F900090F90400012306930AE080492046FBF7BC
:104FA00039FB70B9DAF82C3193F93800042F32D07C
:104FB000119B119320AB03EB061606F8580C013732
:104FC00096E7DFF80CB24FF000095BF8041B2046AF
:104FD000FBF720FBC8B96C4B13F909000028E5DA90
:104FE00001230A2212A92046FCF7B2FD40B2002894
:104FF00003DB129B1B78002BD8D069482246711C1A
:10500000FEF722FA21B0BDE8F08F09F10109B9F1EC
:10501000070FDAD1E4E70023CBE72046FCF738FEA0
:1050200020AB03EB061646F8540CC8E75D49204652
:10503000FCF776FD5C49B0F1000B204618BF4FF03D
:10504000010BFCF76DFD08B14BF0020BDFF884C1DA
:1050500020AB4FEA061903EB0616BCE80F0006F872
:1050600050BC12AE0FC6BCE80F000FC6BCE80F0064
:105070000FC69CE8030086E8030000260DF1480BEC
:105080003346DBF800100793204658F059F9079B88
:1050900010B19BF8042016430133072B0BF1080BCA
:1050A000EFD109F180030DEB030909F84F6C86E796
:1050B0003E492046FBF7AEFAB0B13D492046FBF72A
:1050C000A9FA00283FF47BAF2046FCF7E1FD032856
:1050D00080467FF674AF01463648FEF7B5F991E792
:1050E0003548224608218BE70123059367E7013005
:1050F00007287FF40BAF3148591C81E70133072B98
:105100007FF40BAF324612E70B9B1BB9AAF11402D6
:105110005542554100235F1CE368002B67D194F989
:1051200000B058460DF05CF9D4F8049018B1066848
:10513000002E40F09080B9F1000F237A14BF4E4644
:105140004FF46146666023B91D48FEF77DF90323DD
:105150002372627A2AB11B4807923946FEF774F926
:10516000079A0292237ACDE9006300231A46194672
:1051700058460DF07FF9E06070BB13483946ACE744
:10518000D5ED07082CE907082CEC0608C8FD060831
:10519000CAE90708D5E9070851E907085CE90708E3
:1051A00060E907087BE9070822F807087EE9070895
:1051B000C1E6070884E907089CE90708B8E9070879
:1051C000EEE9070809EA070824EA070868B9002099
:1051D00078060708940607085849594A5948B9F10A
:1051E000000F18BF0A4633463946FEF7CDF8022FA6
:1051F00004F110044FF001038DD1119E0D9F4DB1AC
:105200005148FEF775F833681B6A1BB14F493A469F
:1052100030469847059B002B50D04D49474BBAF17B
:10522000140F18BF19464B48FEF70EF9BAF1140FC8
:1052300009D1059B002B43D03368DB691BB146497C
:10524000002230469847069B002B43D1002231466E
:1052500038464FF093FDE660B9F1000F2CD0494677
:10526000304603F03BFD3D4AB3683D483946FEF702
:10527000EBF894F80890B9F1000F0CD03279914511
:1052800009D038484B463946FEF7DEF833684946C0
:105290009B6930469847637A23B172793248394620
:1052A000FEF7D2F8F36A002BA1D030483946FEF75A
:1052B000CBF80023F3629AE7204AD5E71F49B2E70B
:1052C000B8F1000FBFDB3368DB69002BBBD0284986
:1052D0004246B6E708F0A6FD0520F5F7C3F8DFF86B
:1052E0009490DFF894A000254FF0030B9AF800305B
:1052F000AB42ABD919F8014FC4B1204609F0BCF953
:10530000804698B1204608F0A1FCEBB2044610B1EB
:1053100080F806B0C37120460121F5F77BFB98F8B1
:105320000630DB07204603D5F5F74EFD0135DDE7F6
:10533000F5F73AFDFAE74FF0FF302BE65DEA070894
:1053400036E9070840EA0708F6EA0708DD8C010895
:1053500044E907081FEB0708830D01083FE9070828
:105360005EEA070883EA0708A6EA0708DDEA0708F5
:105370008B0A0108B3280020A80D00102DE9F74F73
:1053800005460846FFF7DEFC0B46044618B9334ACB
:1053900092F898712FB9284603B0BDE8F04FFEF798
:1053A0003BBE2F49DFF8C890DFF8C8A001AA184615
:1053B00057F03BFF264610B908F042FD08E056B909
:1053C000012201462846FFF7D7F9421C04461AD1AC
:1053D00003B0BDE8F08FFCF75BFC2F28834636D87E
:1053E0000FB108F01FFDBBF1060F13D01D490123BB
:1053F00009785FFA8BF2E0B208F070F95946484636
:10540000FEF722F80027164901AA0020013657F0BE
:105410000CFFD0E7DAF800301B0114D5FF2C0ED0BA
:10542000E1B22846FFF7D2F9E8E72846FFF7CEF9C0
:10543000013798F80020F9B28A42F6D8DEE7DFF8A3
:1054400024800027F5E70848FDF752FFD6E7074913
:105450002F222846FEF7CAFDD5E700BF68B9002015
:10546000D5ED0708A80D0010D1E6070853EB070893
:1054700042EB0708CC4200202DE9F74307460846D7
:10548000FFF760FC0B46044628B1384603B0BDE880
:10549000F043FEF7FFBD2F49DFF8B89001AA184688
:1054A00057F0C3FE26460546A04665B92A4B32464C
:1054B000D3F82C01A1B255F0ADF968BB27493846A5
:1054C000FEF794FD28E0B8F1000F06D0B8F1010F07
:1054D00025D03846FEF7DEFD1EE0284655F00EFCCE
:1054E0001F49064602462846FCF7F6FA50B31D4906
:1054F00032462846FCF7F0FA30B31B4932462846BC
:10550000FCF7EAFA10B3194932462846FCF7E4FAE8
:10551000F0B13846FEF780FD03B0BDE8F083B31E5E
:105520005A425A4129463846FFF726F9421C04469A
:10553000F2D001AA4946002057F077FE08F1010891
:105540000546B2E74646F4E70126F2E70226F0E711
:105550000426EEE7D5ED070868B900207FEB0708C1
:1055600073EB070876EB070879EB07087CEB070875
:105570002DE9F74380460846FFF7E4FB0B46054656
:1055800028B14046FEF786FD03B0BDE8F0832E4902
:10559000DFF8B49001AA184657F047FE2F4604469C
:1055A0002E467CB9022DECD1A7F57A73B3F57A7F3C
:1055B00021D926494FF4FA634FF47A724046FEF738
:1055C0003FFEE1E74DB1012D10D001AA4946002070
:1055D00057F02BFE01350446E3E701222146404601
:1055E000FFF7CAF8431C0646EFD1CDE72046FCF78B
:1055F0004FFB0746E9E7164B1B68B8B25B68984754
:10560000FF2EBCEEC00A0CD1124BF8EE407A1A788D
:10561000114BA24213DC10EE101A1048FDF714FFD4
:10562000B2E70F4B0F48F8EE407A03EB860310EE1B
:10563000102A3146C3ED677AFDF706FFA4E7E3ECD5
:10564000017A0134E5E700BFD5ED07088DEC0708C6
:10565000EC140010A80D001004BB0020AAEB0708F2
:1056600068B900209DEB0708F8B507460846FFF724
:1056700069FBC8B11F4B5E69013630460CF0A2FED3
:1056800034460546F0B90134192CA8BF0024204641
:105690000CF098FE0546A8B9B442F4D13846164934
:1056A000BDE8F840FEF7A2BC0846FCF7F1FA044654
:1056B0000CF088FE054628B921461048BDE8F840A0
:1056C000FDF7C2BE0B4B5C610CF09EFF0C482A46F6
:1056D0002146FDF7B9FE182C09D80A4B0C2202FB13
:1056E000043393F80409BDE8F8400CF0C3BF002070
:1056F000F9E700BFB8050020B9EB0708CDEB0708B4
:10570000E3EB0708C8FD060838B5124D0446084605
:10571000FFF718FB60B1104B104893F900104B1CB9
:105720000ABF0F4BC9B21978BDE83840FDF78CBEEF
:105730000846FCF7ADFA032804D8C0B2FDF7D4F947
:105740002946E4E720460749BDE838400322FEF732
:105750004DBC00BF5DEA0708B8050020FCEB070858
:10576000B84200200CEC070838B5124D0446084634
:10577000FFF7E8FA60B1104B104893F901104B1C89
:105780000ABF0F4BC9B25978BDE83840FDF75CBE7F
:105790000846FCF77DFA032804D8C0B213F00EFBCC
:1057A0002946E4E720460749BDE838400322FEF7D2
:1057B0001DBC00BF5DEA0708B8050020F8EB07082C
:1057C000B842002007EC07082DE9F74F444BDFF8FB
:1057D0002C911A785B7889F80130424B00911B7943
:1057E00089F8002005460BB907F01CFAFBF7FAFB15
:1057F00000263D4CB0460D233B4A0099734352F8B6
:1058000003A05046FCF78CF9002841D0B8F1000FF6
:1058100001DDFDF755FD35485146FDF7B5FD002288
:1058200021462846FEF7D4FBFDF74AFD237903F015
:105830001803082B46D0102B49D02046FDF713FE45
:10584000294B0D2202FB0633B3F80900FAF76AFD73
:105850008346D8B12046FBF78EF8DBE902210746E4
:10586000024401442046FBF73FF878B901905146C5
:105870001F48FDF789FDDBF80810019A28461346FA
:10588000CA192146FEF7BAFAFDF71AFD08F1010818
:10589000013640F27D239E4204F10D04ABD100207D
:1058A000FFF7BBF9FF2389F8003089F80130B8F120
:1058B000000F11D1009A0F49284603B0BDE8F04F00
:1058C000FEF794BB0C492846FFF71EFFB5E70A49CF
:1058D0002846FFF749FFB0E703B0BDE8F08F00BFEF
:1058E000B842002070A80020080F070801E9070847
:1058F00027EC0708A4E607085DEA0708B8050020BA
:105900002DE9F74F804608460F4655F0F7F9044653
:1059100020B1012825D13B782A2B22D1A948AA4EB3
:10592000AA4FFDF7E5FC0025B1464FF00D0A04F043
:1059300001040AFB05F3384659F80310FDF724FD6E
:10594000314622464046FEF743FB0135FDF7B8FCE1
:1059500040F27D239D4206F10D06EAD103B0BDE879
:10596000F08F3D21384657F094FC002800F0238149
:1059700003469A4613F8012D202AFAD0AAEB070A0B
:105980000130054610F8013B202BFAD0DFF838B281
:105990005FFA8AFA4FF000090D2303FB09F3524620
:1059A0005BF80310009138460BEB0304FCF794F806
:1059B000064670BB0099084655F0A0F9824528D1EB
:1059C000277907F0E001402900F0898012D871B3EF
:1059D00066797F4A02EBC606002796F89424009267
:1059E000BA463B46009ABA4202D9BAF1000F62D0D9
:1059F0002BB12DE06029ECD0802900F0A480404636
:105A00007449FEF7F3FA204603B0BDE8F04FFDF706
:105A10002ABD09F1010940F27D239945BCD16E49A7
:105A20003A46404603B0BDE8F04FFEF7DFBA07F054
:105A30000703042B1CD10B460A222846FCF788F8E2
:105A4000D4F8053083420146D9D32046FAF7DAFF6D
:105A50000D2303FB09F961485BF80910FDF794FC7D
:105A600000222146404603B0BDE8F04FFEF7B0BA31
:105A7000052B0DD101230A222846FCF769F8D4F83A
:105A8000053083420146BADB5B428342B7DCDCE788
:105A90002846FCF7FDF817F0050F0BBFB4F80520FA
:105AA000B4F90520B4F80730B4F907309042014644
:105AB000A5DB9842EAE7D6F8901451F8270060B1C8
:105AC00029460193FAF7A6FD019B30B939462046D5
:105AD0004FF0010AFAF796FF5346013782E76379E0
:105AE000009307F00707013F009BB342B0DDAA46D1
:105AF00015F8013B202BFAD02046FAF76FFF054638
:105B0000042F04D8DFE807F0030E0E141D005046E2
:105B1000FCF7BEF8A8552C21504657F0BAFB0136C9
:105B2000451CE1E75046FCF7B3F825F81600F2E70C
:105B300000230A2200215046FCF70AF845F8260007
:105B4000E9E70123F5E7284655F0D8F8E37994F81A
:105B500005A0A779DB0706460AD52046FAF73EFFDF
:105B60000378014623B13246284657F0B8FBE0B926
:105B7000DEB1B74219D32046FAF730FF3A4600218A
:105B800057F070FBB2453FF663AF154932462846E1
:105B900057F0A5FB00283FF45BAF2046FAF71EFF45
:105BA0003246294657F006FB52E70E493A46404630
:105BB000FEF71CFA23E73946404603B0BDE8F04F34
:105BC00002E600BF37EC0708080F070801E90708DD
:105BD000C8FD060885EC0708A4E607087AEC070864
:105BE00017FA07084AEC07082DE9F04F914687B0ED
:105BF0000C461A4600218046FFF702F84D4606463D
:105C00000027B9F1000F66D029460622204657F03A
:105C1000ADFB0028324614BF0121002140460CBFD5
:105C20004FF0010A4FF0000AFEF7EAFF0646287817
:105C300014F042FC8346F8B1687914F03DFCAB786F
:105C4000EA789BF805E095F801B04FF461714FF0E8
:105C5000190C1CFB03131CFB0212297900B14079BB
:105C6000CDE90410CDE90232CDE900EB1B4A3B46F9
:105C700051464046FDF770FB207814F01DFC83462A
:105C8000F8B1607914F018FCA378E2789BF805E08D
:105C900094F801B04FF461714FF0190C1CFB031321
:105CA0001CFB0212217900B14079CDE90410CDE945
:105CB0000232CDE900EB094A3B4651464046FDF72A
:105CC00003FB0137142F04F1060405F1060598D1F2
:105CD00007B0BDE8F08FCA46CEE700BF93EC0708D7
:105CE0002DE9F041054686B00846FFF72BF80F4630
:105CF000064638B100235C491A46012006B0BDE8CB
:105D0000F04171E70846FBF7C3FF1328044600F390
:105D1000A18006254543781C8DF81760FBF724F811
:105D2000524E074660B1FBF7B3FFC0B213F02AF83A
:105D300030B17319027983F8D82501238DF8173013
:105D40003846FBF711F8074668B1FBF7A1FF0D28AD
:105D500009D8062303FB046383F8D9059DF817309F
:105D600001338DF81730DFF80081A91C0DF11702FF
:105D700041443846FBF790FFFAF7F6FF074668B153
:105D8000FBF786FF012809D89DF81730062202FB91
:105D90000462013382F8DC058DF817303846FAF7D3
:105DA000E3FF80B1FBF774FFC0B212F0EBFF50B11C
:105DB0009DF817300179062202FB0462013382F854
:105DC000DD158DF817309DF81720042A4FF00603D3
:105DD0002FD103FB04630022A3F8DC25062505FB75
:105DE00004651FF06BFC95F8D80514F065FB95F879
:105DF000DB1595F8DA7519234FF46172804695F832
:105E0000DD0513FB012613FB072714F055FB43792F
:105E100098F80520039395F8DC350097CDE90163E8
:105E2000134895F8D9352146FDF70EFB06B0BDE8BD
:105E3000F081052A05D103FB0463002283F8DD25E8
:105E4000CCE7062ACAD008EB0502002348F8053043
:105E50009380C3E7074913233246284606B0BDE8BE
:105E6000F041FEF7EDB900BF48AE002070A8002059
:105E700093EC0708ACEC07082DE9F04F904689B089
:105E80001A460C4600218146FEF7BAFE384EDFF86E
:105E9000E4B008F1540307464546079394F904001B
:105EA0000CF09EFA002857D0B8F1000F5DD02946BB
:105EB0000C22204657F05AFA00283A4614BF012116
:105EC000002148460CBF4FF0010A4FF0000AFEF7D0
:105ED00097FEEA7995F9043006EB82020746D2F87C
:105EE000E42604922A7A06EB82025146D2F8E4268E
:105EF0000392AA7906EB82024846D2F8E42602927F
:105F00006A7906EB8202D2F8E42601922A680092AE
:105F10005A46FDF721FAE27994F9043006EB820241
:105F20005146D2F8E4260492227A06EB82024846D1
:105F3000D2F8E4260392A27906EB8202D2F8E42694
:105F40000292627906EB8202D2F8E426019222687C
:105F500000925A46FDF7B8F9079B0C35AB4204F1A5
:105F60000C049BD109B0BDE8F08FC246D3E700BF57
:105F7000C8FD0608B2EC07082DE9F04707468AB0CD
:105F80000846FEF7DFFE044638B1002353491A469F
:105F900001200AB0BDE8F0476EE70DF11C0807903C
:105FA000C8E9010008464E1CFBF772FE4B4D40B29B
:105FB00095F90430834200F08C800134072C05F100
:105FC0000C05F5D100252C463046FAF7CDFE0646E5
:105FD00038B100230A221946FBF7BAFD01340790B5
:105FE000E4B2DFF800A14FF000093046FAF7BCFE3A
:105FF000064620B3FBF74CFE394A002352F8041B37
:10600000884224D1DBB20AEB8302D2F8E426904224
:1060100015D1B9F1020F24D0B9F1030F26D05A1EC1
:10602000B9F1010FD2B217D00B2A03D88DF8213065
:106030000134E4B209F10109B9F1040FD5D1052CFD
:106040001AD838460AB0BDE8F047FEF723B8013346
:10605000102BD3D10023D6E7042AEBD88DF82230B9
:10606000E6E7052BE6D88DF82430E1E79A1E0D2AE5
:10607000E0D88DF82330DBE798E80700194B85E876
:1060800007009DF8232003EB82020021D2F8E426CA
:1060900004929DF8242003EB82020846D2F8E426FD
:1060A00003929DF8222003EB8202D2F8E4260292AA
:1060B0009DF8212003EB82030B4AD3F8E4360193C9
:1060C000079B00939DF92030FDF7FEF80AB0BDE86C
:1060D000F0878DF82000012476E700BF2CAD00206A
:1060E000AC040708C8FD0608B2EC07082DE9F04F1C
:1060F00090468BB00C461A4600210746FEF780FDFD
:106100004546099000264FF0190A4FF46179B8F11D
:10611000000F4BD029460A22204657F027F90028C5
:10612000099A14BF0121002138460CBF4FF0010B22
:106130004FF0000BFEF764FD2A890692EA8805926B
:106140002A790492EA780392AA7809901AFB0292BB
:1061500002926A781AFB029201922A7800923346E0
:10616000134A59463846FDF7F7F822890692E28825
:10617000059222790492E2780392A2781AFB0292A5
:10618000029262781AFB0292019214F80A2B009292
:106190003346074A594638460136FDF795F81E2E14
:1061A00005F10A05B3D10BB0BDE8F08FC346DCE7BB
:1061B000CFEC07082DE9F04380468BB00846FEF788
:1061C000C1FD0F46044638B100235E491A4601203E
:1061D0000BB0BDE8F04389E70846FBF759FD1D28E1
:1061E000054600F3A5800A264643781C8DF8274013
:1061F000FAF7BAFD10B101238DF82730FAF7B4FD94
:10620000514C074668B1FBF743FD0D2809D80A2316
:1062100003FB054383F8BC019DF8273001338DF85B
:106220002730DFF82091711C0DF1270249443846D0
:10623000FBF732FDFAF798FD074668B1FBF728FD3A
:10624000222809D89DF827300A2202FB0542013393
:1062500082F8BF018DF827303846FAF785FD0746EA
:1062600068B1FBF715FD0D2809D89DF827300A22E3
:1062700002FB0542013382F8C0018DF827309DF8FA
:106280002730062B0CD009EB06020023404649F8C4
:106290000630536013810BB0BDE8F043FDF7FABE42
:1062A0000A2606FB054600233846A6F8C231A6F8A2
:1062B000C431FAF759FD074618B1FBF7E9FCA6F817
:1062C000C2013846FAF750FD30B1FBF7E1FC0A2372
:1062D00003FB0543A3F8C4011C4B4FF0FF325A6087
:1062E0000A2303FB05424FF46170B2F8C4310693F0
:1062F000B2F8C231059392F8C031049392F8BF31DD
:10630000039392F8BE11192313FB0101029192F835
:10631000BD1113FB0103019392F8BC3100930021DE
:106320000B4A2B460846FCF7CFFF0BB0BDE8F083C5
:1063300008491D23224640460BB0BDE8F043FDF757
:106340007FBF00BF24BB002068B90020B805002033
:10635000CFEC0708ACEC07082DE9F04F2DED088BCA
:10636000DFF828A195B0804691461E460C4615469A
:10637000002794ED008AB5EE408AF1EE10FA7DD048
:10638000D4ED019A94ED029AD4ED038AB9F1000F8D
:1063900049D0D5ED00BA95ED01BAD5ED02AA95ED3B
:1063A00003AAB4EE6B8AF1EE10FA6CD1F4EE4B9ABC
:1063B000F1EE10FA67D1B4EE6A9AF1EE10FA62D1FA
:1063C000F4EE4A8AF1EE10FA0CBF012100213246A8
:1063D0008B46404681F00101FEF712FCB0EE6B0ADD
:1063E000064611A8FAF73EFCB0EE4B0A07900EA83D
:1063F000FAF738FCB0EE6A0A06900BA8FAF732FCFE
:10640000B0EE4A0A059008A8FAF72CFC0599069AFE
:10641000079B039002910192009352463B465946D6
:106420004046FCF799FFB0EE480A11A8FAF71AFCAB
:10643000B0EE690A83460EA8FAF714FCB0EE490ADA
:1064400006900BA8FAF70EFCB0EE680A059008A8B3
:10645000FAF708FC069B059A0390CDE900B3029277
:106460003B465246002140460137FCF72DFF082FDE
:1064700004F1100405F110057FF47BAF15B0BDECFD
:10648000088BBDE8F08F0021A1E700BFF2EC070800
:106490002DE9F14FDFF890B106460D462846FEF78C
:1064A00051FC074638B1002358491A46012001B073
:1064B000BDE8F04F50E7564905222846FBF70CFB94
:1064C00060B9524B00221A601A611A621A631A6488
:1064D0001A651A661A6701B0BDE8F08F04225946A2
:1064E0002846FBF7F9FA04462846002C42D1FAF771
:1064F0003BFC07460028EED054F000FCDFF82CA14E
:106500005FFA80F85AF8049BB9F1000F07D14149AE
:106510002A46304601B0BDE8F04FFDF767BD424660
:1065200049463846FBF7D8FA013484460028E9D1B9
:10653000364A0346154600210133082B42F8101B4A
:10654000FAD1354B03EBC40257682FB93348344DA9
:106550004946FCF779FFA1E713F834E0F445F5DA92
:1065600007EB0C130FCB05EB0C1484E80F000CF1B8
:10657000010CF3E7FBF78CFB072804463DD82846BF
:10658000FAF7F2FB074658B3FAF7E6F81F4B03EBAE
:10659000041383ED000A01253846FAF7E5FB0746A8
:1065A00038B1FAF7D9F8194B03EB041383ED010A5C
:1065B00001353846FAF7D8FB074638B1FAF7CCF878
:1065C000124B03EB041383ED020A01353846FAF748
:1065D000CBFB38B9304601B0BDE8F04FFDF75ABDEE
:1065E0000546D9E7FAF7B8F8084B032D03EB041377
:1065F00083ED030A3FF457AFECE70A4907233A4615
:10660000304601B0BDE8F04FFDF71ABE84430020CC
:106610007EE90708A4E6070834EC06080BED070836
:106620005DEA0708ACEC070806ED07080406070852
:106630002DE9F74F92460C461A4600218146FEF797
:10664000DFFADFF870B0804656460025BAF1000F39
:106650002ED031460422204656F088FE00284246BD
:1066600014BF0121002148460CBF01270027FEF777
:10667000C7FA738801933AF82530009380462B4679
:106680005A4639464846FCF767FE6388019334F85A
:10669000043B00935A462B46394648460135FCF7E1
:1066A00013FE042D06F10406D0D103B0BDE8F08F2F
:1066B0005746EAE715ED07082DE9F3410546084678
:1066C000FEF740FB0C46074638B1002333491A4613
:1066D000012002B0BDE8F041AAE731492046F9F7B0
:1066E00099FF70B92D4B04224FF47A704FF4FA6180
:1066F000013A1880598003F10403F9D102B0BDE8D2
:10670000F0812046FBF7C4FA0328064641D820460C
:10671000FAF72AFB074698B1FBF7BAFA4FF00108DF
:1067200004463846FAF720FB20B1FBF7B1FAB8F17E
:10673000000F09D1284602B0BDE8F041FDF7AABC20
:1067400040F2EE248046ECE7A4F2EE2240F2DC5365
:106750009A4203D8A0F2EE229A420AD9114940F691
:10676000CA0340F2EE22284602B0BDE8F041FDF730
:1067700067BD0D4B0D4A03EB86030021A3F8E842E9
:10678000A3F8EA02CDE9004033460846FCF79CFD39
:10679000B4E7074903233A46E5E700BF50BC0020B1
:1067A0007EE9070826ED070868B9002015ED0708FF
:1067B00024E907082DE9F04F89468FB017460021DC
:1067C0001A460646FEF71CFADFF874A005460024B8
:1067D0000DF1240B59F82480CDF80880594602A801
:1067E0004EF07AFA57B357F82430039398452A4667
:1067F00014BF0121002130460CBF4FF001084FF0BB
:106800000008FEF7FDF904A9054603A84EF064FA56
:1068100004A900912346524641463046FCF79CFDB0
:106820002346CDF800B05246414630460134FCF7CD
:106830004BFD202CCED10FB0BDE8F08FB846EFE76E
:1068400034ED0708F0B5074689B00846FEF77AFA36
:106850000E46054638B1002319491A46012009B0F1
:10686000BDE8F040A6E70846FBF712FA1F280446E9
:106870001DD83046FAF778FA014620463CF080FAF7
:1068800078B10F4803AE314600EB84004EF024FA95
:106890000C4A0096234629462846FCF715FD09B008
:1068A000F0BD384609B0BDE8F040FDF7B5BB06497C
:1068B0001F232A46384609B0BDE8F040FDF7C0BCAA
:1068C00060BC002034ED0708ACEC07082DE9F04F60
:1068D000924685B00C461A4600218146FEF790F993
:1068E000DFF874B0804655460026BAF1000F31D06B
:1068F00029460422204656F039FD0028424614BF9E
:106900000121002148460CBF01270027FEF778F936
:10691000EB780293AB7801932B8800938046334643
:106920005A4639464846FCF717FDE3780293A378A8
:10693000019334F8043B00935A463346394648469F
:106940000136FCF7C1FC102E05F10405CDD105B0D0
:10695000BDE8F08F5746E8E73EED0708F0B507467B
:1069600085B00846FEF7EEF90E46054638B100231D
:106970001C491A46012005B0BDE8F040A6E70846CC
:10698000FBF786F90F28044623DC3046FAF7ECF9CA
:10699000014620463CF0DAFAA8B1134B04F120027C
:1069A00003EB8203294693F8FB22029293F8FA2222
:1069B0000192B3F8F83200930C4A23462846FCF7BC
:1069C00083FC05B0F0BD384605B0BDE8F040FDF7EA
:1069D00023BB07490F232A46384605B0BDE8F040DF
:1069E000FDF72EBCE0BC002068B900203EED070892
:1069F000ACEC07082DE9F04F85B0144602911A4619
:106A000000210546FEF7FCF84FF000080646062375
:106A100003FB08F7C0374FF00009029B13F807B0DB
:106A2000002C7ED0E35D03939B45324614BF0121C9
:106A3000002128460CBF4FF0010A4FF0000AFEF774
:106A4000DFF8039B394ACDE9009306464346514699
:106A50002846FCF781FCCDE9009B344A4346514669
:106A6000284609F10109FCF72FFCB9F1060F07F1DF
:106A70000107D2D108F10108B8F1060FC7D1E42708
:106A8000029BA7F1E40913F807A0002C4BD014F8DF
:106A900007B0DA45324614BF0121002128460CBF59
:106AA0004FF001084FF00008FEF7AAF8CDE9009B6F
:106AB00006461E4A062341462846FCF74DFCCDE912
:106AC000009A1A4A0623414628460137FCF7FCFB88
:106AD000EF2FD5D1029B93F8EF70B4B194F8EF800B
:106AE0004745324614BF0121002128460CBF01242E
:106AF0000024FEF785F8002300930C4ACDF80480AB
:106B0000072321462846FCF727FC00230093074A69
:106B10000197072321462846FCF7D6FB05B0BDE8C0
:106B2000F08FA24697E7A046C9E700BF50ED0708DF
:106B3000F0B5054685B00846FEF704F90B46044655
:106B400038B100231B491A46012005B0BDE8F040CA
:106B500050E71949184F6A46184656F066FB01AED1
:106B600088B1032C04D12846FDF794FA05B0F0BD96
:106B7000FBF78EF86A4646F8040B394600200134CC
:106B800056F053FBECE7032CEDD1DDE90146039F02
:106B900031463A46E0B23CF015FA18B92846FDF7FE
:106BA0003BFAE3E705483B4632462146FCF74CFCFE
:106BB000DCE700BF60BC0020D5ED070850ED0708FA
:106BC0002DE9F04F0E46154689B01A4600210446BD
:106BD000FEF716F8B04681462F464FF0000B002D09
:106BE0007CD039460C22404656F0C0FB00284A466D
:106BF00014BF0121002120460CBF4FF0010A4FF0C5
:106C0000000AFDF7FDFF97F90B20049297F90A207F
:106C10000392B7F908200292B7F906200192B7F95A
:106C2000042000928146384A5B4651462046FCF7D4
:106C300093FB98F90B20049298F90A200392B8F973
:106C400008200292B8F906200192B8F904200092B7
:106C50005B462D4A514620460BF1010BFCF734FBF5
:106C6000BBF1080F08F10C0807F10C07B7D1DFF8EA
:106C70009C804FF0000B0C2303FB0BF985B300271E
:106C800055F8090056F80920012303FA07FA424093
:106C90003AEA020214BF1946002110EA0A0F07D08F
:106CA00000975B46424620460791FCF755FB079943
:106CB00056F809201AEA020F05D000975B464246B3
:106CC0002046FCF701FB01370E2FD9D10BF1010B48
:106CD000BBF1080FCFD109B0BDE8F08FAA46A8E7F5
:106CE0002F4656F80910012303FA07F20A4206D08C
:106CF00000975B46424601212046FCF7E5FA013742
:106D00000E2FEED1E2E700BF64ED07087CED070827
:106D1000F0B506468BB00846FEF714F80D4604465B
:106D200020B300233D491A4601200BB0BDE8F040D6
:106D300046E72D2903D0A1F13003092B49D8052CB2
:106D400005DD30460BB0BDE8F040FDF7A3B928469D
:106D5000FAF79EFF0AAB621C03EB440424F80C0C08
:106D600015F8013F303B092BFAD914462978002940
:106D7000DFD1062CE5D1BDF81C20BDF91C30072A57
:106D8000DFD8BDF91E50A5F5FA7292B2B2F5FA6FCE
:106D900018D8BDF92070A7F5FA7292B2B2F5FA6F61
:106DA00010D8BDF922C065450CDC67450ADBBDF98A
:106DB00024E00EF1640292B2C82A03D8BDF926403D
:106DC000112C11DD164930460BB0BDE8F040FDF73F
:106DD0000DB9202902D101352246C6E730460BB055
:106DE000BDE8F040FDF718B90E4A0C2000FB032265
:106DF00064B2A2F8EC53A2F8EE73A2F8F0C382F8E2
:106E0000F2E382F8F3430846CDE903E4CDE9017CDF
:106E1000054A0095FCF758FA0BB0F0BD50BD0020B4
:106E200091ED070868B9002064ED07082DE9F04FDF
:106E300089468DB0164600211A460746FDF7E0FE4A
:106E4000DFF8DCA005460024C4EBC40309EB030211
:106E500059F8030091889279089040F30748ADF8FB
:106E600024108DF82620B8F1000F54D0002E55D0F4
:106E7000F218F058918893790A90ADF82C100722F7
:106E80000AA908A88DF82E3056F070FA00282A4674
:106E900014BF0121002138460CBF4FF0010B4FF009
:106EA000000BFDF7ADFE9DF82E3006939DF92D30B9
:106EB00005939DF92C3004939DF82B3003939DF995
:106EC0002A3002939DF8293001939DF828300093D1
:106ED00005462346524659463846FCF73DFA9DF88A
:106EE000263006939DF9253005939DF924300493AF
:106EF0009DF82330CDE902839DF8213001939DF860
:106F00002030009352462346594638460134FCF758
:106F1000DBF9102C98D10DB0BDE8F08FB346DEE759
:106F2000A7ED07082DE9F04FDFF8A4828BB00646E5
:106F30000D46284653F0E2FE034630B99649024614
:106F400001200BB0BDE8F04F70E7944905222846B8
:106F5000FAF7C2FD0446C8B9914D0146702205F505
:106F6000896056F07FF9C5F8E843C5F8F443C5F8E1
:106F70000044C5F80C44C5F81844C5F82444C5F8C5
:106F80003044C5F83C440BB0BDE8F08F04224146C4
:106F90002846FAF7A1FD044630BB2846F9F7E4FE7F
:106FA00081460028EFD053F0A9FEDFF828B28246D0
:106FB0005BF8047B3FB97B492A4630460BB0BDE8FD
:106FC000F04FFDF713B8524639464846FAF784FDAC
:106FD00040B920462AF092F97348744D3946FCF7BF
:106FE00033FAA6E70134E3E7714907222846FAF7A6
:106FF00073FD074600287AD12021284656F049F92A
:10700000044670BB6B486C4DFCF7BEF92146284620
:107010000134FCF7B9F90E2CF8D1FCF751F9DFF87F
:10702000B891664FDFF8B481002529464846FCF741
:10703000ABF90C26DFF8A8A16E430024F259604892
:107040000123A34013420CBF414651460134FCF7D3
:107050009BF90E2CF2D10135FCF732F9082DE4D161
:1070600091E75849574D01AA56F0DFF802AC0028C5
:1070700048D0022F11D1029A072A07D8039C0D2C61
:1070800004D80378722B13D06E2B25D04E490823D9
:1070900000223046FDF7D4F875E7FAF7F9FD01AAAA
:1070A00044F8040B29460020013756F0BEF8DEE70D
:1070B0003B490C2303FB02110123D1F8E813A34041
:1070C0000B4337490C2000FB02123949C2F8E83360
:1070D0003046FFF727FF56E7314B0C2000FB023309
:1070E0000121D3F8E833A14023EA0103E9E7284668
:1070F0003449344F01AA56F098F802AD002480B10B
:10710000082C03D13046FCF7C5FF3CE7FAF7C0FD79
:1071100001AA45F8040B39460020013456F085F8E1
:10712000EDE7082CEED1029B0F2B30D8DDF80CE0F8
:10713000BEF1070F2BD8DDF810C0BCF10D0F26D81B
:10714000059F07F16402C82A21D8069DFF2D1ED88D
:10715000079864281BD80899642918D8884216DA39
:10716000099C032C13D8C3EBC3020D4B134483F8C3
:107170004D1483F848E40D4983F849C483F84A74F0
:1071800083F84B5483F84C0483F84E44A0E70F492E
:107190003046FCF72BFFF6E6B0BD00207EE907087D
:1071A00068B90020A4E607080BED07085DEA0708A8
:1071B000C4ED07088FF60708CCED070850BD002086
:1071C000D1ED0708D5ED0708D7ED070891ED0708C1
:1071D00006ED070804060708CEFF0708E7F40708CE
:1071E0008FED07082DE9F04F924689B00C461A46FC
:1071F00000210746FDF704FD002607905546B346DB
:107200004FF019094FF46178BAF1000F28D02946E0
:107210000622204656F0AAF80028079A14BF01213A
:10722000002138460CBF4FF0010B4FF0000BFDF76B
:10723000E7FC6A79079019FB028205922A7919FB0B
:1072400002820492EA780392AA7802926A78019202
:107250002A7800923346124A59463846FCF77CF8A1
:10726000627919FB02820592227919FB028204924B
:10727000E2780392A27802926278019214F8062BC7
:1072800000923346064A594638460136FCF71CF848
:107290000A2E05F10605B7D109B0BDE8F08F00BF91
:1072A000DDED07082DE9F04F074689B00846FDF7E8
:1072B00049FD8B46054638B100234C491A4601204A
:1072C00009B0BDE8F04F8DE7494B084693F878A622
:1072D00093F8799693F86287FAF7DAFC092804465E
:1072E0007BDC062646430BF101008DF81F50F9F7B1
:1072F0003BFD3E4D834638B1FAF7CAFC0D2803D852
:107300000123A8558DF81F305846F9F72DFD834607
:1073100060B1FAF7BDFC504508D8062303FB0453BF
:1073200058709DF81F3001338DF81F305846F9F71B
:107330001BFD824660B1FAF7ABFC484508D806232E
:1073400003FB045398709DF81F3001338DF81F30F4
:107350005046F9F709FD814660B1FAF799FC80457E
:1073600008D3062303FB0453D8709DF81F30013364
:107370008DF81F30311D0DF11F0229444846FAF7E0
:107380008BFC9DF81F30062B09D0AA190023384624
:10739000AB51938009B0BDE8F04FFCF77BBE63436F
:1073A000EA184FF461765079192111FB00600590BD
:1073B000107911FB00610491D178039191780291C9
:1073C00052780192EB5C009300210A4A234608465A
:1073D000FBF77AFF09B0BDE8F08F074909232A4679
:1073E000384609B0BDE8F04FFCF72ABFA0450020A1
:1073F00070A80020DDED0708ACEC07082DE9F04F80
:107400000F468BB0144600211A460646FDF7F8FBDE
:107410000546002C00F0DD8022783B789A4218BFA8
:107420000121024608BF002130460CBF4FF0010881
:107430004FF00008FDF7E4FB23789E4A05464146DD
:107440003046FBF789FF3B789A4A41463046FBF7C6
:107450003BFF002C00F0BF8062787B789A4218BF17
:1074600001212A4608BF002130460CBF4FF0010819
:107470004FF00008FDF7C4FB63788F4A054641468C
:107480003046FBF769FF7B788B4A41463046FBF775
:107490001BFF07F1C9030593A31C0693822307F181
:1074A000020A04F1CA0B07934FF000093B784B45E1
:1074B00000F39380002C00F0F68097F8EA3094F8FF
:1074C000EA209A4218BF01212A4608BF002130460F
:1074D0000CBF4FF001084FF00008FDF791FB94F846
:1074E000EA30764A054641463046FBF735FF97F8C5
:1074F000EA30724A41463046FBF7E6FE002C00F0C7
:10750000D48004F1EA0307F1EA0204F1FA014FF032
:10751000010833F802CF32F8020F844518BF4FF04C
:1075200000089942F5D188F001012A46C9B23046D7
:10753000FDF766FB0821054604F1EC00FAF71AFA9C
:107540005F4A034641463046FBF706FF97F8EA10CC
:1075500007F1EC00FAF70EFA594A03464146304665
:10756000FBF7B2FE002C00F0A2804FF0FC094FF0B8
:10757000010807EB090104EB0900F9F74BF809F1E1
:107580000409002818BF4FF00008B9F58E7FF0D12C
:1075900088F001012A46C9B23046FDF731FB0821C7
:1075A00004F1FC00F9F7F3FB464A03464146304636
:1075B000FBF7D2FE97F8EA1007F1FC00F9F7E7FBBA
:1075C000404A0346414630460BB0BDE8F04FFBF75A
:1075D0007BBEA04637E7A04655E7079BFB180993FB
:1075E000002C5ED0079B0998E31819460893F9F719
:1075F00011F8059B5A789BF800309A42069A06BF0C
:10760000B0FA80F84FEA58184FF00008AAF10203C8
:10761000023A0AF10E0133F802CF32F8020F844524
:1076200018BF4FF000088B42F5D188F001012A46BF
:10763000C9B23046FDF7E4FA6278069905469BF830
:107640001800FAF769F902909BF800300193089B43
:1076500000931D4A09F1010341463046FBF77CFEC9
:10766000059B7A78587E5146FAF756F9059A0290AA
:1076700012F8013F019309F10109099B059200935A
:10768000114A4B4641463046FBF71EFE069B10331F
:107690000693079B09330AF1100A0BF1010B0793BC
:1076A00004E7A046DCE7A04621E7A0464EE7A04657
:1076B00080E700BFF6ED070808EE070836EE07087A
:1076C0004EEE070865EE07081DEE07082DE9F04F9E
:1076D0008FB0044602AA0846B14955F0A6FD0546FA
:1076E00040B903460246AF494120FFF787FE0FB07D
:1076F000BDE8F08FAC49F8F78DFF064628BBA849D6
:1077000002AA55F092FDFAF7C3FA0828054606D9F1
:10771000A649082332462046FCF792FDE7E7A44C31
:1077200094F8783683420CDC84F87856DFE73146EB
:1077300038463AF085F9013694F87836B342F6DCEB
:10774000F2E7064604F5CF67F6E79A492846F8F7C8
:1077500061FF0646E0B9924902AA55F066FDFAF7C4
:1077600097FA0828054603D9934908233246D2E7F9
:107770008F4C94F87936834202DC84F87956B6E768
:107780003046294601364DF07FFA082EF8D1F4E74D
:107790008A492846F8F73EFF064600BB804902AA00
:1077A00055F043FD0028A2D0FAF772FA08280546E2
:1077B00003D9834908233246ADE77D4C94F86237FC
:1077C000834209DD014604F5CF603AF07DF9294690
:1077D00004F5CF603AF086F984F8625787E7794973
:1077E0002846F8F717FF064618BB714BDFF8B09133
:1077F00093F8627706AD01461022284655F032FD17
:10780000A846BE4202AA80F20A814946002055F0ED
:107810000CFD10B96C493A460AE1FAF739FA01361B
:1078200028F8020BEDE795E80F00684C84E80F009C
:107830005DE767492846F8F7EDFE0646C0BB5C4B9E
:10784000DFF85C9193F8627706ADBE4202AA80F23F
:10785000F3804946002055F0E8FC014610B95D4927
:107860003A46E5E00322284655F04BFDAA464FF084
:107870000008284653F042FA404502D80136043544
:10788000E3E79AF80000FAF721F908F101080AF88D
:10789000010BEEE7504DB6000446B4423FF427AF6B
:1078A00006AB1919281903223AF0B4F80434F4E7A6
:1078B0004A492846F8F7AEFE0746002840F0AC805B
:1078C000DFF8EC80364998F8786602AA55F0ADFCEE
:1078D00000283FF40CAFFAF7DBF9451E01D4AE42A5
:1078E00003DC3F493346012215E72D4902AA002057
:1078F00055F09BFC014600283FF4F9AE0026082213
:1079000003A88DF8146055F0FCFC0DF10C0903A8D8
:1079100053F0F4F9B0421BD8214902AA002055F0D7
:1079200084FC00283FF4E3AE037898F879A601932D
:107930000026B14656451A4902AA4FF0000080F2CF
:10794000858055F072FC834650B9264952466FE057
:1079500099F80000FAF7BAF8013609F8010BD6E7F2
:10796000A6B99BF80030303B092B0FD91E49F8F718
:1079700051FE38B11D495846F8F74CFE70B11C490C
:107980005A4655E04FF001094FF0FF365846FAF7D6
:107990007FF9002830DA17495A4649E0B146F3E743
:1079A000D5ED0708E8AE00207CEE070882EE070858
:1079B00070A800208DEE070896EE0708A4EE0708D1
:1079C000B0EE0708C2EE0708B1EF0708D4AF0020F9
:1079D000ECEE0708D1EF0708E4AF002016EF070828
:1079E0001BEF0708F1EF070824DE070827EF070859
:1079F0002EEF070863EF07080EAB03EB46030136D3
:107A000023F8200C96E72049524611E033F8022B68
:107A100024F8022F013730E01C492A4608E01C49AF
:107A2000002055F002FC00283FF4FDAE19493A460B
:107A30002046FCF7DBFA5AE61549002055F0F5FB25
:107A400000283FF427AF14493A46F1E755F0EDFB23
:107A50000028D8D1114C05EBC50082302044082203
:107A600003A939F0D7FF0198FAF730F808EB0503BE
:107A700004EB051483F8420706ABBE42C6DC45445E
:107A800085F85A9733E600BF78EF07089BEF0708A1
:107A9000D5ED0708CEEE0708F8EE0708E8AE00209F
:107AA0002DE9F04F89B00F4690460021139A0393B9
:107AB0000646FDF7A5F887EA08086FEA0803DFF82D
:107AC000849006930446002528460AF069FC129B20
:107AD000184230D0069BDFF870B0034014BF4FF05F
:107AE000010A4FF0000A049310EA07030CBF4A464C
:107AF0005A462846059307920AF064FC039B079AAE
:107B00000090804651463046FBF726FC049BB3FAB2
:107B100083F1224649093046FDF772F8059A039B26
:107B2000CDF800800446002A0CBF5A464A4651460A
:107B30003046FBF7C9FB0135182DC5D109B0BDE8AA
:107B4000F08F00BF16F0070800ED070870B5044677
:107B500008460E4653F0D2F8314605460246204606
:107B6000F9F7BAFF68B9635D1846F9F79FFF00B9E6
:107B700033B901352C44204601340378202BFAD048
:107B800070BD0020FCE708B504460948FBF790FBF0
:107B9000FBF772FB074BD3F82C010AF0CFFC06F081
:107BA000DFF8012C01D150F09FFFF4F7F7FF00BF81
:107BB0001DF0070868B9002010B5044608460B46BA
:107BC000FDF7C0F828B9094903221846F9F784FFE0
:107BD00028B90748FBF792FB0120FFF7D4FF2046A6
:107BE0000449BDE81040FCF701BA00BF29F00708BE
:107BF0002DF00708CFE807082DE9F74F064601AA40
:107C000008462E49DFF8C480DFF8C490DFF8ACA046
:107C100055F00BFB4FF0000B04465D46012714BBEB
:107C2000BBF1000F27D1264C002D43D02548294613
:107C3000FBF70AFC23790BB904F0F4FFF9F7D2F94A
:107C4000002384F87530FBF7EDFA15B12846FCF7F0
:107C5000E4FF9FB13046FCF79BFF78B1FBF730F9AA
:107C60000020FFF790FFBBF1000F0AD02046FAF783
:107C70000FF885B2C5B93046FCF7CEF903B0BDE8C0
:107C8000F08F41462046F9F74BFF80B94946204620
:107C9000F9F746FF0028EED05F4601AA51460020C2
:107CA00055F0C3FA0446BAE74FF0000BF5E74FF082
:107CB000010BF2E70448FBF721FBBFE7D5ED07080E
:107CC00070A8002058F007087BF007084FF007085D
:107CD00073F7070810B50C46FCF75AFF78B1084B4C
:107CE00001229A73FBF7ECF80648FBF707FB0649FD
:107CF0002046F8F78FFC10B10020FFF744FF10BDBD
:107D0000B842002091F0070844DE0708F0B50329C7
:107D100085B005460C46164614D80B4F3970FBF754
:107D2000CFFA0A492846FDF7EFFC0949224601A887
:107D3000F9F79AFD01AB324608212846FCF78EFF81
:107D4000FF233B7005B0F0BDB80500205DEA0708D1
:107D5000FCEB0708F0B5032985B005460C4616462E
:107D600014D80B4F7970FBF7ABFA0A492846FDF798
:107D7000FBFC094922466846F9F776FD6B46324618
:107D800010212846FCF76AFFFF237B7005B0F0BD89
:107D9000B80500205DEA0708F8EB070810B586B0C3
:107DA0000E4B04930E4B03930E4B02930E4B019319
:107DB0000E4B0F4A0F49009304460F4B0F48FBF739
:107DC000E3FAFBF77DFA3CB10D4A0E490E4806B0C6
:107DD000BDE81040FBF738BB06B010BDD8F007086F
:107DE000DDF00708E7F00708F0F00708FCF00708E7
:107DF00098F00708A2F00708BF420020ADF007087E
:107E0000006B0708FC6A070802F107080120C5E7B4
:107E10002DE9F04F0A4689B000210546FCF7F0FE37
:107E2000394C0590394A2378608802EB8303D3F8F4
:107E3000C491F8F777FA364BD0F808B01F7917B12C
:107E40005F46D0F80CB0A379012B38BF012306930D
:107E500000262279637906FB02331BF80380002F8A
:107E60003BD0FB5C059A0793434514BF01210021D9
:107E700028460CBF4FF0010A4FF0000AFCF7C0FE85
:107E8000079B0590013653B303F00F021B094033E3
:107E9000CDE9006302924B461E4A51462846FBF745
:107EA0005BFAB8F1000F24D008F00F034FEA18185E
:107EB000029308F14003CDE90063164A4B46514650
:107EC0002846FBF701FA069BB342C2DC124B08348A
:107ED000A342A7D109B0BDE8F08F3B46C2E7002F0F
:107EE000DFD00E4A00964B4651462846FBF734FA3F
:107EF000D7E76B06E7D4094A00964B465146284619
:107F0000FBF7E2F9DFE700BF00010708C8FD06083C
:107F100070A800202FF107085802070845F107084C
:107F20002DE9F04F0A468DB000218346FCF768FE2C
:107F3000704CDFF8CC91039004F1800A0025A37AFD
:107F400099F80460AB4200F3938010345445F5D1A6
:107F500040F21620F8F7E6F9D0E902450DF1180ACB
:107F6000002E4FF015024FF00001504604BF254689
:107F7000344655F077F900272E78002E3ED06978E8
:107F80000591304606F050FB95F90290049009F1F6
:107F9000010253425341002C00F0A98005990022B0
:107FA000A05CB04240F09F80224492F90280C1451B
:107FB00040F0978052788A4208BF012301220AF8D4
:107FC000072003F0010383F00101039A059358464B
:107FD000FCF716FE059B039044B1474A0499CDE98E
:107FE00000B230464246F8F74BFF059B434A0499DE
:107FF000CDE900B230464A46F8F742FF0137152F67
:1080000005F10305B8D184B3DFF8EC80DFF8EC901C
:10801000564604F13F0716F801ABBAF1000F21D123
:108020002078F8B194F9023001331BD0617806F062
:10803000FBFA039A054601215846FCF7E1FD94F945
:1080400002200390534620782946CDE900B8F8F77E
:1080500017FF20785346CDE900B94FF0FF3229468B
:10806000F8F70EFF0334BC42D5D10DB0BDE8F08F58
:10807000E088F8F757F9D0E90231627A207A002EC9
:1080800008BF194605FB002208BF33468F562BB3A5
:108090009E56039A0493B74214BF0121002158460B
:1080A0000CBF4FF001084FF00008FCF7A9FD049B3E
:1080B000039043B1104B3246CDE900B32946434605
:1080C0002046F8F793FE0D4B2946CDE900B33A461A
:1080D00043462046F8F78AFE013530E74FF0FF3679
:1080E000D7E700236AE703323F2A7FF459AF4FF006
:1080F000FF3868E7D005002059330108C93201086C
:1081000070A800202DE9F04F80468BB008460D4640
:1081100052F0F4FD024678B3A4492846F9F7DCFC96
:10812000044648BBFBF7CCF8A148A24DA24FA34E92
:10813000DFF8D482FBF7DCF814204CF0B9FDE11035
:1081400004F0070201313846FBF71EF92B7F6A7FE6
:1081500006EB8303D3F8C41152B19948FBF774F9C5
:108160000134102C05F12405E9D10BB0BDE8F08FE6
:108170004046FBF769F9F3E72846924905AA55F00E
:1081800054F8054620B901464120FFF7C9FEECE747
:108190008D49F8F73FFA20B98C494046FBF726FF96
:1081A000E3E78B4E0827002431682846F8F732FAB7
:1081B000002808BF3446013F06F11006F4D154B937
:1081C00084492846F8F726FA28B183492A464046CA
:1081D000FBF70CFFC9E700207A498DF8130005AAC8
:1081E00055F023F80646002C39D078B1F9F750FD48
:1081F000451E08D4A37A9D4205DAE26842B1012304
:108200008340134204D175493246E0E7744EFAE7E1
:10821000E088F8F787F87349D0E902230979002943
:1082200018BF1A46217A637A05FB0133002712F939
:1082300003A0039702EB030B624905AA002054F048
:10824000F4FF8146A0BB6849012344B39BF9002099
:108250002046CDE900312946F8F7C8FD85E768B129
:108260000DF11301F9F7EEFC28B19DF813502846E3
:1082700005F0ECFC20B95D493246A8E7584EFAE714
:108280002846F3F759FA8246284606F0B9F90390D2
:10829000284606F0F1F9A34607462546CCE7CDE986
:1082A00000319DF8130052463946F8F7E9FD5CE7C6
:1082B0004549F8F7AFF9064658BBACB14C4FEDB2A3
:1082C000207972B22946F3F711FA00283FF44DAF36
:1082D0000288037800933146C2F303233846120B19
:1082E000FBF7B2F80136EBE7414C7979386872B2A6
:1082F000F3F73EFA00283FF438AF02880378009382
:108300003146C2F303232046120BFBF79DF80136DA
:10831000EBE738494846F8F77DF910B34846F9F7D6
:10832000B7FC064642B26CB12079E9B2F3F7DEF948
:10833000C8B9CDF8009022682F496B1C4046FBF766
:1083400055FE12E779793868F3F712FA58B99DF8B3
:1083500013302A49CDF800901A09403203F00F0378
:10836000ECE74FF0FF3606AF39463046F9F736FBFB
:1083700008A95046F9F732FB564547D076B24CB1C2
:108380008BF80060009721681D4808AB6A1CFBF75A
:108390005BF8EAE69DF81320039B1A489E701109CA
:1083A000009708AB02F00F024031F0E759F10708DF
:1083B0005EF10708B802002074F10708C8FD06083E
:1083C000E3F20708D5ED0708FEE2070885F1070884
:1083D000D0050020B5F4070899F10708A8F10708AF
:1083E0005DEA070870A80020C9320108B8F1070843
:1083F000CAF10708C1E60708EBF107080EF2070803
:1084000036F2070859F2070875E2070834B1216807
:10841000074808AB6A1CFBF717F8A6E69DF813207F
:108420000448110908AB02F00F024031F3E700BF26
:1084300081F207089CF207082DE9F04F07468BB040
:1084400040F216200C46F7F76DFF22460546002144
:108450003846FCF7D5FB424BD5E902451B79002B8A
:1084600008BF254606464FF015024FF0000104A84C
:1084700008BF1C4654F0F6FE05F13F03039395F840
:108480000090B9F1000F31D095F801A0002C65D013
:10849000224600231178494558D128336B4492F87D
:1084A0000180012203F8182CD045324614BF012167
:1084B000002138460CBF4FF0010B4FF0000BFCF7CA
:1084C0009FFB064654B1B8F1000F07D0254B00932F
:1084D0005A463B4641464846F8F718FD224B009362
:1084E0005A463B4651464846F8F710FD039B033574
:1084F0009D42C4D13CB3DFF86C90DFF86CA0651CE2
:108500000DF11008403418F8013BCBB915F8013CC7
:10851000B3B116B13046FAF7F1FE297815F8010C1F
:10852000CDF800903B460022F8F7F0FC002215F849
:10853000010CCDF800A03B461146F8F7E7FC0026F9
:108540000335A542DFD10BB0BDE8F08F0133152B09
:1085500002F103029ED14FF00008A5E7A046A3E771
:1085600070A8002059330108C93201082DE9F04FE5
:1085700007468DB008460D4652F0C0FB044628B9A8
:10858000014601200DB0BDE8F04F55E70246A8496D
:108590002846F9F7A1FA30B9A64938460DB0BDE82A
:1085A000F04FFBF723BDA44922462846F9F794FA79
:1085B000002859D1FAF784FEA048A14FDFF8C092F5
:1085C000DFF8C082FAF794FE17204CF071FB0E25FD
:1085D00017F9016B002E38D031464846FAF7D4FE21
:1085E00000231C46A10089B23046039306F07EF8B2
:1085F000834606F007F90278039B82460134D2B124
:108600000BB9FAF75DFE9BF806109AF800309AF85D
:10861000012001F0020108EB8303CAB189480092EE
:10862000894AD3F8C431002908BF02468748214649
:10863000FAF70AFF0123042CD4D113B98448FAF7BE
:1086400057FE013D15F0FF05C2D10DB0BDE8F08F1A
:108650007C487D4AD3F8C431002908BF02467D48D2
:108660002146FAF7F1FEE5E7002476498DF81B4034
:1086700007AA284654F0D9FD18B93846FBF7CCFCB8
:10868000E3E70DF11B01F9F7DDFA81460028F4D08C
:108690009DF81B50284605F0D9FA20B96E49384696
:1086A000FBF7A4FCD1E7DFF8E08123464FF0FF346D
:1086B00003EB430218F8022095420BD0002C02DA9B
:1086C000002A08BF1C460133152BF1D1002C16DA05
:1086D0006249E4E71C465B4907AA002054F0A5FD67
:1086E0000646002800F096805149F7F793FF30BB0B
:1086F0005B4FDFF85481DFF89491044616E04FF0A9
:108700000009E8E7306896F807A0F3F741FBB17974
:10871000737911F0020F0CBF394641469B0802469F
:108720000091013351464846FAF78EFE0134214646
:10873000284605F079FF06460028E3D185E7494938
:1087400002223046F9F7C8F94FEA151A0AF1400A31
:1087500005F00F0B002845D10390B01CF9F798FAEB
:10876000039902460491284601310592039105F0D0
:108770005BFFDDE90313059A38B93B4900965B4678
:1087800052463846FBF732FC5FE7C0799042E9D1A8
:108790001F466300B9F1000F31D01A1942445678D0
:1087A000013E7A1C234414BF2946002108EB030232
:1087B00008F803107B1C53700AACFF2393703946F2
:1087C00022462846F9F71AF908AA31462846F9F749
:1087D00015F9B74216D1254808AB5A465146FAF763
:1087E00033FE32E722493046F7F714FF20B1214922
:1087F00000965B465246C4E74FF0FF37C9E74FF09B
:10880000FF36CEE71C48009408AB5A465146FAF7AB
:108810001BFE1AE704EB4404184B0093A0440246E5
:1088200098F8011001232846F8F770FB0DE700BF08
:10883000FEE2070885F1070859F10708B8F20708B2
:10884000EC6A0708D5ED07082CDF0708D8F20708FF
:10885000F9F20708EAF20708FFF2070816F307081B
:108860005DEA07083FF3070842F3070894F3070897
:10887000C1E607086EF30708B2F30708C93201081A
:10888000D1F20708C8FD06086C2800202AF3070863
:108890002DE9F04F89B0074605AA08469D4954F0D6
:1088A000C4FC054630B901464120FFF7B1FA09B0D2
:1088B000BDE8F08F9849DFF8A882F7F7ABFE0446D1
:1088C00000283CD19548964D964EDFF89892FAF7DD
:1088D0000FFD14204CF0ECF92968AB79AA8801F15E
:1088E0003F4108EB830301F57E01B2FA82F2890A67
:1088F0004131D3F8C431C2F11F023046FAF744FDCA
:10890000E97911B14846FAF73FFD0134FAF7D8FC8E
:10891000602C05F10805DFD17E4905AA002054F03E
:1089200084FC8149F7F776FE0028C0D138467A49A1
:10893000FFF71CFE78493846FFF7E4FBB7E7002451
:1089400008F54E7A1AF8343008EB83032846D3F83A
:10895000C4914946F7F75EFE40B101342B2CF1D1AA
:1089600072492A463846FBF741FBA0E7694905AA48
:1089700054F05BFC064688B3F9F78AF9054608EB24
:10898000C4084FEAC40B98F83E334BBB002D29DCDA
:108990000AEB0B03588893F804A093F80580F7F7C7
:1089A000C1FCEBB203FB0A880093D0F808A0002EAC
:1089B00000F09A803378002B00F0968006A93046AC
:1089C000F9F740F9002800F08C809DF8185005BB9D
:1089D0000AF808505648FAF78BFC68E70546CEE7D8
:1089E000002D05DD012B1A4638BF0122954208DD16
:1089F000012B504938BF012301223846FBF720FCE8
:108A000055E7444905AA002054F00FFC013D0646F5
:108A1000BEE7284605F01AF9814600285DD02B09EB
:108A200040330293444F0AF8085005F00F034FF00B
:108A300000080393BB79012B38BF01230193002663
:108A4000788897F804B097F805A0F7F76BFC06FB59
:108A50000BA38268D15CA94222D1444504D100997C
:108A6000B1421DD00021D154DDE9021233485FFA32
:108A700086FB5FFA88FAFAF787FC59465046FAF700
:108A8000C5FC444509D12E48FAF77EFC50465946AC
:108A9000FAF7BCFC2B48FAF777FC2B48FAF728FCCE
:108AA000019B0136B342CBDC08F10108B8F12B0F72
:108AB00007F10807BED1D9F80010B9F804202348FF
:108AC00001F13F4101F57E01B2FA82F2890AC2F159
:108AD0001F024131FAF7B8FCE9E63846FBF79CFA89
:108AE000E5E61B4932463DE71AF80830013573B117
:108AF0001A09184903F00F03403206A8F8F7B4FE2C
:108B000006AB15482A464946FAF79EFCCFE6134BBA
:108B1000F7E700BFD5ED070859F10708D8F30708B4
:108B20003023002016F4070821F4070825F407086D
:108B300041F40708ACEC07080001070853F40708E4
:108B4000A7DE070877F4070826F9070881F4070865
:108B50009DF407083EF10708B9F4070878DD070817
:108B6000C8FD0608CDFF0708224BB0F5FA6F1A685A
:108B70000346A8BF4FF4FA63B3F57A7FB8BF4FF44A
:108B80007A73D20416D540F2DC52904215D007EE2B
:108B9000903A40F2DB529042F8EE677A1FD8DFED50
:108BA000166A9FED167A9FED160A77EEE67AA7EE23
:108BB000870A7047B0F57A7F02D89FED120A704796
:108BC00007EE903ADFED106A9FED107A9FED100AE4
:108BD000F8EE677A77EEE67AA7EE870A7047DFED60
:108BE0000D6A9FED0D7A9FED0D0A77EEE67AA7EEFE
:108BF000870A7047CC42002000007A44D62000C08B
:108C000000E082440000000000407A44661000400A
:108C10000000404200A0BB44D62000400000834436
:108C200010B584464FEA810E102312F4004F14BF92
:108C30000E2407245200013BCCF8004092B2F444C9
:108C4000F3D100EB81128C01035142F82130122044
:108C500010BD00BF10B584464FEA810E0424130BEB
:108C600003EB430318331201013CCCF8003092B2FD
:108C7000F444F4D100EB01130A01845043F821407D
:108C8000062010BD704700BF704700BF034B00EBCC
:108C9000400003EBC003587C704700BF480500103C
:108CA00043F63F6303607047704700BF0020704782
:108CB000704700BF0020704701207047704700BF19
:108CC000704700BF704700BF704700BF9FED010AAB
:108CD000704700BF000000000020704703681B6958
:108CE000184700BF2DE9F047DFF870A0BAF8003050
:108CF00004330F469DB201F10908012417F8011B46
:108D0000AC464FF0000E04FA0EF2ACF104030A4038
:108D10009BB219D100EB830901339BB29C45C9F882
:108D20001420F7D10EF1010E0CF1040CBEF1080F66
:108D30001FFA8CFCE7D120354745ADB2DED10023C8
:108D4000AAF80030BDE8F087868900EB8302013382
:108D50009BB263455661F8D1E4E700BF54C90020D7
:108D60002DE9F047DFF87CA0BAF802300B338846D3
:108D70001FFA83FE01F106090024012618F801CB31
:108D800071460025A1F10B039BB23DB1092D20D006
:108D90006A1E06FA02F212EA0C0F1AD0878900EB5B
:108DA000830201339BB299425761F8D10B1D00EB4E
:108DB000830301350C310A2D5C6089B2E2D10EF1DA
:108DC000780EC8451FFA8EFED8D1AAF80240BDE839
:108DD000F0871A1D013300EB82029BB28B42546074
:108DE000F7D1E3E754C900202DE9F0410E78057B67
:108DF000F6430446F6B200F1100300F1380243F8DE
:108E0000045F9342FBD12822002104F13C0054F07E
:108E100029FA4FF000084FF0140C4FF0050E46FAF7
:108E20000EF303F00103002B0CBF0A27192743445C
:108E30001EF0010F0CEB07015FFA83F814BF284600
:108E4000002089B2634604EB830201339BB28B425C
:108E50005061F8D10EF1FF3E6744BEF1FF3F1FFAAB
:108E600087FCDCD118F0010F14BF19210A210CEB8B
:108E7000010080B2634604EB830201339BB283425C
:108E80005561F8D14A1E92B20CF1010313440CF162
:108E900002009BB205490433024492B204EB8303FF
:108EA0008A80002159602261BDE8F08154C9002008
:108EB00070B5094CA36873B10546002606E09968B1
:108EC0001A681E73A1609047A36823B15A68AA1A52
:108ED000002A1846F3DA70BD54C9002070B5214C41
:108EE0002378012B00D070BD1F4B1B68002BFAD0DC
:108EF0001E4D2B6828465B6898470028F3D01C4B12
:108F00001C4E1A68338892889A420ED21A4B1B4A1A
:108F10001B7852680021217003F00203002AE2D07E
:108F200091881268DBB9118370BD15490968002268
:108F30004968EA622A6803FB01F12846D36898472A
:108F40000E4A3388526801333380002ACBD013682D
:108F5000928859690A4214BF5A831A8370BD51839B
:108F600070BD00BF5E3D00209422002098220020AA
:108F7000583D00205C3D0020E0220020E42200203B
:108F8000503D002008B5254B1B68DB040AD5B5EE23
:108F9000400AF1EE10FA12D19FED210A53F0D2FCF3
:108FA00080B208BDDFED1F7AB4EEE70AF1EE10FAE9
:108FB0001CDA9FED1D0A53F0C5FC80B208BDDFED41
:108FC000197AB4EEE70AF1EE10FAE5D49FED177ABC
:108FD000B4EEC70AF1EE10FA14D870EE677A9FED7E
:108FE000147A9FED140AA7EE870AE4E770EE677A19
:108FF0009FED117A9FED110AA7EE870A53F0A2FCAC
:1090000080B208BDDFED0E7A9FED0E7A70EE677AC2
:109010009FED0D0AA7EE870ACDE700BFCC420020E6
:109020000080BB440000404200007A4400E08244DB
:1090300066BEFFBE0060BB4438DFFF3E00407A449E
:109040000000834466BEFF3E00A0BB442DE9F84308
:10905000CF4B1E6816F004072DED048B40F01F81E6
:109060009FEDCC8ACC4C16F0200605D094F8D86041
:1090700016F0020640F0AB8094F81131DFEDC78A9C
:1090800094F8102113F0010340F0B780002A40F05B
:109090009980D4ED457A9FEDC27ADFEDC26A67EE22
:1090A000877A94ED477AE8EE267A38EE477AC4ED6F
:1090B000457A84ED467A66B1012284F8122194F84B
:1090C0002421D4F8DC30C4F82031012A18BFC4F8B8
:1090D0001831B54B93F80080B8F10D0F0BD1D4EDDA
:1090E000377A9FEDB27AB24B67EE877AFDEEE77A78
:1090F00017EE902A9A809FEDA77AAE4DB0EE489A6F
:109100000023D4ED4C7AD4ED4D6A94ED4B8A37EEC2
:10911000677AE6EE877A37EEC87AC4ED4C7AA6EE27
:10912000878A85ED008A84ED4B8A0BB184ED468AEF
:1091300094ED4E7AD4ED507ADFED9F5AD4ED516A1A
:1091400094ED4F0A84ED4E8A38EE477AB0EE676AA6
:1091500097EE256AE6EE867A37EEC07AC4ED507A4D
:10916000A6EE870A84ED4F0A84ED520A53F0EAFB1B
:1091700002B282EAE273A3EBE2739BB2092B40F2E4
:10918000FC80002AACBF0A380A3005B2B8F10D0FD6
:10919000A4F84C5100F0CF80B8F1230F00F0E2802A
:1091A000B8F1370F05D1B0EE480A53F0CBFB804B36
:1091B0009880BDEC048B002E18BF374684F84E71A2
:1091C000BDE8F88384F8123184F8103161E7D4EDFA
:1091D0003A7AB4F8EC30F8EEE77AC4ED377A002B3F
:1091E0007DD1DFED6E8A94F8113194F8102113F0DF
:1091F00001034FF001063FF449AF002A67D0D4EDD8
:10920000479A694B94F8129193F8008038EE699A66
:10921000002E49D0B9F1000F73D094ED370AD4ED88
:10922000487A644D30EE670AB8F10D0F85ED000AFB
:1092300007D1DFED627A20EE270A53F083FB5C4B07
:10924000988094F82431002B40F0998095ED007AB5
:10925000002F3AD094F825319FED596A77EE487A7D
:1092600006EE903A77EEA97AF8EEE66AF0EEE77A43
:1092700067EEA67A3B46F4EEC67AF1EE10FAC4BF6A
:1092800028EE866AC6EE278AF7EE007A77EEE87A4D
:1092900067EE897AE8EE877AB0EE677A31E73E4C7E
:1092A000012794ED338ADEE6B8F10D0F37D0414D3A
:1092B000DFED388AB9F1000FC3D1002F64D094F8E4
:1092C0002431002B5ED1B0EE497A012319E7D4EDA9
:1092D000459A0123C4ED479A84F8103191E707EECF
:1092E000903ADFED356A9FED377AF8EEE77AC6EE11
:1092F000A78AF4EEC78AF1EE10FA88BFF0EE478A2B
:1093000071E7002F60D094ED370A70EE487A0123A0
:1093100077EEA97A84F81231C4ED487A81E7254DB9
:10932000DFED267A95ED000A20EE270A53F00AFBBE
:109330001F4B9880BCE7DFED207A9FED200ADFF815
:10934000708068EEA77A29EE000AFDEEE77A17EE44
:10935000903AA8F8003053F0F5FAA8F80650A8F8AB
:10936000020026E7DFED157A94ED460A20EE270A83
:1093700053F0E8FA0E4B58801BE7002506E7022B56
:1093800002D00FB1012B9ED095ED007A0123B8E6F3
:10939000ACB100200000000054C900209A99993E09
:1093A000CDCC4C3FCDCC4C3E4C2800200AD7233CA2
:1093B00050280020BC4A00200000C842CDCCCC3D43
:1093C00000401C466666663FB8F10D0F064DDBD1C6
:1093D000DFED067A95ED000A20EE270A53F0B2FA87
:1093E000034B9880D0E700BFBC4A0020CDCCCC3DD9
:1093F000502800202DE9F04F6B4B1B7887B0002BD5
:1094000000F0CB80694D6A48A968FAF71DF86968D1
:109410006848FAF719F8684B6848D3E90031C91A67
:10942000674B1A68B1FBF2F2FAF70EF8F9F748FF4A
:109430006448F9F75DFF6448F9F75AFF4FF00008F8
:10944000624B1B785FFA88F4A34222D8F9F738FF01
:109450005F4D604E002455F8041F30460134F9F783
:1094600093FF162CF7D1F9F72BFF5B4D594E0124D2
:109470002B4669681B683046C91A0134F9F784FF26
:10948000162C05F10405F3D107B0BDE8F04FF9F74C
:1094900017BF524B142603EB840306FB045693EDCF
:1094A000000AB6F80E9053F04DFA96F81EA01AF086
:1094B000010F0CBF2D2252221AF0020F0CBF2D23D8
:1094C00054231AF0040F0CBF4FF02D0C4FF0560C24
:1094D0001AF0080F0CBF4FF02D0E4FF0430E81B263
:1094E0001AF0800F4FF03C0BB1FBFBF105914FF0F0
:1094F00064010CBF4FF02D0A4FF0530A80B201FBFC
:1095000009F1671CCDE902A10490CDE900CE3448F1
:109510003946F9F739FFB37FDB073AD55C23314A87
:109520006343D118D05891ED010A70B1DFED2E7A66
:10953000B8EE400A20EE270A07EE900AF8EE677AA6
:1095400080EE270A53F0FEF900B2642290FBF2F19C
:1095500002FB11022548F9F717FF142101FB0757F9
:1095600001FB0454F988628A0491218B0391E18AFA
:109570000291A18B0191A18A009102F003031921AC
:109580004B431B48218A9208F9F75EFF08F1010856
:1095900056E71848F9F78CFEDFE7174807B0BDE833
:1095A000F04FF9F7A5BE00BF04000010000900103D
:1095B00005F5070815F50708100600102CF5070833
:1095C000D01A002059F50708B5F50708A80D0010B6
:1095D000A809001065F60708AC0900101C16001059
:1095E00011F607082006001000401C462EF607085A
:1095F00043F607083AF6070869F607082DE9F84F19
:1096000000261F4DDFF88090DFF880A007460C464B
:10961000B0462046FBF796FBD5F800B048B9214686
:109620005846F8F77DFA20B968682146F8F778FAC5
:1096300080B15846F9F73CFE696811B15046F9F718
:10964000A3FEA96811B14846F9F79EFEF9F738FE66
:109650004FF0010801363A2E05F11005D9D1204608
:10966000FBF770FB48B9B8F1000F06D12246384627
:109670000449BDE8F84FFAF7B9BCBDE8F88F00BF60
:10968000642F070891F607088BF6070885F6070888
:10969000F8B5384C2368002B57D00A2801D00D2884
:1096A00051D1354D95F84F310BB1F9F709FE334ED5
:1096B0002321304653F0EDFD08B1801B2060236864
:1096C000002273B902B12360F9F7C6FD95F84F3156
:1096D000F3B1BDE8F8402A48F9F7EABD01220B468C
:1096E000EFE7591E705C2028F8D092B90022254C73
:1096F000224FF2543B26013E0DD13146224B9C4273
:1097000012D2E3682068984795F85031002BDBD1DE
:10971000F8BD2360EAE721683846FEF717FA0146EC
:109720000028EBD11034E6E795F84F3123B1174903
:109730001748FAF749FBC7E71648F9F7B9FD0F488C
:10974000F9F7D6FDC0E7FF2BE2D8A0F120025E2A90
:10975000DED80BB92028DBD05A1C2260074AD0542F
:10976000054B93F84F31002BD2D0BDE8F840F9F704
:10977000E9BD00BF78B1002054C9002076B00020B8
:109780003FDE0708642F070804330708A5F607081B
:10979000C1F60708C7F60708F1F756BA10B5044630
:1097A00053F0D0F881B22046BDE81040F1F74CBA32
:1097B0002DE9F047A84C2DED048BA368204698476F
:1097C000002800F0BB80B4F90E30A17D06EE903A7F
:1097D000B4F9103007EE103AB4F9123007EE903AAF
:1097E000F8EEE66AB8EEC77AF8EEE77A0929C4ED32
:1097F000126A84ED137AC4ED147A00F0A380974EB8
:1098000004F148002BF05AFDB28DB36A002A40F0F3
:10981000A580934A934D1268520700F1E880B3F98E
:109820000020D4ED147A94ED128AD4ED138A06EE5A
:10983000102AB3F90220B3F9043006EE902A07EE9D
:10984000103A894B894A93F80080B4F8443092F872
:109850006E75B8EEC66AF8EEE66AB8EEC77A38EE0C
:10986000468A37EEC79A78EEE68A07EE903A338852
:1098700084ED128AF8EEE79AC4ED138A84ED149A07
:10988000002B40F0FF80B8F1040F00F0E88195ED67
:10989000606AD5ED616A95ED627A85ED608A38EE91
:1098A000466A78EEE66A39EE477A26EE296A66EE6F
:1098B000A96A27EE297A84ED156AC4ED166AC5ED0A
:1098C000618A84ED177A85ED629A94ED137AD4ED6E
:1098D000167A94ED126AD4ED156A27EE077A67EED0
:1098E000A77AA6EE067AB8F1040FE6EEA67A94ED12
:1098F000146AD4ED176AA6EE067AE6EEA67AB1EE01
:10990000C70AB1EEE77AD4ED006A26EE800A26EEA9
:10991000878A84ED180A84ED198A0CD1DFED548A08
:10992000544D20EE280A53F00DF828EE280AA8809E
:1099300053F008F82881012384F86830BDEC048BCB
:10994000BDE8F087454E04F1200104F148002BF0FA
:109950004FFCB28DB36A002A3FF45BAFB2F5C87F0B
:1099600000F061813F4DD4ED127A95ED557AD4ED3A
:10997000136A94ED146AB8EEC77A4FF0000C37EE14
:10998000277AD5ED567AC4F848C0F8EEE77ABDEEEE
:10999000C77A77EEA67AD5ED576A85ED557AF8EE57
:1099A000E66AFDEEE77A76EE866A17EE901AC5ED66
:1099B000567AFDEEE67A4FF0000E012AA3F800E099
:1099C00017EE100AC4F84CC017EE907AA3F802E024
:1099D000C5ED577AC4F850C0A3F804E000F0078240
:1099E000013AB2851E4A126852077FF518AFB5F8E2
:1099F0006021322A00F0C280002A40F0BB8195F835
:109A00007E21002A3FF40BAFDFF870C0D5F8782133
:109A1000B4F80CE0D5E95C178CFB0298D217C2EBC6
:109A20002812A2EB0E029A808CFB01E2C917C1EB4F
:109A3000221119808CFB0721FA17C2EB21125A80E0
:109A40000D4B00200122D881C3F80A2085F87E0141
:109A5000F9F78CFAB36AE2E6F4140010BC140010B3
:109A6000CC42002054C900204C2800202C0F0010AC
:109A700000007A44502800202CAE00201F85EB51B6
